:020000040800F2
:1000000000BF0020252E0208E1F10108E3F10108FC
:10001000E5F10108E7F10108E9F10108000000003D
:10002000000000000000000000000000EBF10108EB
:10003000EDF1010800000000EFF10108F1F1010805
:10004000A1330208A5330208A9330208AD33020820
:10005000B1330208B5330208B9330208BD330208D0
:100060005BC9000873F20108C9330208CD330208E6
:10007000D13302089DF20108D933020847F2010882
:10008000E1330208A9F20108E9330208ED3302085E
:10009000F1330208F5330208F9330208FD33020890
:1000A0000134020805340208093402080D3402083C
:1000B000113402081534020819340208575A01088D
:1000C0006F5A010825340208293402082D34020829
:1000D000313402083534020885F201083D34020843
:1000E0005FF2010845340208493402084D34020821
:1000F0002BF2010855340208593402085D34020815
:100100006134020865340208F3F101086D34020815
:1001100091F2010875340208793402080FF20108DF
:100120008134020853F20108893402088D34020830
:100130009134020895340208993402089D3402086B
:10014000A1340208A5340208A9340208B5F2010856
:10015000B1340208B5340208B9340208BD340208CB
:10016000C1340208C5340208C9340208CD3402087B
:10017000D1340208D5340208D9340208DD3402082B
:10018000E1340208E534020810B504000021200023
:1001900000F095F8002084F80E0114F50570DFF8E2
:1001A000A413D1E90023C0E9002314F50770DFF898
:1001B0009813D1E90023C0E9002314F50970DFF892
:1001C0008C13D1E90023C0E9002314F50B70DFF88C
:1001D0008013D1E90023C0E9002314F50D70DFF886
:1001E0007413D1E90023C0E9002314F50F70DFF880
:1001F0006813D1E90023C0E9002314F51170DFF87A
:100200005C13D1E90023C0E9002314F51370DFF873
:100210005013D1E90023C0E9002314F51570DFF86D
:100220004413D1E90023C0E9002314F51770DFF867
:100230003813D1E90023C0E9002314F51970DFF861
:100240002C13D1E90023C0E9002314F51B70DFF85B
:100250002013D1E90023C0E9002314F51D70DFF855
:100260001413D1E90023C0E9002314F51F70DFF84F
:100270000813D1E90023C0E9002314F52170DFF849
:10028000FC12D1E90023C0E9002314F52370DFF844
:10029000F012D1E90023C0E9002314F52570DFF83E
:1002A000E412D1E90023C0E90023DFF83408046038
:1002B000200010BDDFF8281800220A6070470022D5
:1002C000A0F80C210022A0F80021002280F80A21C9
:1002D0000022A0F802210022A0F804210022A0F8A8
:1002E0000621C9B2002902D0012180F8B41270475A
:1002F00080B54FF4887200210BF0A2FEDFF8EC0706
:100300000021018601BD10B4DFF8183D1B78002BD9
:1003100024D090F81232002B20D10023A0F8103204
:100320000CE0B0F810321B18B0F81042645C83F88F
:100330001041B0F810325B1CA0F81032B0F8103247
:1003400092B2934203D2B0F81032FF2BE9DBB0F83F
:100350001012002902D0012180F8121210BC70473F
:1003600004E0B0F80611491CA0F80611B0F8061117
:10037000095C00290BD0B0F80611B0F800219142B9
:1003800005D2B0F80611095CC9B22029E9D0B0F84D
:100390000011B0F80621891AA0F80811B0F8080178
:1003A000704710B404E0B0F80621521CA0F80621F2
:1003B000B0F80621125C002A0BD0B0F80621B0F884
:1003C00000319A4205D2B0F80621135CDBB2202B33
:1003D000E9D00022A0F80821B0F8062105E0B0F825
:1003E00008315B1CA0F80831521C92B2135C002B40
:1003F00014D0B0F8003192B29A420FD292B2135C8C
:10040000C9B2002907D0DBB2B3F141041A2C02D2E1
:10041000203392B21354DBB2202BE0D1B0F80801A4
:1004200010BC7047B0F80611B0F808215118A0F8B8
:100430000611704738B504000D0028000BF00AFEC5
:10044000B4F8081180B2884201D000200CE080B2DC
:1004500002002900B4F8060100190BF02DFE002857
:1004600001D1012000E0002032BD38B50400002099
:10047000B4F8081100291AD0B4F80601B4F808112C
:1004800011FA80F0055DB4F80601B4F8081111FA0C
:1004900080F000210155B4F8060100190BF03DFE73
:1004A000B4F80611B4F8082112FA81F10D5532BDE5
:1004B00038B504009FED210AB4F8080100282AD0BD
:1004C000B4F80601B4F8081111FA80F0055DB4F82B
:1004D0000601B4F8081111FA80F00021015500213D
:1004E000B4F8060100190BF01CFE51EC100B0BF0D8
:1004F0001FFE00EE100ADFED120AB4EE600AF1EE04
:1005000010FA01D19FED0D0AB4F80601B4F80811F4
:1005100011FA80F0055531BD10B50400DFF8880CE4
:100520000BF098FD020092B2DFF87C1C2000FFF770
:10053000EAFE012084F8B402012010BD0000000092
:10054000FFFFFF7FC4320208CC320208D432020817
:10055000DC320208E4320208EC320208F43202080B
:10056000FC320208043302080C3302081433020878
:100570001C330208243302082C33020834330208E7
:100580003C3302084433020810B50400B4F80401F7
:10059000042801D0002010BD0422DFF88C1AB4F822
:1005A000020100190BF088FD002840F02982DFF8D5
:1005B0007C0A0BF04FFD0100DFF8700A0BF000FE23
:1005C000DFF86C0A0BF046FD0100DFF8640A0BF05F
:1005D000F7FDDFF8480B0BF03DFD0100DFF83C0BA9
:1005E0000BF0EEFDDFF8380B0BF034FD0100DFF807
:1005F000300B0BF0E5FDDFF82C0B0BF02BFD0100B1
:10060000DFF8200B0BF0DCFD4FF4FA600BF024FE5A
:10061000DFF8140B0BF01EFD0100DFF80C0B0BF0E4
:10062000CFFDDFF8080B0BF015FD0100DFF8FC0A29
:100630000BF0C6FDDFF8F80A0BF00CFD0100DFF847
:10064000F00A0BF0BDFDDFF8640B0BF003FD0100B9
:10065000DFF8580B0BF0B4FDDFF8540B0BF0FAFC8D
:100660000100DFF84C0B0BF0ABFDDFF8480B0BF093
:10067000F1FC0100DFF83C0B0BF0A2FD4FF4FA6037
:100680000BF0EAFDDFF8300B0BF0E4FC0100DFF8C3
:10069000280B0BF095FDDFF8240B0BF0DBFC0100C1
:1006A000DFF8180B0BF08CFDDFF8140B0BF0D2FC0D
:1006B0000100DFF80C0B0BF083FDDFF8080B0BF0EB
:1006C000C9FC0100DFF8FC0A0BF07AFDDFF8F80A3C
:1006D0000BF0C0FC0100DFF8F00A0BF071FD4FF4E5
:1006E000FA600BF0B9FDDFF8E40A0BF0B3FC01008F
:1006F000DFF8D80A0BF064FDDFF8D40A0BF0AAFC8F
:100700000100DFF8CC0A0BF05BFDDFF8C80A0BF044
:10071000A1FC0100DFF8BC0A0BF052FD4FF4FA60B7
:100720000BF09AFDDFF8B00A0BF094FC0100DFF843
:10073000A80A0BF045FDDFF8A40A0BF08BFC0100C2
:10074000DFF8980A0BF03CFDDFF8940A0BF082FC0E
:100750000100DFF88C0A0BF033FDDFF8780B0BF0AB
:1007600079FC0100DFF86C0B0BF02AFD4FF4FA6006
:100770000BF072FDDFF8640B0BF06CFC0100DFF88E
:100780005C0B0BF01DFDDFF8580B0BF063FC010058
:10079000DFF84C0B0BF014FDDFF8480B0BF05AFCA4
:1007A0000100DFF8400B0BF00BFDDFF83C0B0BF00A
:1007B00051FC0100DFF8300B0BF002FD4FF4FA6042
:1007C0000BF04AFDDFF8240B0BF044FC0100DFF8CE
:1007D0001C0B0BF0F5FCDFF8180B0BF03BFC0100D9
:1007E000DFF80C0B0BF0ECFCDFF8080B0BF032FC25
:1007F0000100DFF8000B0BF0E3FCDFF8FC0A0BF064
:1008000029FC0100DFF8F00A0BF0DAFCDFF8EC0A53
:100810000BF020FC0100DFF8E40A0BF0D1FC4FF4F0
:10082000FA600BF019FDDFF8D80A0BF013FC010099
:10083000DFF8CC0A0BF0C4FCDFF8C80A0BF00AFCA6
:100840000100DFF8C00A0BF0BBFCDFF8BC0A0BF0BC
:1008500001FC0100DFF8B00A0BF0B2FCDFF8AC0AD3
:100860000BF0F8FB0100DFF8A40A0BF0A9FCDFF89D
:10087000A00A0BF0EFFB0100DFF8940A0BF0A0FCDC
:10088000DFF8900A0BF0E6FB0100DFF8880A0BF0B6
:1008900097FC4FF4FA600BF0DFFCDFF87C0A0BF0FA
:1008A000D9FB0100DFF8700A0BF08AFCDFF86C0A54
:1008B0000BF0D0FB0100DFF8640A0BF081FCDFF8DD
:1008C000600A0BF0C7FB0100DFF8540A0BF078FC5C
:1008D000DFF8500A0BF0BEFB0100DFF8480A0BF00E
:1008E0006FFCDFF8440A0BF0B5FB0100DFF8380AB3
:1008F0000BF066FCDFF8340A0BF0ACFB0100DFF80C
:100900002C0A0BF05DFC4FF4FA600BF0A5FCDFF84D
:10091000200A0BF09FFB0100DFF8140A0BF050FCDB
:10092000DFF8B40B0BF096FB0100DFF8AC0B0BF01B
:1009300047FCDFF8A80B0BF08DFB0100DFF89C0BE8
:100940000BF03EFCDFF89C0B0BF084FB0100DFF8A2
:10095000940B0BF035FC4FF4FA600BF07DFCDFF8E4
:10096000880B0BF077FB0100DFF87C0B0BF028FC09
:10097000DFF8780B0BF06EFB0100DFF8700B0BF06B
:100980001FFCDFF86C0B0BF065FB0100DFF8600B60
:100990000BF016FCDFF85C0B0BF05CFB0100DFF8E2
:1009A000540B0BF00DFCDFF8500B0BF053FB010068
:1009B000DFF8440B0BF004FC4FF4FA600BF04CFC36
:1009C000DFF8380B0BF046FB0100DFF8300B0BF0C3
:1009D000F7FBDFF82C0B0BF03DFB0100DFF8200BE1
:1009E0000BF0EEFBDFF81C0B0BF034FB0100DFF823
:1009F000140B0BF0E5FB012084F8B4020120CAE5DA
:100A00000020C8E510B59CB00400B4F80401032828
:100A100002D000201CB010BD032233A1B4F80201A3
:100A200000190BF049FB002857D1DFF8DC0A0290CF
:100A30004FF48C7001900020009001230022DFF819
:100A4000CC1A03A80BF076FC03A80BF003FB010003
:100A500003A80BF0B5FB234890F88801022819D1B0
:100A600023480068B0F8F60000902148006890F82C
:100A7000F5301F48006890F8F420DFF8941A03A8B6
:100A80000BF058FC03A80BF0E5FA010003A80BF0EB
:100A900097FB1DE0134890F88801012818D11448ED
:100AA0000068B0F8F60000901148006890F8F53042
:100AB0000F48006890F8F420DFF8581A03A80BF0EC
:100AC00039FC03A80BF0C6FA010003A80BF078FB71
:100AD000012084F8B40201209CE700209AE700007E
:100AE00048B40020101800107665720058330010CA
:100AF00044B4002010B50400B4F80401032801D068
:100B0000002038E20322D3A1B4F8020100190BF04F
:100B1000D3FA002840F02E8201212000FFF741FC8B
:100B2000002803D10020002800F01982D4A1200061
:100B3000FFF780FC002803D10020002800F0FF8090
:100B40002000FFF76FFC01212000FFF72AFC00289E
:100B500003D10020002800F0E680DFF8BC19200057
:100B6000FFF768FC002802D10020002808D0DFF839
:100B7000AC09006850F00200DFF8A0190860EEE14F
:100B8000DFF89C192000FFF755FC002802D1002057
:100B9000002808D0DFF88409006850F00100DFF871
:100BA0007C190860DBE1CBA12000FFF743FC0028A3
:100BB00002D10020002808D0DFF86009006850F05A
:100BC0000400DFF858190860C9E1DFF8581920005F
:100BD000FFF730FC002802D10020002808D0DFF801
:100BE0003C09006850F00800DFF830190860B6E1F1
:100BF000DFF834192000FFF71DFC002802D1002087
:100C0000002808D0DFF81409006850F01000DFF861
:100C10000C190860A3E1CBA12000FFF70BFC002812
:100C200002D10020002808D0DFF8F008006850F05A
:100C30002000DFF8E818086091E1CFA12000FFF75D
:100C4000F9FB002802D10020002808D0DFF8CC08EA
:100C5000006850F04000DFF8C41808607FE1DFF85A
:100C6000CC182000FFF7E6FB002802D10020002866
:100C700008D0DFF8A808006850F48060DFF89C18FE
:100C800008606CE1DFF8A8182000FFF7D3FB00280C
:100C900002D10020002808D0DFF88008006850F05A
:100CA0008000DFF87818086059E1DFF88818200024
:100CB000FFF7C0FB002802D10020002808D0DFF891
:100CC0005C08006850F48070DFF85018086046E156
:100CD000DFF864182000FFF7ADFB002802D10020E8
:100CE000002808D0DFF83408006850F40070DFF8FE
:100CF0002C18086033E1DFF844182000FFF79AFB56
:100D0000002840F02C810020002840F02881DFF8E6
:100D100030080BF09FF9020092B2DFF8241820008F
:100D2000FFF7F1FA1BE1DFF818080BF093F9020066
:100D300092B2DFF80C182000FFF7E5FA0FE18FA15F
:100D40002000FFF777FB002803D10020002800F0E7
:100D5000FB802000FFF766FB01212000FFF721FB4D
:100D6000002803D10020002800F0E680DFF8B0174B
:100D70002000FFF75FFB002802D10020002808D0E8
:100D8000DFF89807006840084000DFF89017086017
:100D9000E5E050A12000FFF74DFB002802D1002024
:100DA000002808D0DFF87407006830F00400DFF88E
:100DB0006C170860D3E0DFF860172000FFF73AFBFC
:100DC000002802D10020002808D0DFF85007006872
:100DD00030F00200DFF844170860C0E0DFF8441785
:100DE0002000FFF727FB002802D10020002808D0B0
:100DF000DFF82807006830F00800DFF820170860E7
:100E0000ADE0DFF824172000FFF714FB002802D123
:100E10000020002808D0DFF80407006830F0100038
:100E2000DFF8F81608609AE046A12000FFF702FB01
:100E3000002802D10020002808D0DFF8E006006872
:100E400030F02000DFF8D416086088E0DFF8E01604
:100E500002E000BF6D6F6E002000FFF7EBFA002884
:100E600002D10020002808D0DFF8B006006830F07A
:100E70008000DFF8A816086071E03FA102E000BF23
:100E80006F6E00002000FFF7D5FA002802D1002085
:100E9000002808D0DFF88406006830F04000DFF852
:100EA0007C1608605BE0DFF884162000FFF7C2FACA
:100EB000002802D10020002808D0DFF86006006872
:100EC00030F48060DFF85416086048E0DFF86416FC
:100ED00002E000BF6D6167002000FFF7ABFA002859
:100EE00002D10020002808D0DFF83006006830F476
:100EF0008070DFF82816086031E0DFF83C1620002B
:100F0000FFF798FA002802D10020002808D0DFF867
:100F10000C06006830F40070DFF8001608601EE070
:100F2000DFF81C060BF096F8020092B2DFF81016FC
:100F30002000FFF7E8F912E0DFF8E005002101608A
:100F40000DE000BF656B6600DFF8F4050BF082F87A
:100F5000020092B2DFF8E8152000FFF7D4F9DFF8BD
:100F6000D00A00680021C0F86011012084F8B402A2
:100F7000012000E0002010BD677073006F666600FE
:100F800010B50400B4F80401042801D0002047E0A3
:100F90000422DFF8A01AB4F8020100190BF08CF853
:100FA00000283CD101212000FFF7FBF9002802D1E5
:100FB0000020002828D07AA12000FFF73BFA002863
:100FC00002D10020002805D0DFF850050021A0F84C
:100FD000E41419E073A12000FFF72CFA002802D1D5
:100FE0000020002805D0DFF834050121A0F8E41422
:100FF0000AE0DFF84C050BF02DF8020092B2DFF8A2
:1010000040152000FFF77FF9DFF8240A006800216F
:10101000C0F86011012084F8B402012000E0002033
:1010200010BD0000B1B40020C4310208E82002085D
:101030004816020810B5B2B00400B4F8040108283C
:1010400001D0002068E00822DFF8EC19B4F80201B2
:1010500000190BF031F800285DD101212000FFF7C5
:10106000A0F9002802D10020002852D0DFF8CC19C6
:101070002000FFF7DFF9002802D10020002819D056
:10108000DFF898040121A0F8E6142000FFF730F9FA
:10109000DFF8AC1900A80BF04DF900A80AF0DAFF50
:1010A000020092B200A92000FFF72DF9002084F879
:1010B000B4022EE0DFF88C192000FFF7BBF90028FE
:1010C00002D10020002816D0DFF850040021A0F83B
:1010D000E814DFF8741900A80BF02CF900A80AF046
:1010E000B9FF020092B200A92000FFF70CF901201D
:1010F00084F8B4020DE0DFF848040AF0ABFF020008
:1011000092B2DFF83C142000FFF7FDF8012084F8CC
:10111000B402012000E0002032B010BD3805020802
:10112000EC000208200902086005020820030208FA
:10113000C8F6010810B592B00400B4F804010628FE
:1011400002D0002012B010BD0622DFF80019B4F85A
:10115000020100190AF0B0FF00281FD101A9DFF831
:10116000F00800680BF072F99DF8060000909DF8F9
:1011700005309DF80420DFF8DC1802A80BF0DAF83F
:1011800002A80AF067FF020092B202A92000FFF74E
:10119000BAF8012084F8B4020120D3E70020D1E797
:1011A0006F6666006F6E000040F8010820FB0108C2
:1011B000D8F401081C0102084C0102084C03020883
:1011C00078030208ECFD010820FE010808FC010874
:1011D00054FE010868FA010888F8010888FE010831
:1011E0008805020838B504000025B4F80401032876
:1011F00001D000206DE0032237A1B4F802010019EC
:101200000AF05AFF002863D101212000FFF7C9F836
:10121000002802D10020002848D0C1492000FFF753
:1012200009F9002802D10020002803D0BB48012181
:1012300081713CE0B8492000FFF7FCF8002802D19A
:101240000020002801D0012531E0A2A12000FFF7F5
:10125000F1F8002802D10020002803D0AF48012176
:10126000C17124E0DFF8F0172000FFF7E3F8002851
:1012700002D10020002806D0A848C07950F0040010
:10128000A649C87113E0DFF8D4172000FFF7D2F8A1
:10129000002802D10020002806D0A048C07910F014
:1012A000F8009E49C87102E0012500E00125EDB279
:1012B000002D0BD0A2480AF0CDFE020092B2A04948
:1012C0002000FFF720F8012084F8B402012000E09C
:1012D000002032BD40FC010863616C00BCFE0108C7
:1012E000F0FE0108B00502087C01020818F90108A7
:1012F000AC010208DC01020824FF01080C0202080C
:10130000D805020878FC010858FF0108A403020868
:101310008CFF0108C0FF0108C8F301082CF5010883
:1013200080F50108D4F501085CF901085CFB0108AF
:1013300014F7010830B5BFB004000025B4F804016B
:10134000042802D000203FB030BD0422DFF810177F
:10135000B4F8020100190AF0AFFE002840F0B8808E
:1013600001212000FFF71DF8002803D100200028EC
:1013700000F09C805AA12000FFF75CF8002802D101
:101380000020002841D00121DFF8A40600680BF0FE
:101390003BFF6248C06B0BF099FFCDE90A015F4843
:1013A000006B0BF093FFCDE908015C48C06A0BF0BD
:1013B0008DFFCDE906015948806A0BF087FFCDE922
:1013C00004015648406A0BF081FFCDE90201534801
:1013D000006A0BF07BFFCDE900015048C0690BF0BB
:1013E00075FF02000B00DFF87C160CA80AF0A2FFC4
:1013F0000CA80AF02FFE020092B20CA92000FEF702
:1014000082FF012084F8B40251E0DFF85C1620006E
:10141000FFF710F8002802D10020002817D0DFF8CD
:101420004C0600680CF0A6F90200DFF844160CA880
:101430000AF080FF0CA80AF00DFE020092B20CA97F
:101440002000FEF760FF012084F8B4022FE0DFF8EF
:1014500024162000FEF7EEFF002802D1002000280D
:1014600022D0DFF8080600680CF0F6FEC0B20028B3
:1014700002D10020002805D0DFF8FC150CA80AF0E6
:1014800059FF04E0DFF8F4150CA80AF053FF0CA88C
:101490000AF0E0FD020092B20CA92000FEF733FF33
:1014A000012084F8B40202E0012500E00125EDB23C
:1014B000002D0BD022480AF0CDFD020092B2204947
:1014C0002000FEF720FF012084F8B40201203AE753
:1014D000002038E76D61670060F7010828F6010811
:1014E00072656600A0F901083C0202086C0202085D
:1014F000F4FF01082800020878F60108ACF701089B
:10150000D0F80108B0FC0108342E0208D0FB010815
:10151000FC08020810050208CC310208101800105F
:10152000D4310208DC310208E4310208EC3102084F
:10153000F4310208402E02084C2E0208FC31020849
:10154000D808020830B5B3B004000025B4F804018F
:10155000052802D0002033B030BD0522DFF8201569
:10156000B4F8020100190AF0A7FD002840F0068235
:1015700001212000FEF715FF002803D100200028DC
:1015800000F0EA81DFF8FC142000FEF753FF00288A
:1015900003D10020002800F005812000FEF742FF63
:1015A00001212000FEF7FDFE002803D100200028C5
:1015B00000F0F680C3A12000FEF73CFF002802D116
:1015C0000020002842D000202BE080B2DFF8B814C1
:1015D00011EBC001002281F8E82180B2DFF8A814E5
:1015E00011EBC001002281F8E92180B2DFF89814E4
:1015F00011EBC0014FF47A72A1F8EA2180B2DFF852
:10160000881411EBC0014FF4FA62A1F8EC2180B20A
:10161000DFF8741411EBC00140F2DC52A1F8EE21A6
:10162000401C80B21828D0DBDFF8601400A80AF054
:1016300081FE00A80AF00EFD020092B200A920006F
:10164000FEF761FE012084F8B40286E1CCA12000FF
:10165000FEF7F0FE002802D10020002842D0002032
:101660002BE080B2DFF8201411EBC001002281F8DA
:10167000A82280B2DFF8101411EBC001002281F81B
:10168000A92280B2DFF8001411EBC0014FF47A7286
:10169000A1F8AA2280B2DFF8F01311EBC0014FF4D9
:1016A000FA62A1F8AC2280B2DFF8DC1311EBC001C2
:1016B00040F2DC52A1F8AE22401C80B21828D0DBE8
:1016C000DFF8C81300A80AF035FE00A80AF0C2FC33
:1016D000020092B200A92000FEF715FE012084F856
:1016E000B4023AE1DFF8A8132000FEF7A3FE0028B9
:1016F00002D10020002851D000200FE089B280B232
:101700000A22DFF8843302FB00328A18002382F8B1
:101710006833491C89B20A29F0DB401C80B21028CA
:1017200001DA0021F6E7DFF86003642180F868132E
:10173000DFF85403642180F87313D348642180F8E0
:101740007E13D148642180F88913CF48642180F842
:101750009413CD48642180F89F13CB48642180F80E
:10176000AA13C948642180F8B513C748642180F8DA
:10177000C013C548642180F8CB13C44900A80AF0FF
:10178000D9FD00A80AF066FC020092B200A9200070
:10179000FEF7B9FD012084F8B402DEE00125DCE0AB
:1017A0000125DAE0BB492000FEF744FE002802D103
:1017B0000020002810D0B84900A80AF0BBFD00A8FE
:1017C0000AF048FC020092B200A92000FEF79BFD3F
:1017D000012084F8B402C0E093A12000FEF72AFEA5
:1017E000002802D10020002812D00EF0DFFEAB4905
:1017F00000A80AF09FFD00A80AF02CFC020092B29B
:1018000000A92000FEF77FFD012084F8B402A4E0C7
:1018100086A12000FEF70EFE002802D1002000283D
:1018200022D00EF0D5FD9E4800680FF08DFA9D483D
:1018300000680FF05FFE9B4800680FF0E9FE9A48D1
:1018400000680FF0C1FF994900A80AF073FD00A8D5
:101850000AF000FC020092B200A92000FEF753FD3E
:10186000012084F8B40278E07F492000FEF7E2FD11
:10187000002802D10020002826D00EF0DAFA0EF05F
:10188000A7FD874800680FF05FFA864800680FF0F0
:1018900031FE844800680FF0BBFE834800680FF0FB
:1018A00093FF834900A80AF045FD00A80AF0D2FB87
:1018B000020092B200A92000FEF725FD012084F865
:1018C000B4024AE0696E00007A492000FEF7B2FDDA
:1018D000002802D1002000283CD0644800680BF0AA
:1018E0002BFD754900A80AF025FD00A80AF0B2FBFF
:1018F000010000A80AF064FC5C4800680CF000FDE0
:10190000C0B2002802D10020002812D05748006839
:101910000BF012FF0200694900A80AF00BFD00A8B5
:101920000AF098FB020092B200A92000FEF7EBFC3F
:101930000CE0634900A80AF0FDFC00A80AF08AFB4D
:10194000020092B200A92000FEF7DDFC012084F81D
:10195000B40202E0012500E00125EDB2002D0BD01C
:1019600058480AF077FB020092B256492000FEF771
:10197000CAFC012084F8B4020120ECE50020EAE56D
:101980006F75740030B5B3B004000025B4F80401DD
:10199000052802D0002033B030BD05224A49B4F8F2
:1019A000020100190AF088FB00283BD10121200028
:1019B000FEF7F7FC002802D10020002820D0434980
:1019C0002000FEF737FD002802D10020002815D0A6
:1019D00029213F48006810F03FFA3E4900A80AF06C
:1019E000A9FC00A80AF036FB020092B200A9200070
:1019F000FEF789FC012084F8B40202E0012500E032
:101A00000125EDB2002D0BD02E480AF023FB020079
:101A100092B22C492000FEF776FC012084F8B40233
:101A20000120B8E70020B6E76F736400696D7500A8
:101A30005CB40020B43202084C310208583102086C
:101A4000F8F70108BC320208B408020804320208A0
:101A500080B40020D0030208582E0208642E020829
:101A60000C320208E8F201081432020854B40020D3
:101A7000E8FC0108702E02085C000208140E02083F
:101A8000A43202081C320208101800103431020877
:101A900024320208F431020840290208F415020831
:101AA00060B4002068B4002050B4002084FD010818
:101AB00028FA01085C32020810160208B8FD010875
:101AC0002C160208D8080208AC320208D42D0208ED
:101AD00074B4002040310208F0B5B7B0040000250E
:101AE000B4F80401032802D0002037B0F0BD03226F
:101AF00048A1B4F8020100190AF0DEFA002842F009
:101B0000978601212000FEF74CFC002803D100201D
:101B1000002802F07A86DFF8881D2000FEF78AFC94
:101B2000002802D1002000281CD0DFF8780D0068C2
:101B3000D0F89C31DFF86C0D0068D0F89821DFF800
:101B4000681D05A80AF0F6FB05A80AF083FA020052
:101B500092B205A92000FEF7D6FB012084F8B4025A
:101B600002F054BEDFF89C1E2000FEF763FC002844
:101B700002D1002000281FD0DFF88C0EB0F914002D
:101B80000090DFF8840EB0F91230DFF87C0EB0F967
:101B90001020DFF8781E05A80AF0CCFB05A80AF093
:101BA00059FA020092B205A92000FEF7ACFB012011
:101BB00084F8B40202F02ABE17A12000FEF73AFC16
:101BC000002802D10020002828D0DFF83C0EB0F910
:101BD0001A000190DFF8300EB0F918000090DFF81D
:101BE000280EB0F91630DFF8AC0E00680278DFF886
:101BF000A81E05A80AF09EFB05A80AF02BFA020011
:101C000092B205A92000FEF77EFB012084F8B40201
:101C100002F0FCBD636174006D616700D8A1200013
:101C2000FEF708FC002803D10020002800F01386EE
:101C3000DFF8D40D807B0190DFF8CC0D8089009017
:101C4000DFF8C40D837ADFF8C00D0289DFF8B81E13
:101C500005A80AF06FFB05A80AF0FCF9010005A829
:101C60000AF0AEFADFF8A00D90F8C924DFF89C1E48
:101C700005A80AF05FFB05A80AF0ECF9010005A829
:101C80000AF09EFADFF8800D90F8CB24DFF8801E72
:101C900005A80AF04FFB05A80AF0DCF9010005A829
:101CA0000AF08EFADFF8600D90F88000C00701D5C9
:101CB000012200E00022D2B2DFF8581E05A80AF087
:101CC00039FB05A80AF0C6F9010005A80AF078FA60
:101CD000DFF8340D90F88000800701D5012200E084
:101CE0000022D2B2DFF88C1E05A80AF023FB05A85B
:101CF0000AF0B0F9010005A80AF062FADFF8080D51
:101D000090F88000400701D5012200E00022D2B205
:101D1000DFF8641E05A80AF00DFB05A80AF09AF981
:101D2000010005A80AF04CFADFF8DC0CD0F88000BE
:101D3000800301D5012200E00022D2B2DFF83C1E70
:101D400005A80AF0F7FA05A80AF084F9010005A829
:101D50000AF036FADFF8B00C90F88000000701D5E1
:101D6000012200E00022D2B2DFF8141E05A80AF01A
:101D7000E1FA05A80AF06EF9010005A80AF020FAB8
:101D8000DFF8840C90F88000C00601D5012200E045
:101D90000022D2B2DFF8EC1D05A80AF0CBFA05A8A4
:101DA0000AF058F9010005A80AF00AFADFF8580C01
:101DB00090F88000800601D5012200E00022D2B216
:101DC000DFF8C81D05A80AF0B5FA05A80AF042F91F
:101DD000010005A80AF0F4F9DFF82C0C90F8800057
:101DE000400601D5012200E00022D2B2DFF8A01D9A
:101DF00005A80AF09FFA05A80AF02CF9010005A829
:101E00000AF0DEF9DFF8000C90F88000000601D53A
:101E1000012200E00022D2B2DFF8781D05A80AF006
:101E200089FA05A80AF016F9010005A80AF0C8F910
:101E3000DFF8D40BD0F88000C00501D5012200E006
:101E40000022D2B2DFF8501D05A80AF073FA05A8E7
:101E50000AF000F9010005A80AF0B2F9DFF8A80BB2
:101E6000D0F88000800501D5012200E00022D2B226
:101E7000DFF8281D05A80AF05DFA05A80AF0EAF8BF
:101E8000010005A80AF09CF9DFF87C0BD0F880006F
:101E9000400501D5012200E00022D2B2DFF8041D86
:101EA00005A80AF047FA05A80AF0D4F8010005A829
:101EB0000AF086F9DFF8500BD0F88000000501D554
:101EC000012200E00022D2B2DFF8DC1C05A80AF0F3
:101ED00031FA05A80AF0BEF8010005A80AF070F969
:101EE000DFF8240BD0F88000C00401D5012200E007
:101EF0000022D2B2DFF8DC1D05A80AF01BFA05A803
:101F00000AF0A8F8010005A80AF05AF9DFF8F80A63
:101F1000D0F88000800401D5012200E00022D2B276
:101F2000DFF8B41D05A80AF005FA05A80AF092F832
:101F3000010005A80AF044F9DFF8CC0AD0F88000C7
:101F4000400401D5012200E00022D2B2DFF88C1D4E
:101F500005A80AF0EFF905A80AF07CF8010005A829
:101F60000AF02EF9DFF8A00AD0F88000000401D5AD
:101F7000012200E00022D2B2DFF8641D02E000BFBF
:101F80006F73640005A80AF0D5F905A80AF062F895
:101F9000010005A80AF014F9DFF86C0AD0F88000F7
:101FA000C00301D5012200E00022D2B2DFF8341DC7
:101FB00005A80AF0BFF905A80AF04CF8010005A829
:101FC0000AF0FEF8DFF8400AD0F88000400301D59F
:101FD000012200E00022D2B2DFF80C1D05A80AF0B1
:101FE000A9F905A80AF036F8010005A80AF0E8F8F2
:101FF000DFF8140AD0F88000000301D5012200E0C8
:102000000022D2B2DFF8E81C05A80AF093F905A86F
:102010000AF020F8010005A80AF0D2F8DFF8E80974
:10202000D0F88000C00201D5012200E00022D2B227
:10203000DFF8C41C05A80AF07DF905A80AF00AF823
:10204000010005A80AF0BCF8DFF8BC09D0F8800050
:10205000800201D5012200E00022D2B2DFF89C1CF0
:1020600005A80AF067F905A809F0F4FF010005A822
:102070000AF0A6F8DFF8900990F8CA24DFF8841C6B
:1020800005A80AF057F905A809F0E4FF010005A822
:102090000AF096F8DFF8700990F8CC24DFF8681C95
:1020A00005A80AF047F905A809F0D4FF010005A822
:1020B0000AF086F84FF4FA600AF0CEF8DFF8480923
:1020C000D0F8080483B2DFF84009D0F80804020C05
:1020D000DFF8381C05A80AF02DF905A809F0BAFFA9
:1020E000010005A80AF06CF8DFF81C09D0F80C0410
:1020F00083B2DFF81409D0F80C04020CDFF8101CCE
:1021000005A80AF017F905A809F0A4FF010005A821
:102110000AF056F8DFF8F008D0F8380483B2DFF898
:10212000E808D0F83804020CDFF8E81B05A80AF02C
:1021300001F905A809F08EFF010005A80AF040F892
:10214000DFF8C408D0F81C0483B2DFF8BC08D0F86C
:102150001C04020CDFF8C01B05A80AF0EBF805A868
:1021600009F078FF010005A80AF02AF8DFF89808BE
:10217000D0F8200483B2DFF89008D0F82004020CD5
:10218000DFF8981B05A80AF0D5F805A809F062FF4A
:10219000010005A80AF014F8DFF86C08D0F818045C
:1021A00083B2DFF86408D0F81804020CDFF8701B63
:1021B00005A80AF0BFF805A809F04CFF010005A822
:1021C00009F0FEFFDFF84008D0F8240483B2DFF8FE
:1021D0003808D0F82404020CDFF8481B05A80AF0E0
:1021E000A9F805A809F036FF010005A809F0E8FFE5
:1021F000DFF81408D0F8280483B2DFF80C08D0F810
:102200002804020CDFF8201B05A80AF093F805A8A3
:1022100009F020FF010005A809F0D2FFDFF8E80768
:10222000D0F82C0483B2DFF8E007D0F82C04020CBD
:10223000DFF8F81A05A80AF07DF805A809F00AFFEA
:10224000010005A809F0BCFFDFF8BC07D0F8300496
:1022500083B2DFF8B407D0F83004020CDFF8D01AEC
:1022600005A80AF067F805A809F0F4FE010005A822
:1022700009F0A6FFDFF89007D0F8340483B2DFF846
:102280008807D0F83404020CDFF8A81A05A80AF071
:1022900051F805A809F0DEFE010005A809F090FF3D
:1022A000DFF86407D0F83C0483B2DFF85C07D0F8AD
:1022B0003C04020CDFF8801A05A80AF03BF805A8D8
:1022C00009F0C8FE010005A809F07AFFDFF8380719
:1022D000D0F8100483B2DFF83007D0F81004020CF5
:1022E000DFF8581A05A80AF025F805A809F0B2FE8B
:1022F000010005A809F064FFDFF80C07D0F814040A
:1023000083B2DFF80407D0F81404020CDFF8301AA7
:1023100005A80AF00FF805A809F09CFE010005A821
:1023200009F04EFFDFF8E006D0F8400483B2DFF892
:10233000D806D0F84004020CDFF8081A05A809F006
:10234000F9FF05A809F086FE010005A809F038FF8D
:102350004FF4FA6009F080FFDFF8AC06D0F84404CF
:1023600083B2DFF8A406D0F84404020CDFF8D819D1
:1023700005A809F0DFFF05A809F06CFE010005A81B
:1023800009F01EFFDFF88006D0F8480483B2DFF8BA
:102390007806D0F84804020CDFF8B01905A809F057
:1023A000C9FF05A809F056FE010005A809F008FFBD
:1023B000DFF85406D0F84C0483B2DFF84C06D0F8AE
:1023C0004C04020CDFF8881905A809F0B3FF05A832
:1023D00009F040FE010005A809F0F2FEDFF828062A
:1023E000D0F8500483B2DFF82006D0F85004020C75
:1023F000DFF8601905A809F09DFF05A809F02AFE7D
:10240000010005A809F0DCFEDFF8FC05D0F8540453
:1024100083B2DFF8F405D0F85404020CDFF8381961
:1024200005A809F087FF05A809F014FE010005A81A
:1024300009F0C6FEDFF8D005D0F8580483B2DFF803
:10244000C805D0F85804020CDFF8101905A809F0E7
:1024500071FF05A809F0FEFD010005A809F0B0FE16
:10246000DFF8A405D0F85C0483B2DFF89C05D0F84F
:102470005C04020CDFF8E81805A809F05BFF05A86A
:1024800009F0E8FD010005A809F09AFEDFF87805DB
:10249000D0F8600483B2DFF87005D0F86004020C55
:1024A000DFF8C01805A809F045FF05A809F0D2FD1E
:1024B000010005A809F084FEDFF84C05D0F864049B
:1024C00083B2DFF84405D0F86404020CDFF89818F2
:1024D00005A809F02FFF05A809F0BCFD010005A81B
:1024E00009F06EFE4FF4FA6009F0B6FEDFF8180549
:1024F000D0F8680483B2DFF81005D0F86804020C45
:10250000DFF8681805A809F015FF05A809F0A2FD75
:10251000010005A809F054FEDFF8EC04D0F86C04C3
:1025200083B2DFF8E404D0F86C04020CDFF8401842
:1025300005A809F0FFFE05A809F08CFD010005A81B
:1025400009F03EFEDFF8C004D0F8700483B2DFF873
:10255000B804D0F87004020CDFF8181805A809F0C8
:10256000E9FE05A809F076FD010005A809F028FE9E
:10257000DFF89404D0F8740483B2DFF88C04D0F848
:102580007404020CDFF8F01705A809F0D3FE05A8C3
:1025900009F060FD010005A809F012FEDFF86804EB
:1025A000D0F8780483B2DFF86004D0F87804020C25
:1025B000DFF8C81705A809F0BDFE05A809F04AFD17
:1025C000010005A809F0FCFDDFF83C04D0F87C040C
:1025D00083B2DFF83404D0F87C04020CDFF8A017D3
:1025E00005A809F0A7FE05A809F034FD010005A81B
:1025F00009F0E6FDDFF81004D0F8800483B2DFF8BC
:102600000804D0F88004020CDFF8781705A809F058
:1026100091FE05A809F01EFD010005A809F0D0FDF6
:10262000DFF8E403D0F8840483B2DFF8DC03D0F8E9
:102630008404020CDFF8501705A809F07BFE05A8FA
:1026400009F008FD010005A809F0BAFDDFF8B8039C
:10265000D0F8880483B2DFF8B003D0F88804020C05
:10266000DFF8281705A809F065FE05A809F0F2FCB7
:10267000010005A809F0A4FD4FF4FA6009F0ECFD93
:10268000E148D0F88C0483B2DF48D0F88C04020C07
:10269000DFF8FC1605A809F04DFE05A809F0DAFCE4
:1026A000010005A809F08CFDD748D0F8900483B24A
:1026B000D548D0F89004020CDFF8D81605A809F028
:1026C00039FE05A809F0C6FC010005A809F078FD4F
:1026D000CD48D0F8940483B2CB48D0F89404020CCF
:1026E000DFF8B41605A809F025FE05A809F0B2FC2C
:1026F000010005A809F064FDC348D0F8980483B22E
:10270000C148D0F89804020CDFF8901605A809F02B
:1027100011FE05A809F09EFC010005A809F050FD76
:10272000B948D0F8AC0483B2B748D0F8AC04020C76
:10273000DFF86C1605A809F0FDFD05A809F08AFC74
:10274000010005A809F03CFDAF48D0F89C0483B215
:10275000AD48D0F89C04020CDFF8481605A809F033
:10276000E9FD05A809F076FC010005A809F028FD9F
:10277000A548D0F8A00483B2A348D0F8A004020C66
:10278000DFF8241605A809F0D5FD05A809F062FCBC
:10279000010005A809F014FD9B48D0F8A40483B2F9
:1027A0009948D0F8A404020CDFF8001605A809F037
:1027B000C1FD05A809F04EFC010005A809F000FDC7
:1027C0009148D0F8A80483B28F48D0F8A804020C2E
:1027D000DFF8DC1505A809F0ADFD05A809F03AFC05
:1027E000010005A809F0ECFC8748D0F8B00483B2DA
:1027F0008548D0F8B004020CDFF8B81505A809F038
:1028000099FD05A809F026FC010005A809F0D8FCEF
:102810007D4890F8CD24DFF8A01505A809F08AFDC1
:1028200005A809F017FC010005A809F0C9FC7648C5
:10283000B0F8B424DFF8841505A809F07BFD05A8DD
:1028400009F008FC010005A809F0BAFC012084F891
:10285000B40201F0DBBFDFF868152000FDF7EAFDE8
:10286000002802D10020002820D0DFF85805006899
:10287000438ADFF850050068028ADFF84C1505A886
:1028800009F058FD05A809F0E5FB020092B205A980
:102890002000FDF738FD012084F8B40201F0B6BF36
:1028A0007C2E020874B4002098FB0108DFF8F01EAB
:1028B0002000FDF7BFFD002803D10020002800F014
:1028C00090822000FDF7AEFD01212000FDF769FD9B
:1028D000002803D10020002800F08082AAA1200057
:1028E000FDF7A8FD002802D1002000285ED0464850
:1028F00090F88821DFF8AC1E05A809F01BFD05A89B
:1029000009F0A8FB010005A809F05AFCDFF8981EA1
:1029100005A809F00FFDDFF8941E05A809F00AFDCF
:1029200005A809F097FB010005A809F049FC00265D
:1029300034E0B6B2344810EBC600B0F8EC010390B6
:10294000B6B2314810EBC600B0F8EE010290B6B254
:102950002D4810EBC600B0F8EA010190B6B22A4843
:1029600010EBC60090F8E9010090B6B2264810EBD3
:10297000C60090F8E831B6B23200DFF8F01E05A8C4
:1029800009F0D8FC05A809F065FB010005A809F0CD
:1029900017FC4FF47A7009F05FFC761CB6B2182E63
:1029A000C7DB012084F8B40201F030BF7CA1200015
:1029B000FDF740FD002802D1002000286ED012480B
:1029C00090F88821DFF8DC1D05A809F0B3FC05A804
:1029D00009F040FB010005A809F0F2FBDFF8901EAA
:1029E00005A809F0A7FCDFF8C41D05A809F0A2FCA2
:1029F00005A809F02FFB010005A809F0E1FB00265E
:102A000040E000BFD43102081018001084F401081F
:102A1000B6B2DFF8600E10EBC600B0F8AC0203905F
:102A2000B6B2DFF8500E10EBC600B0F8AE0202905E
:102A3000B6B2DFF8400E10EBC600B0F8AA02019063
:102A4000B6B2DFF8300E10EBC60090F8A902009085
:102A5000B6B2DFF8200E10EBC60090F8A832B6B27E
:102A60003200DFF8081E05A809F064FC05A809F08B
:102A7000F1FA010005A809F0A3FB4FF47A7009F000
:102A8000EBFB761CB6B2182EC2DB012084F8B40230
:102A900001F0BCBE68B4002028F40108DFF8D81D9E
:102AA0002000FDF7C7FC002803D10020002800F01B
:102AB0009281DFF8C00D90F8C824DFF8C01D05A88A
:102AC00009F038FC05A809F0C5FA010005A809F0CD
:102AD00077FBDFF8AC1D05A809F02CFC05A809F070
:102AE000B9FA010005A809F06BFBDFF8981D05A8ED
:102AF00009F020FC05A809F0ADFA010005A809F0CD
:102B00005FFB012625E000BF58F30108300E0208E4
:102B10005429020880160208B6B23200DFF8681D98
:102B200005A809F007FC05A809F094FA010005A81A
:102B300009F046FBB6B20A2E0ADA6CA105A809F024
:102B4000F9FB05A809F086FA010005A809F038FB91
:102B5000761CB6B20A2EDFDB66A105A809F0EAFBF7
:102B600005A809F077FA010005A809F029FB01265C
:102B70008EE000BF981602084C0E0208B01602083C
:102B80005C21020870210208696E0000C816020864
:102B9000E016020864290208F81602081017020855
:102BA0006F757400680E020828170208BFB2B6B22B
:102BB0000A20DFF8C01C00FB0610381890F96823C3
:102BC0004FA105A809F0B6FB05A809F043FA0100DA
:102BD00005A809F0F5FABFB2B6B20A20DFF8941CD6
:102BE00000FB0610381890F9680300280AD43FA1AA
:102BF00005A809F09FFB05A809F02CFA010005A81B
:102C000009F0DEFABFB2B6B20A20DFF8681C00FB9A
:102C10000610381890F968030FF057F90A280ADAF5
:102C200032A105A809F086FB05A809F013FA0100F6
:102C300005A809F0C5FABFB2B6B20A20DFF8341C05
:102C400000FB0610381890F968030FF03EF964286D
:102C50000ADA26A105A809F06DFB05A809F0FAF922
:102C6000010005A809F0ACFA7F1CBFB20A2F9DDB5A
:102C700020A105A809F05EFB05A809F0EBF9010009
:102C800005A809F09DFA4FF47A7009F0E5FA761C70
:102C9000B6B2102E80F29A80B6B23200DFF8601E13
:102CA00005A809F047FB05A809F0D4F9010005A81B
:102CB00009F086FAB6B20A2E0ADA0CA105A809F0C4
:102CC00039FB05A809F0C6F9010005A809F078FA52
:102CD0000127CAE7840E020850060208A00E020867
:102CE000401702085817020884210208200000003B
:102CF000701702080D0A00008817020898210208C0
:102D00002564200094090208AC21020874290208F5
:102D1000C0210208A0170208D4210208E8210208F5
:102D2000B8170208BC0E0208D80E0208D017020815
:102D3000FC210208E8170208001802081818020807
:102D400030180208481802086018020878180208AB
:102D500090180208F40E0208100F02082C0F020847
:102D6000480F0208640F0208800F0208A818020822
:102D70009C0F0208B80F0208D40F0208C0180208FE
:102D8000D8180208F0180208F00F02080C10020808
:102D900008190208B40902082810020844100208A1
:102DA0007406020820190208601002083819020887
:102DB0007C100208501902086819020880190208DC
:102DC000882E02086CB400209C020208012084F8BE
:102DD000B40201F01BBD012501F018BD012501F071
:102DE00015BDDFF8581E2000FDF724FB002803D195
:102DF0000020002800F0DC84DFF8441E05A809F05C
:102E000099FA05A809F026F9010005A809F0D8F9F2
:102E1000DFF8600AB0F84220DFF8281E05A809F0A4
:102E200089FA05A809F016F9010005A809F0C8F902
:102E3000DFF8400AB0F94420DFF80C1E05A809F0BD
:102E400079FA05A809F006F9010005A809F0B8F912
:102E5000DFF8200AB0F94620DFF8F01D05A809F0D8
:102E600069FA05A809F0F6F8010005A809F0A8F923
:102E7000DFF8000AB0F94820DFF8D41D05A809F0F2
:102E800059FA05A809F0E6F8010005A809F098F933
:102E9000DFF8E009B0F94A20DFF8B81D05A809F00D
:102EA00049FA05A809F0D6F8010005A809F088F943
:102EB000DFF8C009B0F94C20DFF89C1D05A809F027
:102EC00039FA05A809F0C6F8010005A809F078F953
:102ED000DFF8A009B0F94E20DFF8801D05A809F041
:102EE00029FA05A809F0B6F8010005A809F068F963
:102EF000DFF88009B0F95020DFF8641D05A809F05B
:102F000019FA05A809F0A6F8010005A809F058F972
:102F1000DFF86009B0F95220DFF8481D05A809F074
:102F200009FA05A809F096F8010005A809F048F982
:102F3000DFF84009B0F95420DFF82C1D05A809F08E
:102F4000F9F905A809F086F8010005A809F038F993
:102F5000DFF82009B0F95620DFF8101D05A809F0A8
:102F6000E9F905A809F076F8010005A809F028F9A3
:102F70004FF4FA6009F070F9DFF8F808B0F858205B
:102F8000DFF8EC1C05A809F0D5F905A809F062F8EE
:102F9000010005A809F014F9DFF8D808B0F85A20A4
:102FA000DFF8D01C05A809F0C5F905A809F052F80A
:102FB000010005A809F004F9DFF8B808B0F85C20B2
:102FC000DFF8B41C05A809F0B5F905A809F042F826
:102FD000010005A809F0F4F8DFF89808006E0AF07F
:102FE00075F902000B00DFF8941C05A809F0A2F99E
:102FF00005A809F02FF8010005A809F0E1F8DFF8AD
:103000007408406E0AF062F902000B00DFF8701CD1
:1030100005A809F08FF905A809F01CF8010005A81A
:1030200009F0CEF8DFF84C08806E0AF04FF9020084
:103030000B00DFF8501C05A809F07CF905A809F081
:1030400009F8010005A809F0BBF8DFF82808C06EF0
:103050000AF03CF902000B00DFF82C1C05A809F06F
:1030600069F905A808F0F6FF010005A809F0A8F81D
:10307000DFF80008006F0AF029F902000B00DFF802
:103080000C1C05A809F056F905A808F0E3FF01009B
:1030900005A809F095F8DFF8DC07806F0AF016F94B
:1030A00002000B00DFF8E81B05A809F043F905A8AA
:1030B00008F0D0FF010005A809F082F8DFF8B40796
:1030C000D0F888000AF002F902000B00DFF8C41BF8
:1030D00005A809F02FF905A808F0BCFF010005A814
:1030E00009F06EF8DFF88C07D0F88C000AF0EEF8E3
:1030F00002000B00DFF8A01B05A809F01BF905A8CA
:1031000008F0A8FF010005A809F05AF8DFF86407E5
:10311000D0F89C000AF0DAF802000B00DFF87C1B04
:1031200005A809F007F905A808F094FF010005A813
:1031300009F046F84FF4FA6009F08EF8DFF834072A
:10314000D0F8A0000AF0C2F802000B00DFF8501B14
:1031500005A809F0EFF805A808F07CFF010005A814
:1031600009F02EF8DFF80C07D0F8A4000AF0AEF84A
:1031700002000B00DFF82C1B05A809F0DBF805A8FE
:1031800008F068FF010005A809F01AF8DFF8E40666
:10319000D0F8A8000AF09AF802000B00DFF8081B2C
:1031A00005A809F0C7F805A808F054FF010005A814
:1031B00009F006F8DFF8BC06D0F8AC000AF086F893
:1031C00002000B00DFF8E41A05A809F0B3F805A81F
:1031D00008F040FF010005A808F0F2FFDFF89406B0
:1031E000D0F8B0000AF072F802000B00DFF8C01A45
:1031F00005A809F09FF805A808F02CFF010005A814
:1032000008F0DEFFDFF86C06D0F8B4000AF05EF8D4
:1032100002000B00DFF89C1A05A809F08BF805A83E
:1032200008F018FF010005A808F0CAFFDFF84406FF
:10323000D0F8B8000AF04AF802000B00DFF8781A5C
:1032400005A809F077F805A808F004FF010005A813
:1032500008F0B6FFDFF81C06D0F8BC000AF036F81C
:1032600002000B00DFF8541A05A809F063F805A85E
:1032700008F0F0FE010005A808F0A2FFDFF8F40551
:10328000D0F8C0000AF022F802000B00DFF8301A74
:1032900005A809F04FF805A808F0DCFE010005A814
:1032A00008F08EFFDFF8CC05D0F8C4000AF00EF865
:1032B00002000B00DFF8481E05A809F03BF805A83E
:1032C00008F0C8FE010005A808F07AFFDFF8A405A1
:1032D000D0F8C80009F0FAFF02000B00DFF8241E46
:1032E00005A809F027F805A808F0B4FE010005A814
:1032F00008F066FF4FF4FA6008F0AEFFDFF87405DF
:1033000090F8E020DFF8001E05A809F013F805A8E2
:1033100008F0A0FE010005A808F052FFDFF85405F0
:10332000D0F8CC0009F0D2FF02000B00DFF8DC1D62
:1033300005A808F0FFFF05A808F08CFE010005A80D
:1033400008F03EFFDFF82C05D0F8D00009F0BEFFF2
:1033500002000B00DFF8B81D05A808F0EBFF05A878
:1033600008F078FE010005A808F02AFFDFF8040540
:10337000D0F8D40009F0AAFF02000B00DFF8941D7A
:1033800005A808F0D7FF05A808F064FE010005A80D
:1033900008F016FFDFF8DC04D0F8D80009F096FF3B
:1033A00002000B00DFF8701D05A808F0C3FF05A898
:1033B00008F050FE010005A808F002FFDFF8B40491
:1033C000D0F8DC0009F082FF02000B00DFF84C1D92
:1033D00005A808F0AFFF05A808F03CFE010005A80D
:1033E00008F0EEFEDFF88C0490F8E120DFF8301DE5
:1033F00005A808F09FFF05A808F02CFE010005A80D
:1034000008F0DEFEDFF86C04B0F9E220DFF8141DEE
:1034100005A808F08FFF05A808F01CFE010005A80C
:1034200008F0CEFEDFF84C04B0F9E420DFF8F81C19
:1034300005A808F07FFF05A808F00CFE010005A80C
:1034400008F0BEFEDFF82C04D0F8E80009F03EFFDB
:1034500002000B00DFF8D41C05A808F06BFF05A8DC
:1034600008F0F8FD010005A808F0AAFEDFF8040442
:10347000D0F8EC0009F02AFF02000B00DFF8B01CC6
:1034800005A808F057FF05A808F0E4FD010005A80D
:1034900008F096FEDFF8DC03D0F8F00009F016FF24
:1034A00002000B00DFF88C1C05A808F043FF05A8FC
:1034B00008F0D0FD010005A808F082FEDFF8B40393
:1034C000B0F9F420DFF8701C05A808F033FF05A858
:1034D00008F0C0FD010005A808F072FEE548B0F94B
:1034E000F620DFF8581C05A808F024FF05A808F00E
:1034F000B1FD010005A808F063FEDE48B0F9F82030
:10350000DFF83C1C05A808F015FF05A808F0A2FD8F
:10351000010005A808F054FE4FF4FA6008F09CFE84
:10352000D44890F84020DFF81C1C05A808F002FFE2
:1035300005A808F08FFD010005A808F041FECD4860
:10354000B0F82425DFF8001C05A808F0F3FE05A854
:1035500008F080FD010005A808F032FEC548B0F86B
:10356000FA20DFF8E81B05A808F0E4FE05A808F03B
:1035700071FD010005A808F023FEBE48D0F8FC004C
:1035800009F0A4FE02000B00DFF8C41B05A808F038
:10359000D1FE05A808F05EFD010005A808F010FEA8
:1035A000B448B0F90221DFF8AC1B05A808F0C2FE50
:1035B00005A808F04FFD010005A808F001FEAD4880
:1035C000B0F90021DFF8901B05A808F0B3FE05A8AC
:1035D00008F040FD010005A808F0F2FDA548B0F98B
:1035E0000621DFF8781B05A808F0A4FE05A808F05E
:1035F00031FD010005A808F0E3FD9E48B0F9042163
:10360000DFF85C1B05A808F095FE05A808F022FD70
:10361000010005A808F0D4FD9648B0F80821DFF8AD
:10362000441B05A808F086FE05A808F013FD01005C
:1036300005A808F0C5FD8F4890F88921DFF8281B00
:1036400005A808F077FE05A808F004FD010005A80C
:1036500008F0B6FD874890F88821524905A808F07F
:1036600069FE05A808F0F6FC010005A808F0A8FD11
:103670008048B0F8C421DFF8F41A05A808F05AFE13
:1036800005A808F0E7FC010005A808F099FD7948B5
:10369000D0F8C80109F01AFE02000B00DFF8D01ABA
:1036A00005A808F047FE05A808F0D4FC010005A80D
:1036B00008F086FD6F4890F8C824704905A808F006
:1036C00039FE05A808F0C6FC010005A808F078FD41
:1036D0004FF4FA6008F0C0FD6648B0F81425DFF832
:1036E000941A05A808F026FE05A808F0B3FC01000E
:1036F00005A808F065FD5F48D0F8180509F0E6FD5B
:1037000002000B00DFF8701A05A808F013FE05A8E8
:1037100008F0A0FC010005A808F052FD5548B0F8DB
:103720001C25DFF8581A05A808F004FE05A808F0C3
:1037300091FC010005A808F043FD4E48B0F81E2595
:10374000DFF83C1A05A808F0F5FD05A808F082FC92
:10375000010005A808F034FD4648B0F82025DFF840
:10376000241A05A808F0E6FD05A808F073FC01007E
:1037700005A808F025FD3F48B0F82225DFF8081A13
:1037800005A808F0D7FD05A808F064FC010005A80D
:1037900008F016FD012084F8B40201F037B800BF2C
:1037A0001C32020810220208981002081CFD0108B1
:1037B000D2A12000FCF73EFE002802D10020002804
:1037C00064D0DFF8C81905A808F0B4FD05A808F012
:1037D00041FC010005A808F0F3FCDFF8B41905A8C6
:1037E00008F0A8FD05A808F035FC010005A808F0C0
:1037F000E7FC002631E0B6B20C201E4900FB0610A3
:1038000090ED460ABDEEC00A10EE100A00B2049018
:10381000B6B20C20174900FB0610D0F8140109F0CD
:1038200055FDCDE90201B6B20C20124900FB06108D
:10383000D0F8100109F04AFDCDE90001B6B232001E
:10384000DFF8501905A808F075FD05A808F002FC7E
:10385000010005A808F0B4FC761CB6B20A2ECADB3B
:10386000012084F8B40200F0D1BF00BF981902080B
:10387000B410020810180010243202082422020892
:10388000D4090208942E02082C320208DFF8081925
:103890002000FCF7CFFD002803D10020002800F015
:1038A0003181DFF8F808D0F8980109F00FFD020027
:1038B0000B00DFF8EC1805A808F03CFD05A808F09F
:1038C000C9FB010005A808F07BFCDFF8D008D0F8A0
:1038D0009C0109F0FBFC02000B00DFF8C81805A8EA
:1038E00008F028FD05A808F0B5FB010005A808F0C0
:1038F00067FCDFF8A808D0F8A00109F0E7FC020097
:103900000B00DFF8A41805A808F014FD05A808F0BE
:10391000A1FB010005A808F053FCDFF88008D0F8EF
:10392000A40109F0D3FC02000B00DFF8801805A801
:1039300008F000FD05A808F08DFB010005A808F0BF
:103940003FFCDFF85808D0F8A80109F0BFFC0200DE
:103950000B00DFF8E41E05A808F0ECFC05A808F051
:1039600079FB010005A808F02BFCDFF83008D0F83F
:10397000AC0109F0ABFC02000B00DFF8C01E05A88B
:1039800008F0D8FC05A808F065FB010005A808F0C0
:1039900017FCDFF80808D0F8B00109F097FC020026
:1039A0000B00DFF89C1E05A808F0C4FC05A808F071
:1039B00051FB010005A808F003FCDFF8E007D0F890
:1039C000B40109F083FC02000B00DFF8781E05A8A3
:1039D00008F0B0FC05A808F03DFB010005A808F0C0
:1039E000EFFBDFF8B807B0F9CE24DFF85C1E05A8BE
:1039F00008F0A0FC05A808F02DFB010005A808F0C0
:103A0000DFFBDFF89807D0F8B80109F05FFC02008F
:103A10000B00DFF8381E05A808F08CFC05A808F09C
:103A200019FB010005A808F0CBFBDFF87007D0F800
:103A3000BC0109F04BFC02000B00DFF8141E05A8C6
:103A400008F078FC05A808F005FB010005A808F0BF
:103A5000B7FBDFF84807D0F8C00109F037FC0200D7
:103A60000B00DFF8F01D05A808F064FC05A808F0BD
:103A7000F1FA010005A808F0A3FBDFF82007D0F851
:103A80008C0109F023FC02000B00DFF8CC1D05A817
:103A900008F050FC05A808F0DDFA010005A808F0C0
:103AA0008FFBDFF8F806D0F8900109F00FFC020058
:103AB0000B00DFF8A81D05A808F03CFC05A808F0DD
:103AC000C9FA010005A808F07BFBDFF8D006D0F8A2
:103AD000940109F0FBFB02000B00DFF8841D05A830
:103AE00008F028FC05A808F0B5FA010005A808F0C0
:103AF00067FB012084F8B40200F088BE77700000F4
:103B0000A02E0208DFF85C1D2000FCF793FC0028C3
:103B100003D10020002800F0D580DFF88006D0F81F
:103B2000CC0109F0D3FB02000B00DFF83C1D05A817
:103B300008F000FC05A808F08DFA010005A808F0BF
:103B40003FFBDFF85806D0F8D00109F0BFFB0200B8
:103B50000B00DFF8181D05A808F0ECFB05A808F01D
:103B600079FA010005A808F02BFBDFF83006D0F841
:103B7000D40109F0ABFB02000B00DFF8F41C05A830
:103B800008F0D8FB05A808F065FA010005A808F0C0
:103B900017FBDFF80806D0F8D80109F097FB020000
:103BA0000B00DFF85C1D05A808F0C4FB05A808F0B1
:103BB00051FA010005A808F003FBDFF8E005D0F892
:103BC000DC0109F083FB02000B00DFF8381D05A8BB
:103BD00008F0B0FB05A808F03DFA010005A808F0C0
:103BE000EFFADFF8B805D0F8E00109F06FFB02004A
:103BF0000B00DFF8141D05A808F09CFB05A808F0D1
:103C000029FA010005A808F0DBFADFF89005D0F8E2
:103C1000E40109F05BFB02000B00DFF8F01C05A8D3
:103C200008F088FB05A808F015FA010005A808F0BF
:103C3000C7FA012084F8B40200F0E8BDF4310208AC
:103C4000F409020898060208D0100208B019020808
:103C5000C8190208E0190208EC100208F819020855
:103C6000BC060208E0060208140A0208081102084D
:103C700084290208382202084C220208101A02087D
:103C800004070208281A0208401A0208581A0208F3
:103C9000340A0208540A020828070208740A0208B3
:103CA000701A0208881A0208A01A0208B81A020834
:103CB00024110208D01A020840110208940A0208CE
:103CC000B40A0208E2A12000FCF7B4FB002803D1EB
:103CD0000020002800F06C82DFF8C004D0F8B8049F
:103CE00009F0F4FA02000B00DFF8881B05A808F0C1
:103CF00021FB05A808F0AEF9010005A808F060FA5C
:103D0000DFF89804D0F8BC0409F0E0FA02000B00D8
:103D1000DFF8FC1B05A808F00DFB05A808F09AF9D0
:103D2000010005A808F04CFADFF87004D0F8C004D0
:103D300009F0CCFA02000B00DFF8D81B05A808F048
:103D4000F9FA05A808F086F9010005A808F038FA84
:103D5000DFF84804D0F8C40409F0B8FA02000B00F8
:103D6000DFF8B41B05A808F0E5FA05A808F072F919
:103D7000010005A808F024FADFF82004B0F8D024E8
:103D8000DFF8981B05A808F0D5FA05A808F062F935
:103D9000010005A808F014FADFF80004B0F8D224F6
:103DA000DFF87C1B05A808F0C5FA05A808F052F951
:103DB000010005A808F004FADFF8E003B0F8D42405
:103DC000DFF8601B05A808F0B5FA05A808F042F96D
:103DD000010005A808F0F4F9DFF8C003D0F8D80412
:103DE00009F074FA02000B00DFF83C1B05A808F08C
:103DF000A1FA05A808F02EF9010005A808F0E0F9DD
:103E0000E648D0F8DC0409F061FA02000B00DFF8A4
:103E10001C1B05A808F08EFA05A808F01BF9010084
:103E200005A808F0CDF9DD48D0F8E00409F04EFA15
:103E300002000B00DFF8F81A05A808F07BFA05A8C5
:103E400008F008F9010005A808F0BAF9D348D0F83D
:103E5000EC0409F03BFA02000B00DFF8D81A05A8C1
:103E600008F068FA05A808F0F5F8010005A808F0C0
:103E7000A7F9CA48D0F8F40409F028FA02000B00A8
:103E8000DFF8B41A05A808F055FA05A808F0E2F81A
:103E9000010005A808F094F9C048D0F8F80409F02A
:103EA00015FA02000B00DFF8941A05A808F042FA90
:103EB00005A808F0CFF8010005A808F081F9B74877
:103EC000D0F8FC0409F002FA02000B00DFF8701AC7
:103ED00005A808F02FFA05A808F0BCF8010005A80D
:103EE00008F06EF9AD48D0F8000509F0EFF90200CE
:103EF0000B00DFF8501A05A808F01CFA05A808F016
:103F0000A9F8010005A808F05BF9A448D0F8040559
:103F100009F0DCF902000B00DFF82C1A05A808F004
:103F200009FA05A808F096F8010005A808F048F974
:103F30009A48D0F8080509F0C9F902000B00DFF82B
:103F40000C1A05A808F0F6F905A808F083F8010096
:103F500005A808F035F99148D0F80C0509F0B6F934
:103F600002000B00DFF8E81905A808F0E3F905A83E
:103F700008F070F8010005A808F022F98748D0F889
:103F8000100509F0A3F902000B00DFF8C81905A815
:103F900008F0D0F905A808F05DF8010005A808F0C0
:103FA0000FF97E48D0F8F00409F090F902000B00F8
:103FB000DFF8A41905A808F0BDF905A808F04AF82B
:103FC000010005A808F0FCF84FF4FA6008F044F985
:103FD0007248C06909F07AF902000B00DFF87C1919
:103FE00005A808F0A7F905A808F034F8010005A80D
:103FF00008F0E6F86948006A09F068F902000B0069
:10400000DFF85C1905A808F095F905A808F022F872
:10401000010005A808F0D4F86048406A09F056F994
:1040200002000B00DFF83C1905A808F083F905A889
:1040300008F010F8010005A808F0C2F85748806A97
:1040400009F044F902000B00DFF81C1902E000BF80
:10405000696D750005A808F06DF905A807F0FAFF6D
:10406000010005A808F0ACF84C48C06A09F02EF928
:1040700002000B00DFF8F41805A808F05BF905A8AA
:1040800007F0E8FF010005A808F09AF84348006B24
:1040900009F01CF902000B00DFF8D41805A808F09D
:1040A00049F905A807F0D6FF010005A808F088F82F
:1040B0003A48406B09F00AF902000B00DFF8B41827
:1040C00005A808F037F905A807F0C4FF010005A806
:1040D00008F076F83148806B09F0F8F802000B0020
:1040E000DFF8941805A808F025F905A807F0B2FF35
:1040F000010005A808F064F8012084F8B40285E303
:10410000D40A0208F40A02085C110208F803020843
:10411000C8020208140B0208340B0208540B0208F0
:1041200060220208942902087422020888220208E8
:10413000A4290208B42902089C220208B02202081D
:10414000C4290208781102084C07020894110208D9
:1041500070070208E81A0208B0110208CC11020820
:10416000740B020820040208E811020894070208F0
:1041700004120208940B0208B80702082012020871
:10418000001B0208B40B0208D40B0208181B02081B
:1041900048040208301B0208D42902081018001035
:1041A000481B0208601B0208781B0208901B0208CB
:1041B000DFF8C8172000FCF73DF9002803D10020E4
:1041C000002800F09C82DFF8B807006890F895306E
:1041D000DFF8AC07006890F89420DFF8A81705A86E
:1041E00008F0A8F805A807F035FF010005A807F0BA
:1041F000E7FFDFF88C07006890F898000090DFF880
:104200008007006890F89730DFF87407006890F82E
:104210009620DFF8741705A808F08CF805A807F0B9
:1042200019FF010005A807F0CBFFDFF8540700686D
:10423000006D09F04BF802000B00DFF8501705A8DD
:1042400008F078F805A807F005FF010005A807F0B9
:10425000B7FFDFF82C070068406D09F037F802005F
:104260000B00DFF82C1705A808F064F805A807F084
:10427000F1FE010005A807F0A3FFDFF804070068BE
:10428000B0F93A20DFF80C1705A808F053F805A894
:1042900007F0E0FE010005A807F092FFDFF8E00656
:1042A0000068B0F93C20DFF8F01605A808F042F8E5
:1042B00005A807F0CFFE010005A807F081FFDFF891
:1042C000C0060068B0F93E20DFF8D01605A808F057
:1042D00031F805A807F0BEFE010005A807F070FF41
:1042E000DFF89C060068B0F84020DFF8B41605A897
:1042F00008F020F805A807F0ADFE010005A807F0BA
:104300005FFFDFF87C060068B0F84220DFF8941603
:1043100005A808F00FF805A807F09CFE010005A805
:1043200007F04EFFDFF858060068B0F84420DFF8C9
:10433000781605A807F0FEFF05A807F08BFE010020
:1043400005A807F03DFFDFF838060068B0F9462001
:10435000DFF8581605A807F0EDFF05A807F07AFE6C
:10436000010005A807F02CFFDFF814060068B0F97B
:104370004820DFF83C1605A807F0DCFF05A807F089
:1043800069FE010005A807F01BFFDFF8F4050068CF
:10439000B0F94A20DFF81C1605A807F0CBFF05A8E6
:1043A00007F058FE010005A807F00AFFDFF8D00566
:1043B0000068B0F94C20DFF8001605A807F0BAFF36
:1043C00005A807F047FE010005A807F0F9FEDFF891
:1043D000B0050068B0F94E20DFF8E01505A807F039
:1043E000A9FF05A807F036FE010005A807F0E8FEC2
:1043F000DFF88C050068D0F8A80008F067FF02001D
:104400000B00DFF8BC1505A807F094FF05A807F01E
:1044100021FE010005A807F0D3FEDFF8640500685F
:10442000D0F8AC0008F052FF02000B00DFF8941542
:1044300005A807F07FFF05A807F00CFE010005A8FE
:1044400007F0BEFEDFF838050068D0F8B00008F0CD
:104450003DFF02000B00DFF8701505A807F06AFFAA
:1044600005A807F0F7FD010005A807F0A9FEDFF891
:1044700010050068D0F8B40008F028FF02000B0017
:10448000DFF8481505A807F055FF05A807F0E2FD7D
:10449000010005A807F094FEDFF8E4040068D0F8F6
:1044A000B80008F013FF02000B00DFF8241505A880
:1044B00007F040FF05A807F0CDFD010005A807F0B3
:1044C0007FFEDFF8BC040068D0F8BC0008F0FEFEF8
:1044D00002000B00DFF8FC1405A807F02BFF05A86D
:1044E00007F0B8FD010005A807F06AFEDFF89004A8
:1044F0000068D0F8C00008F0E9FE02000B00DFF809
:10450000D81405A807F016FF05A807F0A3FD0100C1
:1045100005A807F055FEDFF868040068D0F8C4006D
:1045200008F0D4FE02000B00DFF8B01405A807F075
:1045300001FF05A807F08EFD010005A807F040FE69
:10454000DFF83C040068D0F8C80008F0BFFE0200A5
:104550000B00DFF88C1405A807F0ECFE05A807F0A7
:1045600079FD010005A807F02BFEDFF814040068B0
:10457000D0F8CC0008F0AAFE02000B00DFF86414AB
:1045800005A807F0D7FE05A807F064FD010005A8FF
:1045900007F016FEDFF8E8030068D0F8D00008F056
:1045A00095FE02000B00DFF8401405A807F0C2FEDC
:1045B00005A807F04FFD010005A807F001FEDFF890
:1045C000C0030068D0F8D40008F080FE02000B00A1
:1045D000DFF8181405A807F0ADFE05A807F03AFDAE
:1045E000010005A807F0ECFDDFF894030068D0F89F
:1045F000D80008F06BFE02000B00DFF8F41305A8EA
:1046000007F098FE05A807F025FD010005A807F0B2
:10461000D7FDDB480068D0F8DC0008F057FE020048
:104620000B00DFF8D01305A807F084FE05A807F0FB
:1046300011FD010005A807F0C3FDD1480068D0F8BE
:10464000E00008F043FE02000B00DFF8AC1305A801
:1046500007F070FE05A807F0FDFC010005A807F0B3
:10466000AFFDC7480068D0F8E40008F02FFE020054
:104670000B00DFF8881305A807F05CFE05A807F01B
:10468000E9FC010005A807F09BFDBD480068806DAE
:1046900008F01CFE02000B00D94905A807F04AFEED
:1046A00005A807F0D7FC010005A807F089FDB4486C
:1046B0000068006E08F00AFE02000B00D14905A850
:1046C00007F038FE05A807F0C5FC010005A807F0B3
:1046D00077FDAB480068C06D08F0F8FD02000B00E4
:1046E000C94905A807F026FE05A807F0B3FC01009C
:1046F00005A807F065FD012084F8B40286E07FA1DB
:104700002000FBF797FE002802D10020002844D0AB
:10471000BE4800680079002816D1BD4905A807F0F9
:1047200009FE05A807F096FC010005A807F048FD62
:10473000B84905A807F0FEFD05A807F08BFC0100AD
:1047400005A807F03DFD19E0B34905A807F0F2FD03
:1047500005A807F07FFC010005A807F031FDAB4874
:104760000068B0F82422AD4905A807F0E3FD05A8CC
:1047700007F070FC010005A807F022FDA3480068BF
:104780008268A74905A807F0D5FD05A807F062FCD7
:10479000010005A807F014FD38E0A2492000FBF74E
:1047A00049FE002802D1002000282CD09E48006835
:1047B00002789E4905A807F0BDFD05A807F04AFC50
:1047C000010005A807F0FCFC97480068D0F82C24ED
:1047D000974905A807F0AEFD05A807F03BFC0100CE
:1047E00005A807F0EDFC9048006890F83024914946
:1047F00005A807F09FFD05A807F02CFC010005A8FF
:1048000007F0DEFC02E0012500E00125EDB2002DFD
:104810000BD0894807F01EFC020092B286492000A6
:10482000FBF771FD012084F8B4020120FDF75DB9AA
:104830000020FDF75AB900BFA81B0208C4220208D5
:10484000C01B0208D81B02083C120208D82202082A
:10485000F01B0208081C0208201C0208381C020871
:10486000501C0208AC2E02085812020874120208EA
:1048700090120208C812020838B504000025B4F8E6
:104880000401042801D0002032BD04226B49B4F891
:104890000201001907F010FC00282CD10121200092
:1048A000FBF77FFD002802D10020002811D0200056
:1048B000FBF7DBFDC0B2082809DA0100C9B2604885
:1048C00000680DF087FB012084F8B40202E00125A6
:1048D00000E00125EDB2002D0BD0574807F0BAFBE0
:1048E000020092B254492000FBF70DFD012084F82C
:1048F000B4020120C8E70020C6E70000677073001B
:10490000F40B0208140C0208AC120208340C020862
:10491000E4120208681C0208DC070208801C020876
:10492000981C0208B01C0208001302081C1302089D
:10493000C81C020838130208540C0208740C020840
:10494000940C020800080208B40C0208D40C0208F7
:10495000F40C02082408020854130208EC2202088E
:104960000023020814230208282302083C2302081B
:104970005023020864230208E01C0208DC3102080C
:1049800040B4002078230208F81C0208B82E020860
:10499000C42E0208D02E0208DC2E0208E82E0208DF
:1049A000F42E0208002F02080C2F020834320208ED
:1049B0003C320208443202084C32020854320208E7
:1049C000182F0208242F0208302F02083C2F02085B
:1049D000482F0208542F0208602F02086C2F02088B
:1049E000782F0208842F0208902F02089C2F0208BB
:1049F000A82F0208B42F0208C02F0208CC2F0208EB
:104A00008C230208E4290208F42902084CB400208F
:104A1000042A0208A0230208142A0208242A0208F1
:104A2000701302085C32020854B40020B423020858
:104A3000101D0208342A0208D8080208643202084D
:104A400078B400202DE9F0472DED028B9EB00400D4
:104A50000025B4F80401032805D000201EB0BDECE9
:104A6000028BBDE8F0870322D4A1B4F8020100193B
:104A700007F022FB002847F0B78001212000FBF758
:104A800090FC002803D10020002807F09880DFF870
:104A9000D01D2000FBF7CEFC002802D1002000280A
:104AA00032D02000FBF7BEFC01212000FBF779FC8F
:104AB000002802D10020002823D02000FBF7D5FCDD
:104AC0000700DFF80C0E8773DFF8040E817B89B2D4
:104AD00008200DF0CFFADFF8F80D827BDFF8F41D27
:104AE00005A807F027FC05A807F0B4FA020092B267
:104AF00005A92000FBF707FC012084F8B40207F0A9
:104B00005FB8012507F05CB8DFF8CC1D2000FBF78B
:104B100091FC002802D1002000282BD02000FBF7B8
:104B200081FC01212000FBF73CFC002802D1002081
:104B300000281CD02000FBF798FC0700DFF8900D40
:104B40008772DFF88C0D827ADFF8001E05A807F067
:104B5000F1FB05A807F07EFA020092B205A9200039
:104B6000FBF7D1FB012084F8B40207F029B8012536
:104B700007F026B8DFF8D81D2000FBF75BFC002803
:104B800002D1002000282FD02000FBF74BFC012190
:104B90002000FBF706FC002802D10020002820D0CE
:104BA0002000FBF762FC0700390089B2DFF8140E21
:104BB000006807F035FDDFF8180D8289DFF8081E60
:104BC00005A807F0B7FB05A807F044FA020092B267
:104BD00005A92000FBF797FB012084F8B40206F03A
:104BE000EFBF012506F0ECBFDFF8E01D2000FBF76A
:104BF00021FC002802D1002000282BD02000FBF748
:104C000011FC01212000FBF7CCFB002802D1002081
:104C100000281CD02000FBF728FC0700DFF8B00CB0
:104C20000781DFF8AC0C0289DFF8141E05A807F035
:104C300081FB05A807F00EFA020092B205A9200038
:104C4000FBF761FB012084F8B40206F0B9BF01252F
:104C500006F0B6BFDFF8EC1D2000FBF7EBFB0028E9
:104C600002D1002000283BD02000FBF7DBFB012114
:104C70002000FBF796FB002802D1002000282CD052
:104C80002000FBF7F2FB0700DFF8440C80F8C97442
:104C9000DFF83C0C90F8C924DFF81C1E05A807F0CB
:104CA00049FB05A807F0D6F9020092B205A9200039
:104CB000FBF729FBDFF8180C90F8C914DFF8FC0D9E
:104CC00000680DF032FADFF8F40D00680DF055FAC7
:104CD000012084F8B40206F073BF012506F070BF0E
:104CE000DFF8DC1D2000FBF7A5FB002802D1002027
:104CF00000282DD02000FBF795FB01212000FBF7B9
:104D000050FB002802D1002000281ED02000FBF715
:104D1000ACFB0700DFF8B80B80F8CB74DFF8B00B02
:104D200090F8CB24DFF80C1E05A807F003FB05A8BC
:104D300007F090F9020092B205A92000FBF7E3FA10
:104D4000012084F8B40206F03BBF012506F038BF0D
:104D5000DFF8E41D2000FBF76DFB002802D10020E6
:104D6000002830D02000FBF75DFB01212000FBF77D
:104D700018FB002802D10020002821D02000FBF7DA
:104D800074FB0700DFF8480B80F8CD74DFF8400BA8
:104D900090F8CD24DFF81C1E05A807F0CBFA05A873
:104DA00007F058F9020092B205A92000FBF7ABFA10
:104DB000012084F8B40206F003BF00BF73657400DD
:104DC000012506F0FDBEDFF8F01D2000FBF732FBE9
:104DD000002802D1002000282DD02000FBF722FB64
:104DE00001212000FBF7DDFA002802D10020002875
:104DF0001ED02000FBF739FB0700DFF8D40AA0F82B
:104E0000B474DFF8CC0AB0F8B424DFF8301E05A87B
:104E100007F090FA05A807F01DF9020092B205A963
:104E20002000FBF770FA012084F8B40206F0C8BE37
:104E3000012506F0C5BEDFF8081E2000FBF7FAFAD0
:104E4000002802D10020002830D02000FBF7EAFA29
:104E500001212000FBF7A5FA002802D1002000283C
:104E600021D02000FBF724FBDFF8640A80ED280A3C
:104E7000DFF85C0AD0F8A00008F028FA02000B0066
:104E8000DFF8C01D05A807F055FA05A807F0E2F8FD
:104E9000020092B205A92000FBF735FA012084F840
:104EA000B40206F08DBE012506F08ABEDFF8181E9A
:104EB0002000FBF7BFFA002802D10020002830D0E4
:104EC0002000FBF7AFFA01212000FBF76AFA002867
:104ED00002D10020002821D02000FBF7E9FADFF8FA
:104EE000F00980ED2B0ADFF8E809D0F8AC0008F0F3
:104EF000EDF902000B00DFF8D41D05A807F01AFA3F
:104F000005A807F0A7F8020092B205A92000FBF758
:104F1000FAF9012084F8B40206F052BE012506F029
:104F20004FBEDFF8281E2000FBF784FA002802D1CC
:104F30000020002830D02000FBF774FA0121200067
:104F4000FBF72FFA002802D10020002821D02000F2
:104F5000FBF7AEFADFF8780980ED290ADFF870096F
:104F6000D0F8A40008F0B2F902000B00DFF8E01D51
:104F700005A807F0DFF905A807F06CF8020092B267
:104F800005A92000FBF7BFF9012084F8B40206F060
:104F900017BE012506F014BEDFF82C1E2000FBF71B
:104FA00049FA002802D10020002830D02000FBF769
:104FB00039FA01212000FBF7F4F9002802D1002082
:104FC000002821D02000FBF773FADFF8040980EDF8
:104FD0002C0ADFF8FC08D0F8B00008F077F90200DE
:104FE0000B00DFF8E81D05A807F0A4F905A807F0F5
:104FF00031F8020092B205A92000FBF784F90120E4
:1050000084F8B40206F0DCBD012506F0D9BDDFF856
:10501000381E2000FBF70EFA002802D100200028DD
:1050200030D02000FBF7FEF901212000FBF7B9F991
:10503000002802D10020002821D02000FBF738FAF8
:10504000DFF88C0880ED2A0ADFF88408D0F8A80081
:1050500008F03CF902000B00DFF8F01D05A807F08E
:1050600069F905A806F0F6FF020092B205A9200032
:10507000FBF749F9012084F8B40206F0A1BD01252F
:1050800006F09EBDDFF8C81D2000FBF7D3F900280D
:1050900002D10020002830D02000FBF7C3F9012105
:1050A0002000FBF77EF9002802D10020002821D043
:1050B0002000FBF7FDF9DFF8180880ED2D0ADFF876
:1050C0001008D0F8B40008F001F902000B00DFF876
:1050D000FC1D05A807F02EF905A806F0BBFF02008D
:1050E00092B205A92000FBF70EF9012084F8B40262
:1050F00006F066BD012506F063BDDFF8D41D200073
:10510000FBF798F9002802D1002000282CD02000BD
:10511000FBF788F901212000FBF743F9002802D1B1
:10512000002000281DD02000FBF79FF90700DFF8C2
:10513000A007C782DFF89807B0F91620DFF80C1E29
:1051400005A807F0F7F805A806F084FF020092B260
:1051500005A92000FBF7D7F8012084F8B40206F077
:105160002FBD012506F02CBDDFF8E41D2000FBF764
:1051700061F9002802D1002000282CD02000FBF784
:1051800051F901212000FBF70CF9002802D1002081
:1051900000281DD02000FBF768F90700DFF8300772
:1051A0000783DFF82C07B0F91820DFF8201E05A8C8
:1051B00007F0C0F805A806F04DFF020092B205A95D
:1051C0002000FBF7A0F8012084F8B40206F0F8BC38
:1051D000012506F0F5BCDFF8F81D2000FBF72AF9E1
:1051E000002802D1002000282CD02000FBF71AF95B
:1051F00001212000FBF7D5F8002802D1002000286B
:105200001DD02000FBF731F90700DFF8C406478303
:10521000DFF8BC06B0F91A20DFF8301E05A807F049
:1052200089F805A806F016FF020092B205A9200031
:10523000FBF769F8012084F8B40206F0C1BC01252F
:1052400006F0BEBCDFF8081E2000FBF7F3F80028CC
:1052500002D1002000282CD02000FBF7E3F8012128
:105260002000FBF79EF8002802D1002000281DD066
:105270002000FBF7FAF80700DFF854060782DFF892
:105280005006B0F91020DFF8441E05A807F052F8C8
:1052900005A806F0DFFE020092B205A92000FBF788
:1052A00032F8012084F8B40206F08ABC012506F029
:1052B00087BCDFF81C1E2000FBF7BCF8002802D1D9
:1052C000002000282CD02000FBF7ACF801212000A2
:1052D000FBF767F8002802D1002000281DD020002D
:1052E000FBF7C3F80700DFF8E8054782DFF8E005C1
:1052F000B0F91220DFF8DC1D05A807F01BF805A89F
:1053000006F0A8FE020092B205A92000FAF7FBFF02
:10531000012084F8B40206F053BC012506F050BC0D
:10532000DFF82C1E2000FBF785F8002802D10020B2
:1053300000282CD02000FBF775F801212000FBF796
:1053400030F8002802D1002000281DD02000FBF7F3
:105350008CF80700DFF878058782DFF87405B0F96C
:105360001420DFF8F01D05A806F0E4FF05A806F0FC
:1053700071FE020092B205A92000FAF7C4FF0120D5
:1053800084F8B40206F01CBC012506F019BCDFF855
:10539000401E2000FBF74EF8002802D10020002814
:1053A0002DD02000FBF73EF801212000FAF7F9FF8D
:1053B000002802D1002000281ED02000FBF755F85D
:1053C0000700DFF80C0580F8E070DFF8040590F8BE
:1053D000E020DFF8001E05A806F0ACFF05A806F0E7
:1053E00039FE020092B205A92000FAF78CFF0120D5
:1053F00084F8B40206F0E4BB012506F0E1BBDFF857
:10540000501E2000FBF716F8002802D100200028CB
:1054100030D02000FBF706F801212000FAF7C1FF89
:10542000002802D10020002821D02000FBF740F8FE
:10543000DFF89C0480ED2E0ADFF89404D0F8B80061
:1054400007F044FF02000B00DFF8081E05A806F075
:1054500071FF05A806F0FEFD020092B205A920002A
:10546000FAF751FF012084F8B40206F0A9BB012528
:1054700006F0A6BBDFF8501E2000FAF7DBFF00287D
:1054800002D10020002830D02000FAF7CBFF012104
:105490002000FAF786FF002802D10020002821D042
:1054A0002000FBF705F8DFF8280480ED2F0ADFF86D
:1054B0002004D0F8BC0007F009FF02000B00DFF861
:1054C0000C1E05A806F036FF05A806F0C3FD020075
:1054D00092B205A92000FAF716FF012084F8B40261
:1054E00006F06EBB012506F06BBBDFF8541E2000F2
:1054F000FAF7A0FF002802D1002000282FD02000BA
:10550000FAF790FF01212000FAF74BFF002802D1A3
:105510000020002820D02000FAF7CAFFDFF8B003EF
:1055200080ED190ADFF8A803406E07F0CFFE0200F5
:105530000B00DFF8101E05A806F0FCFE05A806F01B
:1055400089FD020092B205A92000FAF7DCFE0120D5
:1055500084F8B40206F034BB012506F031BBDFF855
:10556000E81D2000FAF766FF002802D1002000287D
:105570002ED02000FAF756FF01212000FAF711FF84
:10558000002802D1002000281FD02000FAF790FF49
:10559000CF4880ED300ACE48D0F8C00007F096FE24
:1055A00002000B00DFF8141E05A806F0C3FE05A8D4
:1055B00006F050FD020092B205A92000FAF7A3FE02
:1055C000012084F8B40206F0FBBA012506F0F8BA0F
:1055D000DFF8EC1D2000FAF72DFF002802D1002093
:1055E00000282ED02000FAF71DFF01212000FAF735
:1055F000D8FE002802D1002000281FD02000FAF792
:1056000057FFB34880ED310AB148D0F8C40007F025
:105610005DFE02000B00DFF8181E05A806F08AFEEA
:1056200005A806F017FD020092B205A92000FAF7BE
:105630006AFE012084F8B40206F0C2BA012506F021
:10564000BFBADFF8F01D2000FAF7F4FE002802D1FF
:10565000002000282ED02000FAF7E4FE01212000CF
:10566000FAF79FFE002802D1002000281FD020005A
:10567000FAF71EFF964880ED320A9548D0F8C80028
:1056800007F024FE02000B00DFF8181E05A806F044
:1056900051FE05A806F0DEFC020092B205A920002A
:1056A000FAF731FE012084F8B40206F089BA012528
:1056B00006F086BADFF8F01D2000FAF7BBFE0028DE
:1056C00002D1002000282BD02000FAF7ABFE0121E8
:1056D0002000FAF766FE002802D1002000281CD026
:1056E0002000FAF7C2FE07007948A0F84670784813
:1056F000B0F94620DFF8201E05A806F01BFE05A81D
:1057000006F0A8FC020092B205A92000FAF7FBFD02
:10571000012084F8B40206F053BA012506F050BA0D
:10572000DFF8F81D2000FAF785FE002802D10020DE
:1057300000282BD02000FAF775FE01212000FAF78F
:1057400030FE002802D1002000281CD02000FAF7EB
:105750008CFE07005E48A0F844705D48B0F9442014
:10576000DFF8281E05A806F0E5FD05A806F072FC86
:10577000020092B205A92000FAF7C5FD012084F8C5
:10578000B40206F01DBA012506F01ABADFF8001EB1
:105790002000FAF74FFE002802D1002000282BD06D
:1057A0002000FAF73FFE01212000FAF7FAFD002859
:1057B00002D1002000281CD02000FAF756FE070076
:1057C0004348A0F848704248B0F94820DFF8301E3E
:1057D00005A806F0AFFD05A806F03CFC020092B259
:1057E00005A92000FAF78FFD012084F8B40206F025
:1057F000E7B9012506F0E4B9DFF8081E2000FAF742
:1058000019FE002802D1002000282ED02000FAF72F
:1058100009FE01212000FAF7C4FD002802D1002072
:1058200000281FD02000FAF720FE07002848A0F823
:1058300050702748B0F95020DFF8381E05A806F050
:1058400079FD05A806F006FC020092B205A9200029
:10585000FAF759FD012084F8B40206F0B1B900BF8F
:10586000C8230208012506F0ABB9DFF80C1E2000A2
:10587000FAF7E0FD002802D10020002831D02000F6
:10588000FAF7D0FD01212000FAF78BFD002802D1A4
:105890000020002822D02000FAF7E7FD07000C487E
:1058A000A0F852700A48B0F95220DFF8401E05A84F
:1058B00006F040FD05A806F0CDFB020092B205A956
:1058C0002000FAF720FD012084F8B40206F078B930
:1058D00010180010281D0208401D0208012506F0BE
:1058E0006FB9DFF80C1E2000FAF7A4FD002802D1E2
:1058F0000020002831D02000FAF794FD012120007B
:10590000FAF74FFD002802D10020002822D0200005
:10591000FAF7ABFD0700DFF8500EA0F85470DFF87F
:10592000480EB0F95420DFF8441E05A806F002FD29
:1059300005A806F08FFB020092B205A92000FAF735
:10594000E2FC012084F8B40206F03AB98C13020894
:10595000442A0208012506F033B9DFF8141E20009E
:10596000FAF768FD002802D10020002833D020007B
:10597000FAF758FD01212000FAF713FD002802D1A3
:105980000020002824D02000FAF76FFD0700DFF880
:10599000D80DA0F85670DFF8D00DB0F95620DFF81A
:1059A0004C1E05A806F0C6FC05A806F053FB020035
:1059B00092B205A92000FAF7A6FC012084F8B402EF
:1059C00006F0FEB880B40020581D0208DC2302084F
:1059D000012506F0F5B8DFF8181E2000FAF72AFDB9
:1059E000002802D10020002831D02000FAF71AFD4B
:1059F00001212000FAF7D5FC002802D10020002860
:105A000022D02000FAF731FD0700DFF85C0DA0F886
:105A10004A70DFF8540DB0F94A20DFF8501E05A88F
:105A200006F088FC05A806F015FB020092B205A955
:105A30002000FAF768FC012084F8B40206F0C0B830
:105A4000701D0208F0230208012506F0B9B8DFF83E
:105A5000201E2000FAF7EEFC002802D100200028CA
:105A600033D02000FAF7DEFC01212000FAF799FC80
:105A7000002802D10020002824D02000FAF7F5FCED
:105A80000700DFF8E40CA0F84C70DFF8DC0CB0F98C
:105A90004C20DFF8581E05A806F04CFC05A806F0BF
:105AA000D9FA020092B205A92000FAF72CFC0120D5
:105AB00084F8B40206F084B8300E02086CB40020FA
:105AC000D82F0208012506F07BB8DFF8241E20003D
:105AD000FAF7B0FC002802D10020002831D02000C5
:105AE000FAF7A0FC01212000FAF75BFC002802D1A4
:105AF0000020002822D02000FAF7B7FC0700DFF8CA
:105B0000680CA0F84E70DFF8600CB0F94E20DFF89A
:105B1000541E05A806F00EFC05A806F09BFA02002C
:105B200092B205A92000FAF7EEFB012084F8B40236
:105B300006F046B85429020804240208012506F09C
:105B40003FB8DFF8241E2000FAF774FC002802D1C9
:105B50000020002838D02000FAF764FC0121200042
:105B6000FAF71FFC002802D10020002829D02000CD
:105B7000FAF77BFC0700381EB0F5806F1ED2DFF805
:105B8000E80BA0F85870DFF8E00BB0F85820DFF809
:105B90004C1E05A806F0CEFB05A806F05BFA020035
:105BA00092B205A92000FAF7AEFB012084F8B402F6
:105BB00006F006B86819020818240208012505F045
:105BC000FFBF012505F0FCBFDFF8141E2000FAF727
:105BD00031FC002802D1002000283BD02000FAF739
:105BE00021FC01212000FAF7DCFB002802D1002073
:105BF00000282CD02000FAF738FC0700381EB0F53A
:105C0000806F21D2DFF8600BA0F85A70DFF8580BD4
:105C1000B0F85A20DFF83C1E05A806F08BFB05A85B
:105C200006F018FA020092B205A92000FAF76BFB01
:105C3000012084F8B40205F0C3BF00BF8019020838
:105C4000542A0208701A0208012505F0B9BF01257F
:105C500005F0B6BFDFF8001E2000FAF7EBFB0028C6
:105C600002D10020002839D02000FAF7DBFB012107
:105C70002000FAF796FB002802D1002000282AD045
:105C80002000FAF7F2FB0700381EB0F5806F1FD234
:105C9000DFF8D40AA0F85C70DFF8CC0AB0F85C201A
:105CA000DFF8281E05A806F045FB05A806F0D2F986
:105CB000020092B205A92000FAF725FB012084F822
:105CC000B40205F07DBF00BF2C240208B81A0208F8
:105CD000012505F075BF012505F072BFDFF8F01D45
:105CE0002000FAF7A7FB002802D10020002834D0BA
:105CF0002000FAF797FB01212000FAF752FB002859
:105D000002D10020002825D02000FAF7D1FBDFF8CF
:105D1000580A80ED180ADFF8500A006E07F0D6FA2C
:105D200002000B00DFF81C1E05A806F003FB05A807
:105D300006F090F9020092B205A92000FAF7E3FA02
:105D4000012084F8B40205F03BBF00BF40240208E4
:105D5000881A0208012505F033BFDFF8EC1D20008A
:105D6000FAF768FB002802D10020002833D0200079
:105D7000FAF758FB01212000FAF713FB002802D1A3
:105D80000020002824D02000FAF792FBDFF8D80981
:105D900080ED1E0ADFF8D009806F07F097FA020045
:105DA0000B00DFF8181E05A806F0C4FA05A806F0D7
:105DB00051F9020092B205A92000FAF7A4FA0120D5
:105DC00084F8B40205F0FCBE542402082411020831
:105DD000012505F0F5BEDFF8581E2000FAF72AFB72
:105DE000002802D10020002837D02000FAF71AFB43
:105DF00001212000FAF7D5FA002802D1002000285E
:105E000028D02000FAF754FBDFF85C0980ED230A64
:105E1000DFF85409D0F88C0007F058FA02000B00A4
:105E2000DFF8101E05A806F085FA05A806F012F99D
:105E3000020092B205A92000FAF765FA012084F861
:105E4000B40205F0BDBE00BF642A0208A01A020811
:105E5000742A0208012505F0B3BEDFF84C1E2000AD
:105E6000FAF7E8FA002802D10020002835D02000F7
:105E7000FAF7D8FA01212000FAF793FA002802D1A4
:105E80000020002826D02000FAF712FBDFF8D808FF
:105E900080ED270ADFF8D008D0F89C0007F016FA4A
:105EA00002000B00DFF8041E05A806F043FA05A85F
:105EB00006F0D0F8020092B205A92000FAF723FA02
:105EC000012084F8B40205F07BBE00BFD01A02089E
:105ED000E42F0208012505F073BEDFF8441E200000
:105EE000FAF7A8FA002802D10020002835D02000B7
:105EF000FAF798FA01212000FAF753FA002802D1A4
:105F00000020002826D02000FAF7D2FADFF858083F
:105F100080ED330ADFF85008D0F8CC0007F0D6F94E
:105F200002000B00DFF8FC1D05A806F003FA05A827
:105F300006F090F8020092B205A92000FAF7E3F902
:105F4000012084F8B40205F03BBE00BF842A020899
:105F5000F02F0208012505F033BEDFF83C1E2000BB
:105F6000FAF768FA002802D10020002835D0200076
:105F7000FAF758FA01212000FAF713FA002802D1A3
:105F80000020002826D02000FAF792FADFF8D80780
:105F900080ED340ADFF8D007D0F8D00007F096F98A
:105FA00002000B00DFF8F41D05A806F0C3F905A8F0
:105FB00006F050F8020092B205A92000FAF7A3F902
:105FC000012084F8B40205F0FBBD00BF942A02084A
:105FD000FC2F0208012505F0F3BDDFF8341E200078
:105FE000FAF728FA002802D10020002835D0200036
:105FF000FAF718FA01212000FAF7D3F9002802D1A4
:106000000020002826D02000FAF752FADFF85807BF
:1060100080ED350ADFF85007D0F8D40007F056F9C4
:1060200002000B00DFF8EC1D05A806F083F905A8B7
:1060300006F010F8020092B205A92000FAF763F901
:10604000012084F8B40205F0BBBD00BFA42A0208F9
:1060500008300208012505F0B3BDDFF8BC1D2000A3
:10606000FAF7E8F9002802D10020002837D02000F4
:10607000FAF7D8F901212000FAF793F9002802D1A4
:106080000020002828D02000FAF712FADFF8D806FE
:1060900080ED360ADFF8D006D0F8D80007F016F900
:1060A00002000B00DFF8741D05A806F043F905A8EF
:1060B00005F0D0FF020092B205A92000FAF723F9FB
:1060C000012084F8B40205F07BBD00BF68240208FB
:1060D000143002087C240208012505F071BDDFF8A8
:1060E000401D2000FAF7A6F9002802D10020002860
:1060F00035D02000FAF796F901212000FAF751F97E
:10610000002802D10020002826D02000FAF7D0F97C
:10611000DFF8540680ED720ADFF84C06D0F8C801AB
:1061200007F0D4F802000B00DFF8F81C05A806F011
:1061300001F905A805F08EFF020092B205A9200022
:10614000FAF7E1F8012084F8B40205F039BD00BF88
:106150002030020890240208012505F031BDDFF847
:10616000081E2000FAF766F9002802D10020002856
:1061700035D02000FAF756F901212000FAF711F97D
:10618000002802D10020002826D02000FAF790F93C
:10619000DFF8D40580ED370ADFF8CC05D0F8DC0055
:1061A00007F094F802000B00DFF8C01D05A806F008
:1061B000C1F805A805F04EFF020092B205A9200023
:1061C000FAF7A1F8012084F8B40205F0F9BC00BF89
:1061D000A42402085C110208012505F0F1BCDFF8D7
:1061E000901D2000FAF726F9002802D1002000288F
:1061F00035D02000FAF716F901212000FAF7D1F87E
:10620000002802D10020002826D02000FAF750F9FB
:10621000DFF8540580ED3A0ADFF84C05D0F8E800C5
:1062200007F054F802000B00DFF8481D05A806F03F
:1062300081F805A805F00EFF020092B205A9200022
:10624000FAF761F8012084F8B40205F0B9BC00BF88
:10625000881D020840110208012505F0B1BCDFF8D5
:10626000181D2000FAF7E6F8002802D100200028C7
:1062700031D02000FAF7D6F801212000FAF791F882
:10628000002802D10020002822D02000FAF7EDF8E3
:106290000700DFF8D40480F8E170DFF8CC0490F850
:1062A000E120DFF8D81C05A806F044F805A805F0A1
:1062B000D1FE020092B205A92000FAF724F80120CD
:1062C00084F8B40205F07CBCA01D0208940A020800
:1062D000012505F075BCDFF8A81C2000FAF7AAF824
:1062E000002802D10020002833D02000FAF79AF8C5
:1062F00001212000FAF755F8002802D100200028DB
:1063000024D02000FAF7B1F80700DFF85C0480F829
:106310004070DFF8540490F84020DFF8681C05A8AE
:1063200006F008F805A805F095FE020092B205A94E
:106330002000F9F7E8FF012084F8B40205F040BC22
:10634000A813020804070208B81D0208012505F079
:1063500037BCDFF8341C2000FAF76CF8002802D1B3
:106360000020002831D02000FAF75CF8012120003D
:10637000FAF717F8002802D10020002822D02000C8
:10638000FAF773F80700DFF8E003A0F82475DFF8E8
:10639000D803B0F82425DFF8F81B05A805F0CAFFDC
:1063A00005A805F057FE020092B205A92000F9F7F2
:1063B000AAFF012084F8B40205F002BCB40A020866
:1063C000C4130208012505F0FBBBDFF8C81B200041
:1063D000FAF730F8002802D1002000282FD0200042
:1063E000FAF720F801212000F9F7DBFF002802D19D
:1063F0000020002820D02000FAF737F80700DA48FC
:10640000A0F8E270D848B0F9E220DFF88C1B05A8AC
:1064100005F090FF05A805F01DFE020092B205A947
:106420002000F9F770FF012084F8B40205F0C8BB22
:10643000D40A0208D01D0208012505F0C1BBDFF80F
:106440005C1B2000F9F7F6FF002802D1002000288D
:106450002FD02000F9F7E6FF01212000F9F7A1FF76
:10646000002802D10020002820D02000F9F7FDFFED
:106470000700BD48A0F8F470BB48B0F9F420DFF87D
:10648000201B05A805F056FF05A805F0E3FD020056
:1064900092B205A92000F9F736FF012084F8B40272
:1064A00005F08EBBF40A0208B8240208012505F0A5
:1064B00087BBDFF8541E2000F9F7BCFF002802D18B
:1064C000002000282FD02000F9F7ACFF0121200088
:1064D000F9F767FF002802D10020002820D0200013
:1064E000F9F7C3FF0700A048A0F8F6709E48B0F97E
:1064F000F620DFF8181E05A805F01CFF05A805F01A
:10650000A9FD020092B205A92000F9F7FCFE0120C6
:1065100084F8B40205F054BBB0190208CC24020878
:10652000012505F04DBBDFF8E81D2000F9F782FFDB
:10653000002802D1002000282FD02000F9F772FF98
:1065400001212000F9F72DFF002802D100200028AA
:1065500020D02000F9F789FF07008348A0F8F870E1
:106560008148B0F9F820DFF8AC1D05A805F0E2FE7F
:1065700005A805F06FFD020092B205A92000F9F709
:10658000C2FE012084F8B40205F01ABBD010020844
:10659000E0240208012505F013BBDFF87C1D200074
:1065A000F9F748FF002802D1002000282FD0200052
:1065B000F9F738FF01212000F9F7F3FE002802D196
:1065C0000020002820D02000F9F74FFF0700664880
:1065D000A0F8E4706448B0F9E420DFF8381E05A89C
:1065E00005F0A8FE05A805F035FD020092B205A948
:1065F0002000F9F788FE012084F8B40205F0E0BA23
:10660000C8190208140D0208012505F0D9BADFF8EF
:10661000081E2000F9F70EFF002802D100200028F4
:106620002FD02000F9F7FEFE01212000F9F7B9FE76
:10663000002802D10020002820D02000F9F715FF03
:1066400007004948A0F8FA704748B0F8FA20DFF888
:10665000601E05A805F06EFE05A805F0FBFC020013
:1066600092B205A92000F9F74EFE012084F8B40289
:1066700005F0A6BABC060208E0130208012505F0E1
:106680009FBADFF8301E2000F9F7D4FE002802D1AF
:106690000020002831D02000F9F7C4FE012120009D
:1066A000F9F77FFE002802D10020002822D0200028
:1066B000F9F7FEFE2C4880ED1C0A2B48006F06F00F
:1066C00005FE02000B00DFF8F01D05A805F032FE04
:1066D00005A805F0BFFC020092B205A92000F9F759
:1066E00012FE012084F8B40205F06ABAE00602083E
:1066F000E81D0208012505F063BADFF85C1E2000E2
:10670000F9F798FE002802D10020002835D020009B
:10671000F9F788FE01212000F9F743FE002802D195
:106720000020002826D02000F9F7C2FE0E4880ED98
:106730003B0A0D48D0F8EC0006F0C8FD02000B0043
:10674000DFF8181E05A805F0F5FD05A805F082FC88
:10675000020092B205A92000F9F7D5FD012084F8C6
:10676000B40205F02DBA00BF10180010140A020878
:10677000001E0208012505F023BADFF8601E200084
:10678000F9F758FE002802D10020002835D020005B
:10679000F9F748FE01212000F9F703FE002802D195
:1067A0000020002826D02000F9F782FEDFF8300E06
:1067B00080ED3C0ADFF8280ED0F8F00006F086FDE8
:1067C00002000B00DFF81C1E05A805F0B3FD05A8AC
:1067D00005F040FC020092B205A92000F9F793FDF4
:1067E000012084F8B40205F0EBB900BF08110208DB
:1067F000F4240208012505F0E3B9DFF8641E200047
:10680000F9F718FE002802D10020002835D020001A
:10681000F9F708FE01212000F9F7C3FD002802D195
:106820000020002826D02000F9F742FEDFF8B00D46
:1068300080ED3F0ADFF8A80DD0F8FC0006F046FD19
:1068400002000B00DFF81C1E05A805F073FD05A86B
:1068500005F000FC020092B205A92000F9F753FDF3
:10686000012084F8B40205F0ABB900BFE0190208BA
:1068700008250208012505F0A3B9DFF8701E2000E5
:10688000F9F7D8FD002802D10020002835D02000DB
:10689000F9F7C8FD01212000F9F783FD002802D196
:1068A0000020002826D02000F9F702FEDFF8300D86
:1068B00080ED220ADFF8280DD0F8880006F006FDEA
:1068C00002000B00DFF8281E05A805F033FD05A81F
:1068D00005F0C0FB020092B205A92000F9F713FDF4
:1068E000012084F8B40205F06BB900BFEC10020877
:1068F0001C250208012505F063B9DFF8701E200091
:10690000F9F798FD002802D10020002831D020009E
:10691000F9F788FD01212000F9F743FD002802D195
:106920000020002822D02000F9F79FFD0700DFF8A3
:10693000B00CA0F80071DFF8A80CB0F90021DFF866
:10694000301E05A805F0F6FC05A805F083FB020043
:1069500092B205A92000F9F7D6FC012084F8B40210
:1069600005F02EB9F81902082C300208012505F0AF
:1069700027B9DFF87C1E2000F9F75CFD002802D162
:106980000020002831D02000F9F74CFD0121200023
:10699000F9F707FD002802D10020002822D02000AE
:1069A000F9F763FD0700DFF8380CA0F80271DFF893
:1069B000300CB0F90221DFF8401E05A805F0BAFC42
:1069C00005A805F047FB020092B205A92000F9F7DF
:1069D0009AFC012084F8B40205F0F2B88429020878
:1069E00038300208012505F0EBB8DFF8881E2000DA
:1069F000F9F720FD002802D10020002831D0200026
:106A0000F9F710FD01212000F9F7CBFC002802D195
:106A10000020002822D02000F9F727FD0700DFF82A
:106A2000C00BA0F80671DFF8B80BB0F90621DFF84B
:106A3000481E05A805F07EFC05A805F00BFB02002A
:106A400092B205A92000F9F75EFC012084F8B40297
:106A500005F0B6B83025020844300208012505F0DB
:106A6000AFB8DFF8181E2000F9F7E4FC002802D1C7
:106A70000020002831D02000F9F7D4FC01212000AB
:106A8000F9F78FFC002802D10020002822D0200036
:106A9000F9F7EBFC0700DFF8480BA0F80471DFF80A
:106AA000400BB0F90421DFF8581E05A805F042FCA0
:106AB00005A805F0CFFA020092B205A92000F9F767
:106AC00022FC012084F8B40205F07AB844250208BB
:106AD00058250208012505F073B8DFF8281E2000AC
:106AE000F9F7A8FC002802D10020002831D02000AE
:106AF000F9F798FC01212000F9F753FC002802D196
:106B00000020002822D02000F9F7AFFC0700DFF8B2
:106B1000D00AA0F80871DFF8C80AB0F80821DFF839
:106B2000681E05A805F006FC05A805F093FA02000A
:106B300092B205A92000F9F7E6FB012084F8B4021F
:106B400005F03EB8181E0208FC130208012505F0E6
:106B500037B8DFF8381E2000F9F76CFC002802D1A6
:106B6000002000282FD02000F9F75CFC0121200034
:106B7000F9F717FC002802D10020002820D02000BF
:106B8000F9F773FC0700DFF8580A80F88871DFF81E
:106B9000500A90F88821DFF8781E05A805F0CAFB96
:106BA00005A805F057FA020092B205A92000F9F7EE
:106BB000AAFB012084F8B40205F002B8340A0208E6
:106BC000012504F0FDBFDFF84C1E2000F9F732FC70
:106BD000002802D10020002831D02000F9F722FC43
:106BE00001212000F9F7DDFB002802D10020002858
:106BF00022D02000F9F739FC0700DFF8E40980F81B
:106C0000CA74DFF8DC0990F8CA24DFF88C1E05A8E6
:106C100005F090FB05A805F01DFA020092B205A947
:106C20002000F9F770FB012084F8B40204F0C8BF1B
:106C30001814020828070208012504F0C1BFDFF874
:106C40005C1E2000F9F7F6FB002802D10020002886
:106C500031D02000F9F7E6FB01212000F9F7A1FB74
:106C6000002802D10020002822D02000F9F7FDFBE7
:106C70000700DFF86C0980F8CC74DFF8640990F83D
:106C8000CC24DFF81C1E05A805F054FB05A805F070
:106C9000E1F9020092B205A92000F9F734FB0120C6
:106CA00084F8B40204F08CBF301E0208340D0208D0
:106CB000012504F085BFDFF86C1E2000F9F7BAFB50
:106CC000002802D10020002831D02000F9F7AAFBCB
:106CD00001212000F9F765FB002802D100200028DF
:106CE00022D02000F9F7C1FB0700DFF8F408A0F874
:106CF000C471DFF8EC08B0F8C421DFF82C1E05A839
:106D000005F018FB05A805F0A5F9020092B205A947
:106D10002000F9F7F8FA012084F8B40204F050BF1B
:106D200048080208F8030208012504F049BFDFF80B
:106D30007C1E2000F9F77EFB002802D100200028ED
:106D400031D02000F9F76EFB01212000F9F729FB73
:106D5000002802D10020002822D02000F9F785FB6E
:106D60000700DFF87C0880F8C874DFF8740890F832
:106D7000C824DFF83C1E05A805F0DCFA05A805F0DC
:106D800069F9020092B205A92000F9F7BCFA0120C6
:106D900084F8B40204F014BF6C080208C8020208A8
:106DA000012504F00DBFDFF88C1E2000F9F742FB2F
:106DB000002802D10020002839D02000F9F732FB4A
:106DC00001212000F9F7EDFA002802D10020002867
:106DD0002AD02000F9F749FB0700DFF80408A0F8E3
:106DE000CE74DFF8FC07B0F9CE24DFF84C1E05A8FE
:106DF00005F0A0FA05A805F02DF9020092B205A948
:106E00002000F9F780FA012084F8B40204F0D8BE1B
:106E1000481E0208140B020834140208340B02083E
:106E20006C25020804120208012504F0C9BE57A10E
:106E30002000F9F7FFFA002803D10020002800F015
:106E4000C0802000F9F7EEFA01212000F9F7A9FA35
:106E5000002803D10020002800F0B0802000F9F7BE
:106E600004FB0700381E0A2880F0A5802000F9F7EF
:106E7000D9FA01212000F9F794FA002803D1002063
:106E8000002800F095802000F9F712FBB0EE408A50
:106E90002000F9F7C7FA01212000F9F782FA00284B
:106EA00003D10020002800F080802000F9F700FBCB
:106EB000F0EE408A2000F9F7B5FA01212000F9F739
:106EC00070FA002802D1002000286BD02000F9F7CA
:106ED000CCFA00EE100AB8EEC00A0C20DFF800175A
:106EE00000FB071080ED448A0C20DFF8F41600FB4D
:106EF0000710C0ED458A0C20DFF8E41600FB0710F0
:106F000080ED460A0C20DFF8D81600FB071090ED44
:106F1000460ABDEEC00A10EE100A00B204900C2022
:106F2000DFF8BC1600FB0710D0F8140106F0CEF90C
:106F3000CDE902010C20DFF8A81600FB0710D0F8FD
:106F4000100106F0C3F9CDE900013A00DFF8501E48
:106F500005A805F0EFF905A805F07CF8010005A8E3
:106F600005F02EF904F02CBE50140208540B020850
:106F7000B42A020888220208C42A020860220208F1
:106F8000601E020878110208540D02087770000094
:106F90004C0702085030020894290208D42A02083B
:106FA0009C220208012504F00BBE012504F008BE56
:106FB000012504F005BE012504F002BE012504F000
:106FC000FFBDDFF8381E2000F9F734FA002803D19E
:106FD0000020002800F0D6802000F9F723FA0121D4
:106FE0002000F9F7DEF9002803D10020002800F086
:106FF000C6802000F9F739FA0600381E182880F0FC
:10700000BB802000F9F70EFA01212000F9F7C9F939
:10701000002803D10020002800F0AB802000F9F701
:1070200024FA07002000F9F7FDF901212000F9F703
:10703000B8F9002803D10020002800F09780200034
:10704000F9F713FA80462000F9F7ECF90121200046
:10705000F9F7A7F9002803D10020002800F0838069
:107060002000F9F702FA81462000F9F7DBF9012147
:107070002000F9F796F9002802D1002000286FD0EF
:107080002000F9F7F2F982462000F9F7CBF9012147
:107090002000F9F786F9002802D1002000285CD0F2
:1070A0002000F9F7E2F9F6B2DFF8341511EBC6016A
:1070B00081F8E871F6B2DFF8281511EBC60181F806
:1070C000E981F6B2DFF8181511EBC601A1F8EA91D3
:1070D000F6B2DFF80C1511EBC601A1F8EEA1F6B27D
:1070E000DFF8FC1411EBC601A1F8EC01F6B2DFF8F1
:1070F000F00410EBC600B0F8EC010390F6B2DFF834
:10710000E00410EBC600B0F8EE010290F6B2DFF832
:10711000D00410EBC600B0F8EA010190F6B2DFF837
:10712000C00410EBC60090F8E9010090F6B2DFF859
:10713000B00410EBC60090F8E831F6B23200DFF888
:10714000381E05A805F0F6F805A804F083FF010035
:1071500005A805F035F804F033BD012504F030BD75
:10716000012504F02DBD012504F02ABD012504F000
:1071700027BD012504F024BD012504F021BD012512
:1071800004F01EBDDFF84C1E2000F9F753F900286B
:1071900003D10020002800F0D6802000F9F742F942
:1071A00001212000F9F7FDF8002803D10020002874
:1071B00000F0C6802000F9F758F90600381E18289C
:1071C00080F0BB802000F9F72DF901212000F9F7AC
:1071D000E8F8002803D10020002800F0AB80200050
:1071E000F9F743F907002000F9F71CF90121200005
:1071F000F9F7D7F8002803D10020002800F0978085
:107200002000F9F732F980462000F9F70BF9012147
:107210002000F9F7C6F8002803D10020002800F06C
:1072200083802000F9F721F981462000F9F7FAF868
:1072300001212000F9F7B5F8002802D1002000282C
:107240006FD02000F9F711F982462000F9F7EAF82B
:1072500001212000F9F7A5F8002802D1002000281C
:107260005CD02000F9F701F9F6B2DD4911EBC60157
:1072700081F8A872F6B2DA4911EBC60181F8A98249
:10728000F6B2D74911EBC601A1F8AA92F6B2D449D9
:1072900011EBC601A1F8AEA2F6B2D14911EBC601BD
:1072A000A1F8AC02F6B2CE4810EBC600B0F8AC02C2
:1072B0000390F6B2CA4810EBC600B0F8AE020290D6
:1072C000F6B2C74810EBC600B0F8AA020190F6B2B9
:1072D000C34810EBC60090F8A9020090F6B2C0486F
:1072E00010EBC60090F8A832F6B23200DFF8881C26
:1072F00005A805F01FF805A804F0ACFE010005A8DC
:1073000004F05EFF04F05CBCE42A0208B02202082C
:107310005C300208C4290208F42A0208012504F09E
:107320004FBC012504F04CBC012504F049BC0125EB
:1073300004F046BC012504F043BC012504F040BC28
:10734000012504F03DBCC8A12000F9F773F800281E
:1073500003D10020002800F0C3802000F9F762F874
:1073600001212000F9F71DF8002803D10020002892
:1073700000F0B3802000F9F778F80600F6B2B6F115
:107380000A00062880F0A6802000F9F74BF80121BA
:107390002000F9F706F8002803D10020002800F0AB
:1073A00096802000F9F761F80700FFB2002F00F087
:1073B0008B80FFB20A2F80F287802000F9F732F825
:1073C00001212000F8F7EDFF002802D1002000285D
:1073D00077D02000F9F749F840B210F16401C929CB
:1073E0006CD2FFB2F6B20A217D4A01FB0621791860
:1073F00081F86803F6B23200DFF8DC1D05A804F05E
:1074000099FF05A804F026FE010005A804F0D8FEA7
:1074100001273CE074220208781E0208BFB2F6B2CF
:107420000A206F4900FB0610381890F968030028FD
:107430002CD0BFB2F6B20A20694900FB06103818FA
:1074400090F9680300280AD4CAA105A804F072FFC5
:1074500005A804F0FFFD010005A804F0B1FEBFB2CD
:107460003B00BFB2F6B20A205D4900FB0610381897
:1074700090F96823DFF8F81D05A804F05BFF05A864
:1074800004F0E8FD010005A804F09AFE7F1CBFB2DD
:107490000A2FC3DBD7A105A804F04CFF05A804F010
:1074A000D9FD010005A804F08BFE04F089BB00BFE4
:1074B00094110208042B0208901E0208012504F012
:1074C0007FBB012504F07CBB012504F079BB0125BD
:1074D00004F076BB012504F073BB012504F070BBFA
:1074E000DFF8E01D2000F8F7A5FF002802D10020FA
:1074F000002838D02000F8F795FF01212000F8F788
:1075000050FF002802D10020002829D02000F8F7E1
:10751000CFFF334880ED630ADFF8AC0D00680F2120
:1075200001712F48D0F88C0105F0D0FE02000B004D
:10753000DFF8981D05A804F0FDFE05A804F08AFDFB
:10754000020092B205A92000F8F7DDFE012084F8C0
:10755000B40204F035BB00BF68300208A429020859
:10756000012504F02DBBDFF8FC1D2000F8F762FFB9
:10757000002802D10020002839D02000F8F752FF5F
:1075800001212000F8F70DFF002802D1002000287B
:107590002AD02000F8F78CFF114880ED640ADFF84C
:1075A000280D00680F2101710D48D0F8900105F0F9
:1075B0008DFE02000B00DFF8B01D05A804F0BAFE36
:1075C00005A804F047FD020092B205A92000F8F7D3
:1075D0009AFE012084F8B40204F0F2BA7430020872
:1075E00010180010B4290208012504F0E9BADFF8E8
:1075F0007C1D2000F8F71EFF002802D10020002883
:1076000037D02000F8F70EFF01212000F8F7C9FE5F
:10761000002802D10020002828D02000F8F748FFD9
:10762000DFF8E00D80ED6C0ADFF8D80DD0F8B0017E
:1076300005F04CFE02000B00DFF8CC1D05A804F09D
:1076400079FE05A804F006FD020092B205A920000B
:10765000F8F759FE012084F8B40204F0B1BA00BF73
:107660006C140208700702086D697800012504F0A7
:10767000A7BADFF8981D2000F8F7DCFE002802D139
:107680000020002839D02000F8F7CCFE012120008E
:10769000F8F787FE002802D1002000282AD0200019
:1076A000F8F706FFDFF85C0D80ED650ADFF8180CCF
:1076B00000680F210171DFF84C0DD0F8940105F03E
:1076C00005FE02000B00DFF8E41D05A804F032FE01
:1076D00005A804F0BFFC020092B205A92000F8F74B
:1076E00012FE012084F8B40204F06ABAA81E02084F
:1076F000540A0208012504F063BADFF8B41D200023
:10770000F8F798FE002802D10020002837D020008A
:10771000F8F788FE01212000F8F743FE002802D187
:107720000020002828D02000F8F7C2FEDFF8D40C93
:1077300080ED6D0ADFF8CC0CD0F8B40105F0C6FD81
:1077400002000B00DFF86C1D05A804F0F3FD05A88E
:1077500004F080FC020092B205A92000F8F7D3FDE6
:10776000012084F8B40204F02BBA00BFC01E020846
:10777000B01102082B000000012504F021BADFF847
:10778000D41D2000F8F756FE002802D10020002862
:1077900037D02000F8F746FE01212000F8F701FE5F
:1077A000002802D10020002828D02000F8F780FE11
:1077B000DFF8500C80ED6F0ADFF8480CD0F8BC0100
:1077C00005F084FD02000B00DFF88C1D05A804F015
:1077D000B1FD05A804F03EFC020092B205A920000C
:1077E000F8F791FD012084F8B40204F0E9B900BF74
:1077F000802502080D0A0000E81A0208012504F09D
:10780000DFB9DFF8581D2000F8F714FE002802D178
:107810000020002837D02000F8F704FE01212000C6
:10782000F8F7BFFD002802D10020002828D0200052
:10783000F8F73EFEDFF8CC0B80ED700ADFF8C40BE2
:10784000D0F8C00105F042FD02000B00DFF8AC1DCE
:1078500005A804F06FFD05A804F0FCFB020092B23D
:1078600005A92000F8F74FFD012084F8B40204F0C8
:10787000A7B900BFD81E0208CC110208F01E0208EA
:10788000012504F09DB9DFF8D81D2000F8F7D2FDDE
:10789000002802D10020002839D02000F8F7C2FDCE
:1078A00001212000F8F77DFD002802D100200028EA
:1078B0002AD02000F8F7FCFDDFF8480B80ED660ABF
:1078C000DFF8040A00680F210171DFF8380BD0F8E7
:1078D000980105F0FBFC02000B00DFF8C41D05A8B1
:1078E00004F028FD05A804F0B5FB020092B205A93A
:1078F0002000F8F708FD012084F8B40204F060B914
:10790000740B020890080208012504F059B9DFF849
:10791000941D2000F8F78EFD002802D100200028D9
:1079200039D02000F8F77EFD01212000F8F739FD5D
:10793000002802D1002000282AD02000F8F7B8FD46
:10794000DFF8C00A80ED670ADFF87C0900680F21C4
:107950000171DFF8B00AD0F89C0105F0B7FC020015
:107960000B00DFF8441D05A804F0E4FC05A804F0B2
:1079700071FB020092B205A92000F8F7C4FC0120B7
:1079800084F8B40204F01CB920040208142B020885
:10799000012504F015B9DFF8B01D2000F8F74AFD05
:1079A000002802D10020002839D02000F8F73AFD45
:1079B00001212000F8F7F5FC002802D10020002862
:1079C0002AD02000F8F774FDDFF8380A80ED680A45
:1079D000DFF8F40800680F210171DFF8280AD0F8F9
:1079E000A00105F073FC02000B00DFF8601D05A884
:1079F00004F0A0FC05A804F02DFB020092B205A93A
:107A00002000F8F780FC012084F8B40204F0D8B814
:107A100010220208081F0208012504F0D1B8DFF87F
:107A2000CC1D2000F8F706FD002802D10020002818
:107A30003BD02000F8F7F6FC01212000F8F7B1FC5C
:107A4000002802D1002000282CD02000F8F730FDBB
:107A5000DFF8B00980ED690ADFF86C0800680F21D3
:107A60000171DFF8A009D0F8A40105F02FFC020095
:107A70000B00DFF87C1D05A804F05CFC05A804F0F1
:107A8000E9FA020092B205A92000F8F73CFC0120B7
:107A900084F8B40204F094B894090208242B020874
:107AA000AC210208012504F08BB8DFF8481D200046
:107AB000F8F7C0FC002802D10020002839D02000AF
:107AC000F8F7B0FC01212000F8F76BFC002802D188
:107AD000002000282AD02000F8F7EAFCDFF824096B
:107AE00080ED6A0ADFF8E00700680F210171DFF816
:107AF0001409D0F8A80105F0E9FB02000B00DFF83B
:107B0000941D05A804F016FC05A804F0A3FA0200D1
:107B100092B205A92000F8F7F6FB012084F8B40220
:107B200004F04EB88814020894070208012504F0F6
:107B300047B8DFF8641D2000F8F77CFC002802D16C
:107B40000020002839D02000F8F76CFC012120002B
:107B5000F8F727FC002802D1002000282AD02000B6
:107B6000F8F7A6FCDFF89C0880ED6B0ADFF85807F1
:107B700000680F210171DFF88C08D0F8AC0105F026
:107B8000A5FB02000B00DFF8B01D05A804F0D2FB36
:107B900005A804F05FFA020092B205A92000F8F7E8
:107BA000B2FB012084F8B40204F00AB8342B0208B6
:107BB00024220208012504F003B8DFF8801D20000C
:107BC000F8F738FC002802D10020002839D0200026
:107BD000F8F728FC01212000F8F7E3FB002802D188
:107BE000002000282AD02000F8F762FCDFF81408F3
:107BF00080ED6E0ADFF8D00600680F210171DFF812
:107C00000408D0F8B80105F061FB02000B00DFF8B2
:107C1000301D05A804F08EFB05A804F01BFA020035
:107C200092B205A92000F8F76EFB012084F8B40297
:107C300003F0C6BF201F02083C120208012503F012
:107C4000BFBFDFF89C1D2000F8F7F4FB002802D12D
:107C50000020002838D02000F8F7E4FB01212000A4
:107C6000F8F79FFB002802D10020002829D020002F
:107C7000F8F7FBFB0700781E03281FD2DFF8840704
:107C800080F88971DFF84006006801214171DFF852
:107C9000740790F88921DFF8AC1D05A804F04AFBB1
:107CA00005A804F0D7F9020092B205A92000F8F760
:107CB0002AFB012084F8B40203F082BF012503F0FF
:107CC0007FBF012503F07CBFDFF8B81D2000F8F767
:107CD000B1FB002802D10020002842D02000F8F794
:107CE000A1FB01212000F8F75CFB002802D1002055
:107CF000002833D02000F8F7B8FB0700002F01D090
:107D0000012700E00027002F0AD0DFF8F806D0F89E
:107D1000800050F00100DFF8EC16C1F8800009E0A7
:107D2000DFF8E006D0F8800040084000DFF8D41605
:107D3000C1F880003A00DFF8C81D05A804F0FAFA7F
:107D400005A804F087F9020092B205A92000F8F70F
:107D5000DAFA012084F8B40203F032BF012503F0FF
:107D60002FBFDFF8A01D2000F8F764FB002802D128
:107D70000020002847D02000F8F754FB0121200004
:107D8000F8F70FFB002802D10020002838D020008F
:107D9000F8F76BFB0700002F04D0012703E000BFBA
:107DA000301B02080027002F0AD0DFF85806D0F851
:107DB000800050F00200DFF84C16C1F8800009E0A6
:107DC000DFF84006D0F8800030F00200DFF834160B
:107DD000C1F880003A00DFF8A81D05A804F0AAFA4F
:107DE00005A804F037F9020092B205A92000F8F7BF
:107DF0008AFA012084F8B40203F0E2BE6C32020871
:107E0000012503F0DDBEDFF87C1D2000F8F712FB32
:107E1000002802D10020002842D02000F8F702FB01
:107E200001212000F8F7BDFA002802D10020002827
:107E300033D02000F8F719FB0700002F01D00127ED
:107E400000E00027002F0AD0DFF8B805D0F8800046
:107E500050F00400DFF8AC15C1F8800009E0DFF84D
:107E6000A405D0F8800030F00400DFF89815C1F8C0
:107E700080003A00DFF8881D05A804F05BFA05A829
:107E800004F0E8F8020092B205A92000F8F73BFAE6
:107E9000012084F8B40203F093BE012503F090BEE4
:107EA000DFF8D81D2000F8F7C5FA002802D100201D
:107EB000002842D02000F8F7B5FA01212000F8F799
:107EC00070FA002802D10020002833D02000F8F7F3
:107ED000CCFA0700002F01D0012700E00027002F77
:107EE0000AD0DFF82005D0F8800050F40010DFF849
:107EF0001415C1F8800009E0DFF80805D0F880000B
:107F000030F40010DFF8FC14C1F880003A00DFF80C
:107F1000701D05A804F00EFA05A804F09BF80200F5
:107F200092B205A92000F8F7EEF9012084F8B40216
:107F300003F046BE012503F043BEDFF8C01D20005C
:107F4000F8F778FA002802D10020002847D0200056
:107F5000F8F768FA01212000F8F723FA002802D187
:107F60000020002838D02000F8F77FFA0700002F03
:107F700004D0012703E000BF8C0002080027002F77
:107F80000AD0DFF88004D0F8800050F40030DFF829
:107F90007414C1F8800009E0DFF86804D0F88000AC
:107FA00030F40030DFF85C14C1F880003A00DFF8EC
:107FB000C81D05A804F0BEF905A804F04BF802009E
:107FC00092B205A92000F8F79EF9012084F8B402C6
:107FD00003F0F6BD74320208012503F0F1BDDFF8AD
:107FE0009C1D2000F8F726FA002802D10020002866
:107FF00042D02000F8F716FA01212000F8F7D1F955
:10800000002802D10020002833D02000F8F72DFAF4
:108010000700002F01D0012700E00027002F0AD021
:10802000DFF8E003D0F8800050F00800DFF8D41348
:10803000C1F8800009E0DFF8CC03D0F8800030F010
:108040000800DFF8C013C1F880003A00DFF8A81D6F
:1080500005A804F06FF905A803F0FCFF020092B236
:1080600005A92000F8F74FF9012084F8B40203F0C5
:10807000A7BD012503F0A4BDDFF8801D2000F8F79F
:10808000D9F9002802D1002000283ED02000F8F7BE
:10809000C9F901212000F8F784F9002802D1002055
:1080A00000282FD02000F8F7E0F90700002F01D0BA
:1080B000012700E00027002F08D0D248D0F8800028
:1080C00050F01000CF49C1F8800007E0CD48D0F84B
:1080D000800030F01000CB49C1F880003A00DFF892
:1080E000BC1D05A804F026F905A803F0B3FF0200A3
:1080F00092B205A92000F8F706F9012084F8B4022D
:1081000003F05EBD012503F05BBDDFF8941D200088
:10811000F8F790F9002802D1002000283ED0200076
:10812000F8F780F901212000F8F73BF9002802D187
:10813000002000282FD02000F8F797F90700002F23
:1081400001D0012700E00027002F08D0AD48D0F86B
:10815000800050F02000AB49C1F8800007E0A9483A
:10816000D0F8800030F02000A649C1F880003A0025
:10817000DFF8D01D05A804F0DDF805A803F06AFFBC
:10818000020092B205A92000F8F7BDF8012084F89A
:10819000B40203F015BD012503F012BDDFF8A81DE0
:1081A0002000F8F747F9002802D10020002840D02D
:1081B0002000F8F737F901212000F8F7F2F800283D
:1081C00002D10020002831D02000F8F74EF9070036
:1081D000002F03D0012702E0442B02080027002FC4
:1081E00008D08848D0F8800050F040008549C1F898
:1081F000800007E08348D0F8800030F040008149DB
:10820000C1F880003A00DFF8E41D05A804F092F8F8
:1082100005A803F01FFF020092B205A92000F8F79D
:1082200072F8012084F8B40203F0CABC012503F0FF
:10823000C7BCDFF8BC1D2000F8F7FCF8002802D10D
:108240000020002847D02000F8F7ECF8012120009A
:10825000F8F7A7F8002802D10020002838D0200025
:10826000F8F703F90700002F04D0012703E000BF4F
:108270007C3202080027002F08D06248D0F8800026
:1082800050F080005F49C1F8800007E05D48D0F8F9
:10829000800030F080005B49C1F880003A00DFF8D0
:1082A000F41D05A804F046F805A803F0D3FE02006B
:1082B00092B205A92000F8F726F8012084F8B4024C
:1082C00003F07EBC542B020874B40020201C02086A
:1082D000012503F075BCDFF8C01D2000F8F7AAF8EF
:1082E000002802D10020002845D02000F8F79AF895
:1082F00001212000F8F755F8002802D100200028BD
:1083000036D02000F8F7B1F80700002F01D0012780
:1083100000E00027002F08D03A48D0F8800050F441
:1083200080703849C1F8800007E03648D0F88000F6
:1083300030F480703349C1F880003A00DFF8FC1D4A
:1083400005A803F0F7FF05A803F084FE020092B22F
:1083500005A92000F7F7D7FF012084F8B40203F045
:108360002FBC00BF642B0208381C020894250208A9
:10837000012503F025BCDFF8C81D2000F8F75AF8E6
:10838000002802D10020002845D02000F8F74AF844
:1083900001212000F8F705F8002802D1002000286C
:1083A00036D02000F8F761F80700002F01D0012730
:1083B00000E00027002F08D01248D0F8800050F4C9
:1083C00000701049C1F8800007E00E48D0F8800026
:1083D00030F400700B49C1F880003A00DFF8041E49
:1083E00005A803F0A7FF05A803F034FE020092B22F
:1083F00005A92000F7F787FF012084F8B40203F0F5
:10840000DFBB00BF10180010C01B0208742B02084D
:10841000012503F0D5BBDFF8D01D2000F8F70AF8DE
:10842000002802D10020002849D02000F7F7FAFFE9
:1084300001212000F7F7B5FF002802D10020002815
:108440003AD02000F8F711F80700002F01D00127DB
:1084500000E00027002F0AD0DFF8900DD0F8800050
:1084600050F48060DFF8841DC1F8800009E0DFF877
:108470007C0DD0F8800030F48060DFF8701DC1F80A
:1084800080003A00DFF80C1E05A803F053FF05A892
:1084900003F0E0FD020092B205A92000F7F733FFD8
:1084A000012084F8B40203F08BBB00BF501C02080B
:1084B000A8250208D81B0208012503F081BBDFF8BC
:1084C000D81D2000F7F7B6FF002802D100200028B1
:1084D00049D02000F7F7A6FF01212000F7F761FF40
:1084E000002802D1002000283AD02000F7F7BDFF75
:1084F0000700002F01D0012700E00027002F0AD03D
:10850000DFF8E80CD0F8800050F40060DFF8DC1CE5
:10851000C1F8800009E0DFF8D40CD0F8800030F416
:108520000060DFF8C81CC1F880003A00DFF8101EB8
:1085300005A803F0FFFE05A803F08CFD020092B22F
:1085400005A92000F7F7DFFE012084F8B40203F04C
:1085500037BB00BF842B0208F01B0208942B0208D3
:10856000012503F02DBBDFF8DC1D2000F7F762FFCB
:10857000002802D10020002845D02000F7F752FF44
:1085800001212000F7F70DFF002802D1002000286C
:1085900036D02000F7F769FF0700002F01D0012730
:1085A00000E00027002F0AD0DFF8400CD0F8800050
:1085B00050F48050DFF8341CC1F8800009E0DFF887
:1085C0002C0CD0F8800030F48050DFF8201CC1F86B
:1085D00080003A00DFF8141E05A803F0ABFE05A8E2
:1085E00003F038FD020092B205A92000F7F78BFED8
:1085F000012084F8B40203F0E3BA00BF081C0208AB
:10860000012503F0DDBADFF8E81D2000F7F712FFBF
:10861000002802D1002000284BD02000F7F702FFED
:1086200001212000F7F7BDFE002802D1002000281C
:108630003CD02000F7F719FF0700002F01D00127D9
:1086400000E00027002F0DD0DFF8A00BD0F880004D
:1086500050F40050DFF8941BC1F880000CE000BF1C
:10866000A42B0208DFF8840BD0F8800030F400500F
:10867000DFF8781BC1F880003A00DFF81C1E05A85F
:1086800003F058FE05A803F0E5FC020092B205A92C
:108690002000F7F738FE012084F8B40203F090BA06
:1086A000481B0208B42B0208601B0208012503F0D6
:1086B00087BADFF8E81D2000F7F7BCFE002802D1DA
:1086C0000020002847D02000F7F7ACFE0121200051
:1086D000F7F767FE002802D10020002838D02000DC
:1086E000F7F7C3FE0700002F01D0012700E00027A5
:1086F000002F0AD0DFF8F40AD0F8800050F4804050
:10870000DFF8E81AC1F8800009E0DFF8E00AD0F8E5
:10871000800030F48040DFF8D41AC1F880003A00BD
:10872000DFF8201E05A803F005FE05A803F092FC63
:10873000020092B205A92000F7F7E5FD012084F8B8
:10874000B40203F03DBA00BFC42B0208781B020834
:10875000012503F035BADFF8F01D2000F7F76AFEB7
:10876000002802D10020002849D02000F7F75AFE47
:1087700001212000F7F715FE002802D10020002873
:108780003AD02000F7F771FE0700002F01D0012733
:1087900000E00027002F0AD0DFF8500AD0F8800050
:1087A00050F40040DFF8441AC1F8800009E0DFF817
:1087B0003C0AD0F8800030F40040DFF8301AC1F8ED
:1087C00080003A00DFF8281E05A803F0B3FD05A8D5
:1087D00003F040FC020092B205A92000F7F793FDD8
:1087E000012084F8B40203F0EBB900BFD42B0208D7
:1087F000901B0208E42B0208012503F0E1B9DFF821
:10880000F41D2000F7F716FE002802D100200028F2
:1088100047D02000F7F706FE01212000F7F7C1FD41
:10882000002802D10020002838D02000F7F71DFED4
:108830000700002F01D0012700E00027002F0AD0F9
:10884000DFF8A809D0F8800050F48030DFF89C19D8
:10885000C1F8800009E0DFF89409D0F8800030F416
:108860008030DFF88819C1F880003A00DFF82C1E4C
:1088700005A803F05FFD05A803F0ECFB020092B22F
:1088800005A92000F7F73FFD012084F8B40203F0AA
:1088900097B900BFA81B020880300208012503F029
:1088A0008FB9DFF8FC1D2000F7F7C4FD002802D1C6
:1088B0000020002849D02000F7F7B4FD0121200056
:1088C000F7F76FFD002802D1002000283AD02000E1
:1088D000F7F7CBFD0700002F01D0012700E00027AC
:1088E000002F0AD0DFF80409D0F8800050F40020EF
:1088F000DFF8F818C1F8800009E0DFF8F008D0F8D8
:10890000800030F40020DFF8E418C1F880003A005D
:10891000DFF8341E05A803F00DFD05A803F09AFB4F
:10892000020092B205A92000F7F7EDFC012084F8BF
:10893000B40203F045B900BFC42202088C3002081B
:10894000D8220208012503F03BB9DFF8001E200001
:10895000F7F770FD002802D10020002845D0200044
:10896000F7F760FD01212000F7F71BFD002802D179
:108970000020002836D02000F7F777FD0700002FF1
:1089800001D0012700E00027002F0AD0DFF85C08A3
:10899000D0F8800050F48010DFF85018C1F8800043
:1089A00009E0DFF84808D0F8800030F48010DFF8E4
:1089B0003C18C1F880003A00DFF8381E05A803F023
:1089C000B9FC05A803F046FB020092B205A92000FD
:1089D000F7F799FC012084F8B40203F0F1B800BF66
:1089E000381F0208012503F0EBB8DFF80C1E200049
:1089F000F7F720FD002802D10020002847D02000F2
:108A0000F7F710FD01212000F7F7CBFC002802D179
:108A10000020002838D02000F7F727FD0700002F9E
:108A200001D0012700E00027002F0DD0DFF8BC07A0
:108A3000D0F8800050F48020DFF8B017C1F8800033
:108A40000CE000BFE8110208DFF8A007D0F88000B2
:108A500030F48020DFF89417C1F880003A00DFF886
:108A6000401E05A803F066FC05A803F0F3FA020017
:108A700092B205A92000F7F746FC012084F8B40261
:108A800003F09EB8BC250208012503F099B8DFF871
:108A9000141E2000F7F7CEFC002802D10020002889
:108AA00035D02000F7F7BEFC01212000F7F779FC54
:108AB000002802D10020002826D02000F7F7F8FC7B
:108AC000DFF8280780ED730ADFF82007D0F8CC0123
:108AD00004F0FCFB02000B00DFF8CC1D05A803F03E
:108AE00029FC05A803F0B6FA020092B205A92000FD
:108AF000F7F709FC012084F8B40203F061B800BF65
:108B000080160208D0250208012503F059B8DFF8C5
:108B1000401E2000F7F78EFC002802D1002000281C
:108B200035D02000F7F77EFC01212000F7F739FC53
:108B3000002802D10020002826D02000F7F7B8FC3A
:108B4000DFF8A80680ED740ADFF8A006D0F8D0019F
:108B500004F0BCFB02000B00DFF8F81D05A803F0D1
:108B6000E9FB05A803F076FA020092B205A92000FD
:108B7000F7F7C9FB012084F8B40203F021B800BF65
:108B800098160208501F0208012503F019B8DFF8F3
:108B9000C81D2000F7F74EFC002802D10020002855
:108BA00033D02000F7F73EFC01212000F7F7F9FB56
:108BB000002802D10020002824D02000F7F778FCFC
:108BC000DFF8280680ED750ADFF82006D0F8D4011A
:108BD00004F07CFB02000B00DFF8241E05A803F064
:108BE000A9FB05A803F036FA020092B205A92000FD
:108BF000F7F789FB012084F8B40202F0E1BF00BF5F
:108C00004C0E0208012502F0DBBFDFF8F81D200042
:108C1000F7F710FC002802D10020002835D02000F2
:108C2000F7F700FC01212000F7F7BBFB002802D179
:108C30000020002826D02000F7F73AFCDFF8AC052A
:108C400080ED760ADFF8A405D0F8D80104F03EFBE9
:108C500002000B00DFF8B01D05A803F06BFB05A8B0
:108C600003F0F8F9020092B205A92000F7F74BFBD8
:108C7000012084F8B40202F0A3BF00BFF42B020865
:108C800098210208012502F09BBFDFF8241E200076
:108C9000F7F7D0FB002802D10020002833D02000B5
:108CA000F7F7C0FB01212000F7F77BFB002802D17A
:108CB0000020002824D02000F7F7FAFBDFF82C056D
:108CC00080ED770ADFF82405D0F8DC0104F0FEFA25
:108CD00002000B00DFF8DC1D05A803F02BFB05A844
:108CE00003F0B8F9020092B205A92000F7F70BFBD8
:108CF000012084F8B40202F063BF00BF042C020814
:108D0000012502F05DBFDFF8B01D2000F7F792FBF0
:108D1000002802D10020002835D02000F7F782FB80
:108D200001212000F7F73DFB002802D10020002898
:108D300026D02000F7F7BCFBDFF8B00480ED780AFE
:108D4000DFF8A804D0F8E00104F0C0FA02000B003C
:108D5000DFF80C1E05A803F0EDFA05A803F07AF978
:108D6000020092B205A92000F7F7CDFA012084F89D
:108D7000B40202F025BF00BFB0160208142C02088E
:108D8000012502F01DBFDFF8DC1D2000F7F752FBC4
:108D9000002802D10020002835D02000F7F742FB40
:108DA00001212000F7F7FDFA002802D10020002859
:108DB00026D02000F7F77CFBDFF8300480ED790A3D
:108DC000DFF82804D0F8E40104F080FA02000B0078
:108DD000DFF8381E05A803F0ADFA05A803F03AF94C
:108DE000020092B205A92000F7F78DFA012084F85D
:108DF000B40202F0E5BE00BF5C210208242C020888
:108E0000012502F0DDBEDFF8081E2000F7F712FB97
:108E1000002802D1002000284AD02000F7F702FBEA
:108E200001212000F7F7BDFA002802D10020002818
:108E30003BD02000F7F719FB07002000F7F7F2FA04
:108E400001212000F7F7ADFA002802D10020002808
:108E500028D02000F7F709FB50EA0740DFF88C1311
:108E6000C1F80804DFF88403D0F8080483B2DF48AF
:108E7000D0F80804020CDFF8401E05A803F05AFAE7
:108E800005A803F0E7F8020092B205A92000F7F761
:108E90003AFA012084F8B40202F092BE702102086E
:108EA000E4250208012502F08BBE012502F088BEF0
:108EB000DFF8081E2000F7F7BDFA002802D10020D5
:108EC000002849D02000F7F7ADFA01212000F7F77C
:108ED00068FA002802D1002000283AD02000F7F7D5
:108EE000C4FA07002000F7F79DFA01212000F7F7E8
:108EF00058FA002802D10020002827D02000F7F7D8
:108F0000B4FA50EA0740B949C1F80C04B748D0F8A0
:108F10000C0483B2B548D0F80C04020CDFF8401EF4
:108F200005A803F007FA05A803F094F8020092B22E
:108F300005A92000F7F7E7F9012084F8B40202F050
:108F40003FBE00BFC8160208F8250208012502F03E
:108F500037BE012502F034BEDFF8081E2000F7F707
:108F600069FA002802D10020002849D02000F7F734
:108F700059FA01212000F7F714FA002802D1002045
:108F800000283AD02000F7F770FA07002000F7F722
:108F900049FA01212000F7F704FA002802D1002045
:108FA000002827D02000F7F760FA50EA07408F49E1
:108FB000C1F838048D48D0F8380483B28B48D0F813
:108FC0003804020CDFF8401E05A803F0B3F905A829
:108FD00003F040F8020092B205A92000F7F793F9D8
:108FE000012084F8B40202F0EBBD00BFE0160208D5
:108FF00098300208012502F0E3BD012502F0E0BD32
:10900000DFF8081E2000F7F715FA002802D100202B
:10901000002849D02000F7F705FA01212000F7F7D2
:10902000C0F9002802D1002000283AD02000F7F72C
:109030001CFA07002000F7F7F5F901212000F7F7E7
:10904000B0F9002802D10020002827D02000F7F72F
:109050000CFA50EA07406549C1F81C046348D0F88F
:109060001C0483B26148D0F81C04020CDFF8401ED7
:1090700005A803F05FF905A802F0ECFF020092B228
:1090800005A92000F7F73FF9012084F8B40202F0A7
:1090900097BD00BF642902080C260208012502F0D2
:1090A0008FBD012502F08CBDDFF8081E2000F7F708
:1090B000C1F9002802D10020002849D02000F7F78C
:1090C000B1F901212000F7F76CF9002802D1002046
:1090D00000283AD02000F7F7C8F907002000F7F77A
:1090E000A1F901212000F7F75CF9002802D1002046
:1090F000002827D02000F7F7B8F950EA07403B498D
:10910000C1F820043948D0F8200483B23748D0F899
:109110002004020CDFF8401E05A803F00BF905A897
:1091200002F098FF020092B205A92000F7F7EBF8D1
:10913000012084F8B40202F043BD00BFF816020813
:1091400020260208012502F03BBD012502F038BDB2
:10915000DFF8081E2000F7F76DF9002802D1002083
:1091600000284BD02000F7F75DF901212000F7F728
:1091700018F9002802D1002000283CD02000F7F781
:1091800074F907002000F7F74DF901212000F7F7E7
:1091900008F9002802D10020002829D02000F7F784
:1091A00064F950EA07401149C1F818040F48D0F893
:1091B000180483B20D48D0F81804020CDFF8401EE2
:1091C00005A803F0B7F805A802F044FF020092B228
:1091D00005A92000F7F797F8012084F8B40202F0FF
:1091E000EFBC00BF10170208342602081018001048
:1091F000012502F0E5BC012502F0E2BCDFF8041E07
:109200002000F7F717F9002802D1002000284BD0E2
:109210002000F7F707F901212000F7F7C2F800282E
:1092200002D1002000283CD02000F7F71EF90700EB
:109230002000F7F7F7F801212000F7F7B2F800282F
:1092400002D10020002829D02000F7F70EF950EABB
:109250000740DFF8B41DC1F82404DFF8AC0DD0F8E6
:10926000240483B2DFF8A00DD0F82404020CDFF848
:10927000401E05A803F05EF805A802F0EBFE020010
:1092800092B205A92000F7F73EF8012084F8B40255
:1092900002F096BC680E020848260208012502F07A
:1092A0008FBC012502F08CBCDFF8081E2000F7F708
:1092B000C1F8002802D1002000284BD02000F7F789
:1092C000B1F801212000F7F76CF8002802D1002046
:1092D00000283CD02000F7F7C8F807002000F7F777
:1092E000A1F801212000F7F75CF8002802D1002046
:1092F000002829D02000F7F7B8F850EA0740DFF837
:10930000081DC1F82804DFF8000DD0F8280483B246
:10931000DFF8F40CD0F82804020CDFF8401E05A892
:1093200003F008F805A802F095FE020092B205A924
:109330002000F6F7E8FF012084F8B40202F040BCF8
:1093400028170208681F0208012502F039BC012510
:1093500002F036BCDFF8081E2000F7F76BF8002893
:1093600002D1002000284BD02000F7F75BF8012144
:109370002000F7F716F8002802D1002000283CD082
:109380002000F7F772F807002000F7F74BF80121EB
:109390002000F7F706F8002802D10020002829D085
:1093A0002000F7F762F850EA0740DFF85C1CC1F8CC
:1093B0002C04DFF8540CD0F82C0483B2DFF8480CEE
:1093C000D0F82C04020CDFF8401E05A802F0B2FF12
:1093D00005A802F03FFE020092B205A92000F6F7B0
:1093E00092FF012084F8B40202F0EABB840E020866
:1093F000740D0208012502F0E3BB012502F0E0BB79
:10940000DFF8081E2000F7F715F8002802D1002029
:1094100000284BD02000F7F705F801212000F6F7CF
:10942000C0FF002802D1002000283CD02000F7F720
:109430001CF807002000F6F7F5FF01212000F6F7E1
:10944000B0FF002802D10020002829D02000F7F723
:109450000CF850EA0740DFF8B01BC1F83004DFF821
:10946000A80BD0F8300483B2DFF89C0BD0F830049E
:10947000020CDFF8401E05A802F05CFF05A802F010
:10948000E9FD020092B205A92000F6F73CFF012099
:1094900084F8B40202F094BB500602085C2602086D
:1094A000012502F08DBB012502F08ABBDFF8081E02
:1094B0002000F6F7BFFF002802D1002000284BD083
:1094C0002000F6F7AFFF01212000F6F76AFF002821
:1094D00002D1002000283CD02000F6F7C6FF07008C
:1094E0002000F6F79FFF01212000F6F75AFF002821
:1094F00002D10020002829D02000F6F7B6FF50EA5C
:109500000740DFF8041BC1F83404DFF8FC0AD0F888
:10951000340483B2DFF8F00AD0F83404020CDFF828
:10952000401E05A802F006FF05A802F093FD020008
:1095300092B205A92000F6F7E6FE012084F8B402F5
:1095400002F03EBBA00E020870260208012502F0C0
:1095500037BB012502F034BBDFF8081E2000F6F708
:1095600069FF002802D1002000284BD02000F6F728
:1095700059FF01212000F6F714FF002802D1002036
:1095800000283CD02000F6F770FF07002000F6F717
:1095900049FF01212000F6F704FF002802D1002036
:1095A000002829D02000F6F760FF50EA0740DFF8D6
:1095B000581AC1F83C04DFF8500AD0F83C0483B2D2
:1095C000DFF8440AD0F83C04020CDFF8401E05A87E
:1095D00002F0B0FE05A802F03DFD020092B205A91E
:1095E0002000F6F790FE012084F8B40202F0E8BAF9
:1095F00040170208342C0208012502F0E1BA0125C7
:1096000002F0DEBADFF8081E2000F6F713FF00288C
:1096100002D1002000284BD02000F6F703FF0121E3
:109620002000F6F7BEFE002802D1002000283CD022
:109630002000F6F71AFF07002000F6F7F3FE0121DD
:109640002000F6F7AEFE002802D10020002829D025
:109650002000F6F70AFF50EA0740DFF8AC19C1F81E
:109660001004DFF8A409D0F8100483B2DFF89809D9
:10967000D0F81004020CDFF8401E05A802F05AFED4
:1096800005A802F0E7FC020092B205A92000F6F757
:109690003AFE012084F8B40202F092BA5817020888
:1096A00084260208012502F08BBA012502F088BA4F
:1096B000DFF8081E2000F6F7BDFE002802D10020CA
:1096C00000284BD02000F6F7ADFE01212000F6F770
:1096D00068FE002802D1002000283CD02000F6F7C8
:1096E000C4FE07002000F6F79DFE01212000F6F7DA
:1096F00058FE002802D10020002829D02000F6F7CB
:10970000B4FE50EA0740DFF80019C1F81404DFF88E
:10971000F808D0F8140483B2DFF8EC08D0F8140489
:10972000020CDFF8401E05A802F004FE05A802F0B6
:1097300091FC020092B205A92000F6F7E4FD012099
:1097400084F8B40202F03CBA70170208442C0208F4
:10975000012502F035BA012502F032BADFF8081E01
:109760002000F6F767FE002802D1002000284BD029
:109770002000F6F757FE01212000F6F712FE002820
:1097800002D1002000283CD02000F6F76EFE070032
:109790002000F6F747FE01212000F6F702FE002820
:1097A00002D10020002829D02000F6F75EFE50EA02
:1097B0000740DFF85418C1F84004DFF84C08D0F82F
:1097C000400483B2DFF84008D0F84004020CDFF810
:1097D000401E05A802F0AEFD05A802F03BFC020009
:1097E00092B205A92000F6F78EFD012084F8B4029C
:1097F00002F0E6B988170208542C0208012502F08D
:10980000DFB9012502F0DCB9DFF8081E2000F6F709
:1098100011FE002802D1002000284DD02000F6F7CC
:1098200001FE01212000F6F7BCFD002802D1002036
:1098300000283ED02000F6F718FE07002000F6F7BB
:10984000F1FD01212000F6F7ACFD002802D1002037
:1098500000282BD02000F6F708FE50EA0740DFF87A
:10986000A817C1F84404DFF8A007D0F8440483B275
:10987000DFF89407D0F84404020CDFF8401E05A876
:1098800002F058FD05A802F0E5FB020092B205A91E
:109890002000F6F738FD012084F8B40202F090B9F8
:1098A0008421020898260208A4140208012502F067
:1098B00087B9012502F084B9DFF8041E2000F6F70D
:1098C000B9FD002802D1002000284DD02000F6F775
:1098D000A9FD01212000F6F764FD002802D1002037
:1098E00000283ED02000F6F7C0FD07002000F6F764
:1098F00099FD01212000F6F754FD002802D1002037
:1099000000282BD02000F6F7B0FD50EA0740DFF822
:10991000F816C1F84804DFF8F006D0F8480483B21E
:10992000DFF8E406D0F84804020CDFF83C1E05A876
:1099300002F000FD05A802F08DFB020092B205A91D
:109940002000F6F7E0FC012084F8B40202F038B9F8
:10995000801F0208C0140208AC260208012502F08C
:109960002FB9012502F02CB9DFF8001E2000F6F710
:1099700061FD002802D1002000284DD02000F6F71C
:1099800051FD01212000F6F70CFD002802D1002036
:1099900000283ED02000F6F768FD07002000F6F70B
:1099A00041FD01212000F6F7FCFC002802D1002037
:1099B00000282BD02000F6F758FD50EA0740DFF8CA
:1099C0004816C1F84C04DFF84006D0F84C0483B2C6
:1099D000DFF83406D0F84C04020CDFF8381E05A876
:1099E00002F0A8FC05A802F035FB020092B205A91E
:1099F0002000F6F788FC012084F8B40202F0E0B8F9
:109A0000DC140208981F0208940D0208012502F0D8
:109A1000D7B8012502F0D4B8DFF8FC1D2000F6F716
:109A200009FD002802D1002000284DD02000F6F7C3
:109A3000F9FC01212000F6F7B4FC002802D1002037
:109A400000283ED02000F6F710FD07002000F6F7B2
:109A5000E9FC01212000F6F7A4FC002802D1002037
:109A600000282BD02000F6F700FD50EA0740DFF871
:109A70009815C1F85004DFF89005D0F8500483B26F
:109A8000DFF88405D0F85004020CDFF8341E05A876
:109A900002F050FC05A802F0DDFA020092B205A91E
:109AA0002000F6F730FC012084F8B40202F088B8F8
:109AB000B01F0208B40D0208C81F0208012502F0F9
:109AC0007FB8012502F07CB8DFF8F81D2000F6F71A
:109AD000B1FC002802D1002000284BD02000F6F76E
:109AE000A1FC01212000F6F75CFC002802D1002037
:109AF00000283CD02000F6F7B8FC07002000F6F75D
:109B000091FC01212000F6F74CFC002802D1002036
:109B1000002829D02000F6F7A8FC50EA0740DFF81B
:109B2000E814C1F85404DFF8E004D0F8540483B218
:109B3000DFF8D404D0F85404020CDFF8301E05A876
:109B400002F0F8FB05A802F085FA020092B205A91E
:109B50002000F6F7D8FB012084F8B40202F030B8F8
:109B6000F8140208E01F0208012502F029B80125B7
:109B700002F026B8DFF8F81D2000F6F75BFC00289D
:109B800002D1002000284BD02000F6F74BFC012129
:109B90002000F6F706FC002802D1002000283CD067
:109BA0002000F6F762FC07002000F6F73BFC0121DD
:109BB0002000F6F7F6FB002802D10020002829D06B
:109BC0002000F6F752FC50EA0740DFF83C14C1F8D9
:109BD0005804DFF83404D0F8580483B2DFF82804BE
:109BE000D0F85804020CDFF8301E05A802F0A2FBE2
:109BF00005A802F02FFA020092B205A92000F6F79C
:109C000082FB012084F8B40201F0DABFD40D02080F
:109C100084320208012501F0D3BF012501F0D0BF35
:109C2000DFF8F81D2000F6F705FC002802D100201F
:109C300000284BD02000F6F7F5FB01212000F6F7B5
:109C4000B0FB002802D1002000283CD02000F6F70D
:109C50000CFC07002000F6F7E5FB01212000F6F7D9
:109C6000A0FB002802D10020002829D02000F6F710
:109C7000FCFB50EA0740DFF89013C1F85C04DFF802
:109C80008803D0F85C0483B2DF48D0F85C04020C8F
:109C9000DFF8301E05A802F04DFB05A802F0DAF946
:109CA000020092B205A92000F6F72DFB012084F8EE
:109CB000B40201F085BF00BF74290208A430020875
:109CC000012501F07DBF012501F07ABFDFF8F81D05
:109CD0002000F6F7AFFB002802D10020002849D071
:109CE0002000F6F79FFB01212000F6F75AFB002821
:109CF00002D1002000283AD02000F6F7B6FB07007A
:109D00002000F6F78FFB01212000F6F74AFB002820
:109D100002D10020002827D02000F6F7A6FB50EA49
:109D20000740B949C1F86004B748D0F8600483B26D
:109D3000B548D0F86004020CDFF8141E05A802F044
:109D4000F9FA05A802F086F9020092B205A92000EE
:109D5000F6F7D9FA012084F8B40201F031BF00BF50
:109D6000C0210208642C0208012501F029BF012549
:109D700001F026BFDFF8DC1D2000F6F75BFB0028B2
:109D800002D10020002849D02000F6F74BFB01212A
:109D90002000F6F706FB002802D1002000283AD068
:109DA0002000F6F762FB07002000F6F73BFB0121DD
:109DB0002000F6F7F6FA002802D10020002827D06C
:109DC0002000F6F752FB50EA07408F49C1F86404BF
:109DD0008D48D0F8640483B28B48D0F86404020C38
:109DE000DFF8F41D05A802F0A5FA05A802F032F983
:109DF000020092B205A92000F6F785FA012084F846
:109E0000B40201F0DDBE00BFA0170208B0300208A6
:109E1000012501F0D5BE012501F0D2BEDFF83C1EC0
:109E20002000F6F707FB002802D10020002849D0C7
:109E30002000F6F7F7FA01212000F6F7B2FA002821
:109E400002D1002000283AD02000F6F70EFB0700D0
:109E50002000F6F7E7FA01212000F6F7A2FA002821
:109E600002D10020002827D02000F6F7FEFA50EAA1
:109E700007406549C1F868046348D0F8680483B2B4
:109E80006148D0F86804020CDFF8481E05A802F00B
:109E900051FA05A802F0DEF8020092B205A92000EE
:109EA000F6F731FA012084F8B40201F089BE00BF50
:109EB000D4210208BC300208012501F081BE012531
:109EC00001F07EBEDFF8101E2000F6F7B3FA00287E
:109ED00002D10020002849D02000F6F7A3FA012182
:109EE0002000F6F75EFA002802D1002000283AD0C0
:109EF0002000F6F7BAFA07002000F6F793FA0121DE
:109F00002000F6F74EFA002802D10020002827D0C2
:109F10002000F6F7AAFA50EA07403B49C1F86C0462
:109F20003948D0F86C0483B23748D0F86C04020C7E
:109F3000DFF8281E05A802F0FDF905A802F08AF84E
:109F4000020092B205A92000F6F7DDF9012084F89D
:109F5000B40201F035BE00BFE8210208742C0208EB
:109F6000012501F02DBE012501F02ABEDFF8F01D0C
:109F70002000F6F75FFA002802D1002000284BD01D
:109F80002000F6F74FFA01212000F6F70AFA002820
:109F900002D1002000283CD02000F6F766FA070026
:109FA0002000F6F73FFA01212000F6F7FAF9002821
:109FB00002D10020002829D02000F6F756FA50EAF6
:109FC00007401149C1F870040F48D0F8700483B2FB
:109FD0000D48D0F87004020CDFF8081E05A802F046
:109FE000A9F905A802F036F8020092B205A92000EE
:109FF000F6F789F9012084F8B40201F0E1BD00BF51
:10A00000B8170208C026020810180010012501F038
:10A01000D7BD012501F0D4BDDFF84C1E2000F6F7B6
:10A0200009FA002802D1002000284BD02000F6F7C2
:10A03000F9F901212000F6F7B4F9002802D1002037
:10A0400000283CD02000F6F710FA07002000F6F7B1
:10A05000E9F901212000F6F7A4F9002802D1002037
:10A06000002829D02000F6F700FA50EA0740DFF870
:10A07000FC1DC1F87404DFF8F40DD0F8740483B249
:10A08000DFF8E80DD0F87404020CDFF85C1E05A8B8
:10A0900002F050F905A801F0DDFF020092B205A917
:10A0A0002000F6F730F9012084F8B40201F088BDF1
:10A0B000BC0E0208D4260208012501F081BD01254D
:10A0C00001F07EBDDFF8241E2000F6F7B3F900286A
:10A0D00002D1002000284BD02000F6F7A3F901217F
:10A0E0002000F6F75EF9002802D1002000283CD0BD
:10A0F0002000F6F7BAF907002000F6F793F90121DE
:10A100002000F6F74EF9002802D10020002829D0BF
:10A110002000F6F7AAF950EA0740DFF8501DC1F811
:10A120007804DFF8480DD0F8780483B2DFF83C0DEE
:10A13000D0F87804020CDFF8301E05A802F0FAF817
:10A1400005A801F087FF020092B205A92000F6F7EA
:10A15000DAF8012084F8B40201F032BDD80E02080A
:10A16000842C0208012501F02BBD012501F028BD3A
:10A17000DFF8F81D2000F6F75DF9002802D1002075
:10A1800000284BD02000F6F74DF901212000F6F70A
:10A1900008F9002802D1002000283CD02000F6F762
:10A1A00064F907002000F6F73DF901212000F6F7D9
:10A1B000F8F8002802D10020002829D02000F6F766
:10A1C00054F950EA0740DFF8A41CC1F87C04DFF81A
:10A1D0009C0CD0F87C0483B2DFF8900CD0F87C049F
:10A1E000020CDFF8041E05A802F0A4F805A801F08F
:10A1F00031FF020092B205A92000F6F784F8012091
:10A2000084F8B40201F0DCBCD0170208C8300208A0
:10A21000012501F0D5BC012501F0D2BCDFF8441EB8
:10A220002000F6F707F9002802D1002000284BD0C3
:10A230002000F6F7F7F801212000F6F7B2F8002821
:10A2400002D1002000283CD02000F6F70EF90700CC
:10A250002000F6F7E7F801212000F6F7A2F8002821
:10A2600002D10020002829D02000F6F7FEF850EA9D
:10A270000740DFF8F81BC1F88004DFF8F00BD0F8D6
:10A28000800483B2DFF8E40BD0F88004020CDFF81E
:10A29000501E05A802F04EF805A801F0DBFE0200F2
:10A2A00092B205A92000F6F72EF8012084F8B40236
:10A2B00001F086BCFC210208942C0208012501F063
:10A2C0007FBC012501F07CBCDFF8181E2000F6F7EA
:10A2D000B1F8002802D1002000284BD02000F6F76A
:10A2E000A1F801212000F6F75CF8002802D1002037
:10A2F00000283CD02000F6F7B8F807002000F6F759
:10A3000091F801212000F6F74CF8002802D1002036
:10A31000002829D02000F6F7A8F850EA0740DFF817
:10A320004C1BC1F88404DFF8440BD0F8840483B2DA
:10A33000DFF8380BD0F88404020CDFF8241E05A8DF
:10A3400001F0F8FF05A801F085FE020092B205A910
:10A350002000F5F7D8FF012084F8B40201F030BCEA
:10A36000E8170208A42C0208012501F029BC0125E8
:10A3700001F026BCDFF8641E2000F6F75BF8002829
:10A3800002D1002000284BD02000F6F74BF8012125
:10A390002000F6F706F8002802D1002000283CD063
:10A3A0002000F6F762F807002000F6F73BF80121DD
:10A3B0002000F5F7F6FF002802D10020002829D060
:10A3C0002000F6F752F850EA0740DFF8A01AC1F86B
:10A3D0008804DFF8980AD0F8880483B2DFF88C0A82
:10A3E000D0F88804020CDFF8701E05A801F0A2FF67
:10A3F00005A801F02FFE020092B205A92000F5F792
:10A4000082FF012084F8B40201F0DABB00180208D0
:10A41000B42C0208012501F0D3BB012501F0D0BB0B
:10A42000DFF8381E2000F6F705F8002802D10020DA
:10A4300000284BD02000F5F7F5FF01212000F5F7AB
:10A44000B0FF002802D1002000283CD02000F6F701
:10A450000CF807002000F5F7E5FF01212000F5F7D3
:10A46000A0FF002802D10020002829D02000F5F705
:10A47000FCFF50EA0740DFF8F419C1F88C04DFF85C
:10A48000EC09D0F88C0483B2DFF8E009D0F88C0432
:10A49000020CDFF8441E05A801F04CFF05A801F0EE
:10A4A000D9FD020092B205A92000F5F72CFF01208A
:10A4B00084F8B40201F084BB18180208C42C020806
:10A4C000012501F07DBB012501F07ABBDFF80C1EF0
:10A4D0002000F5F7AFFF002802D1002000284BD064
:10A4E0002000F5F79FFF01212000F5F75AFF002813
:10A4F00002D1002000283CD02000F5F7B6FF07006D
:10A500002000F5F78FFF01212000F5F74AFF002812
:10A5100002D10020002829D02000F5F7A6FF50EA3C
:10A520000740DFF84819C1F89004DFF84009D0F877
:10A53000900483B2DFF83409D0F89004020CDFF8FD
:10A54000181E05A801F0F6FE05A801F083FD020023
:10A5500092B205A92000F5F7D6FE012084F8B402D6
:10A5600001F02EBB30180208D42C0208012501F09E
:10A5700027BB012501F024BBDFF8541E2000F5F7AE
:10A5800059FF002802D1002000284BD02000F5F709
:10A5900049FF01212000F5F704FF002802D1002027
:10A5A00000283CD02000F5F760FF07002000F5F7F9
:10A5B00039FF01212000F5F7F4FE002802D1002028
:10A5C000002829D02000F5F750FF50EA0740DFF8B7
:10A5D0009C18C1F89404DFF89408D0F8940483B26E
:10A5E000DFF88808D0F89404020CDFF85C1E05A898
:10A5F00001F0A0FE05A801F02DFD020092B205A910
:10A600002000F5F780FE012084F8B40201F0D8BAEA
:10A6100048180208E42C0208012501F0D1BA0125EE
:10A6200001F0CEBADFF8241E2000F5F703FF002862
:10A6300002D1002000284BD02000F5F7F3FE0121C5
:10A640002000F5F7AEFE002802D1002000283CD003
:10A650002000F5F70AFF07002000F5F7E3FE0121CF
:10A660002000F5F79EFE002802D10020002829D006
:10A670002000F5F7FAFE50EA0740DFF8F017C1F8BE
:10A680009804DFF8E807D0F8980483B2DFF8DC0715
:10A69000D0F89804020CDFF8281E05A801F04AFE45
:10A6A00005A801F0D7FC020092B205A92000F5F739
:10A6B0002AFE012084F8B40201F082BA6018020870
:10A6C000F42C0208012501F07BBA012501F078BACB
:10A6D000DFF8601E2000F5F7ADFE002802D1002053
:10A6E00000284BD02000F5F79DFE01212000F5F752
:10A6F00058FE002802D1002000283CD02000F5F7A9
:10A70000B4FE07002000F5F78DFE01212000F5F7CB
:10A7100048FE002802D10020002829D02000F5F7AB
:10A72000A4FE50EA0740DFF84417C1F89C04DFF8A4
:10A730003C07D0F89C0483B2DFF83007D0F89C04C3
:10A74000020CDFF8641E05A801F0F4FD05A801F075
:10A7500081FC020092B205A92000F5F7D4FD01208A
:10A7600084F8B40201F02CBA78180208042D02080B
:10A77000012501F025BA012501F022BADFF82C1ECF
:10A780002000F5F757FE002802D1002000284BD00A
:10A790002000F5F747FE01212000F5F702FE002812
:10A7A00002D1002000283CD02000F5F75EFE070013
:10A7B0002000F5F737FE01212000F5F7F2FD002813
:10A7C00002D10020002829D02000F5F74EFE50EAE3
:10A7D0000740DFF89816C1F8A004DFF89006D0F81B
:10A7E000A00483B2DFF88406D0F8A004020CDFF8DE
:10A7F000301E05A801F09EFD05A801F02BFC02000B
:10A8000092B205A92000F5F77EFD012084F8B4027C
:10A8100001F0D6B990180208E8260208012501F0D7
:10A82000CFB9012501F0CCB9DFF8F81D2000F5F70C
:10A8300001FE002802D1002000284BD02000F5F7AF
:10A84000F1FD01212000F5F7ACFD002802D1002028
:10A8500000283CD02000F5F708FE07002000F5F79F
:10A86000E1FD01212000F5F79CFD002802D1002028
:10A87000002829D02000F5F7F8FD50EA0740DFF85E
:10A88000EC15C1F8A404DFF8E405D0F8A40483B201
:10A89000DFF8D805D0F8A404020CDFF8041E05A8E0
:10A8A00001F048FD05A801F0D5FB020092B205A910
:10A8B0002000F5F728FD012084F8B40201F080B9EA
:10A8C000F40E0208FC260208012501F079B90125E1
:10A8D00001F076B9DFF8441E2000F5F7ABFD002843
:10A8E00002D1002000284BD02000F5F79BFD01216C
:10A8F0002000F5F756FD002802D1002000283CD0AA
:10A900002000F5F7B2FD07002000F5F78BFD0121CF
:10A910002000F5F746FD002802D10020002829D0AC
:10A920002000F5F7A2FD50EA0740DFF84015C1F816
:10A93000A804DFF83805D0F8A80483B2DFF82C05A6
:10A94000D0F8A804020CDFF8441E05A801F0F2FCC0
:10A9500005A801F07FFB020092B205A92000F5F7DF
:10A96000D2FC012084F8B40201F02AB9100F0208C9
:10A9700010270208012501F023B9012501F020B9B3
:10A98000DFF80C1E2000F5F755FD002802D100204D
:10A9900000284BD02000F5F745FD01212000F5F7F8
:10A9A00000FD002802D1002000283CD02000F5F74F
:10A9B0005CFD07002000F5F735FD01212000F5F7CB
:10A9C000F0FC002802D10020002829D02000F5F753
:10A9D0004CFD50EA0740DFF89414C1F8B004DFF8EA
:10A9E0008C04D0F8B00483B2DFF88004D0F8B0044F
:10A9F000020CDFF80C1E05A801F09CFC05A801F074
:10AA000029FB020092B205A92000F5F77CFC012089
:10AA100084F8B40201F0D4B82C0F020824270208ED
:10AA2000012501F0CDB8012501F0CAB8DFF8401EBC
:10AA30002000F5F7FFFC002802D1002000284BD0B1
:10AA40002000F5F7EFFC01212000F5F7AAFC002813
:10AA500002D1002000283CD02000F5F706FD0700B9
:10AA60002000F5F7DFFC01212000F5F79AFC002813
:10AA700002D10020002829D02000F5F7F6FC50EA8A
:10AA80000740DFF8E813C1F8AC04DFF8E003D0F8C2
:10AA9000A80483B2DFF8D403D0F8AC04020CDFF8CA
:10AAA000D41D05A801F046FC05A801F0D3FA020068
:10AAB00092B205A92000F5F726FC012084F8B40223
:10AAC00001F07EB8480F020838270208012501F07E
:10AAD00077B8012501F074B8DFF80C1E2000F5F7F7
:10AAE000A9FC002802D10020002838D02000F5F76A
:10AAF00099FC01212000F5F754FC002802D1002028
:10AB0000002829D02000F5F7D3FCDFF8E00D80ED18
:10AB1000000ADFF8DC0D006806F056FED348D0F8D6
:10AB2000B80402F0D3FB02000B00DFF8301E05A8CA
:10AB300001F000FC05A801F08DFA020092B205A90F
:10AB40002000F5F7E0FB012084F8B40201F038B8EA
:10AB5000640F02084C270208012501F031B8DFF824
:10AB6000001E2000F5F766FC002802D10020002816
:10AB700037D02000F5F756FC01212000F5F711FC35
:10AB8000002802D10020002828D02000F5F790FCF2
:10AB9000DFF8D00D80ED000ADFF8540D006806F0F4
:10ABA00013FEB248D0F8BC0402F090FB02000B0088
:10ABB000DFF81C1E05A801F0BDFB05A801F04AFA4C
:10ABC000020092B205A92000F5F79DFB012084F850
:10ABD000B40200F0F5BF00BF800F0208012500F0AD
:10ABE000EFBFDFF8F01D2000F5F724FC002802D1AC
:10ABF0000020002837D02000F5F714FC01212000A8
:10AC0000F5F7CFFB002802D10020002828D0200033
:10AC1000F5F74EFCDFF8280E80ED000ADFF8D00CC7
:10AC2000006806F0D1FD9148D0F8C00402F04EFB58
:10AC300002000B00DFF80C1E05A801F07BFB05A845
:10AC400001F008FA020092B205A92000F5F75BFBBB
:10AC5000012084F8B40200F0B3BF00BF142D020835
:10AC6000012500F0ADBFDFF8E01D2000F5F7E2FBA5
:10AC7000002802D10020002833D02000F5F7D2FBB5
:10AC800001212000F5F78DFB002802D100200028CB
:10AC900024D02000F5F70CFCDFF8180E80ED000A38
:10ACA0007248D0F8C40402F011FB02000B00DFF878
:10ACB000081E05A801F03EFB05A801F0CBF9020033
:10ACC00092B205A92000F5F71EFB012084F8B4021A
:10ACD00000F076BFA818020860270208012500F0DE
:10ACE0006FBFDFF8D81D2000F5F7A4FB002802D1C4
:10ACF0000020002839D02000F5F794FB0121200026
:10AD0000F5F74FFB002802D1002000282AD02000B0
:10AD1000F5F7CEFBDFF8100E80ED000ADFF80C0E21
:10AD2000006806F011F85148D0F8D80402F0CEFAC5
:10AD300002000B00DFF8F81D05A801F0FBFA05A8DA
:10AD400001F088F9020092B205A92000F5F7DBFABC
:10AD5000012084F8B40200F033BF00BF9C0F02084A
:10AD600074270208012500F02BBFDFF8C81D200062
:10AD7000F5F760FB002802D10020002837D0200022
:10AD8000F5F750FB01212000F5F70BFB002802D15D
:10AD90000020002828D02000F5F78AFBDFF8980D66
:10ADA00080ED000ADFF8940D006806F0A3FB2F4841
:10ADB000D0F8DC0402F08AFA02000B00DFF8801DF4
:10ADC00005A801F0B7FA05A801F044F9020092B213
:10ADD00005A92000F5F797FA012084F8B40200F0E5
:10ADE000EFBE00BFB80F0208012500F0E9BEDFF892
:10ADF000001E2000F5F71EFB002802D100200028CD
:10AE000039D02000F5F70EFB01212000F5F7C9FA33
:10AE1000002802D1002000282AD02000F5F748FBA6
:10AE2000DFF8D00D80ED000ADFF8100D006806F0A5
:10AE3000EFFB0E48D0F8E00402F048FA02000B00E5
:10AE4000DFF8B41D05A801F075FA05A801F002F9B4
:10AE5000020092B205A92000F5F755FA012084F806
:10AE6000B40200F0ADBE00BF882702081018001021
:10AE7000012500F0A5BEDFF8841D2000F5F7DAFA01
:10AE8000002802D10020002835D02000F5F7CAFAAA
:10AE900001212000F5F785FA002802D100200028C2
:10AEA00026D02000F5F704FBDFF8540D80ED000AF2
:10AEB000DFF8500DD0F8EC0402F008FA02000B00A5
:10AEC000DFF8441D05A801F035FA05A801F0C2F825
:10AED000020092B205A92000F5F715FA012084F8C6
:10AEE000B40200F06DBE00BFD40F0208242D02088A
:10AEF000012500F065BEDFF8141D2000F5F79AFA71
:10AF0000002802D10020002835D02000F5F78AFA69
:10AF100001212000F5F745FA002802D10020002881
:10AF200026D02000F5F7C4FADFF8E40C80ED000A23
:10AF3000DFF8D00CD0F8F40402F0C8F902000B00DE
:10AF4000DFF8D01C05A801F0F5F905A801F082F89A
:10AF5000020092B205A92000F5F7D5F9012084F886
:10AF6000B40200F02DBE00BFC0180208342D020844
:10AF7000012500F025BEDFF8A01C2000F5F75AFAE5
:10AF8000002802D10020002833D02000F5F74AFA2B
:10AF900001212000F5F705FA002802D10020002841
:10AFA00024D02000F5F784FADFF8700C80ED000A59
:10AFB000DFF8500CD0F8040502F088F902000B000D
:10AFC000DFF85C1C05A801F0B5F905A801F042F80E
:10AFD000020092B205A92000F5F795F9012084F846
:10AFE000B40200F0EDBD00BFD8180208012500F042
:10AFF000E7BDDFF8301C2000F5F71CFA002802D16D
:10B000000020002833D02000F5F70CFA01212000A1
:10B01000F5F7C7F9002802D10020002824D020002D
:10B02000F5F746FADFF8000C80ED000ADFF8D40BE4
:10B03000D0F8F80402F04AF902000B00DFF8EC1B2C
:10B0400005A801F077F905A801F004F8020092B212
:10B0500005A92000F5F757F9012084F8B40200F0A3
:10B06000AFBD00BF442D0208012500F0A9BDDFF8E7
:10B07000C01B2000F5F7DEF9002802D100200028CF
:10B0800035D02000F5F7CEF901212000F5F789F938
:10B09000002802D10020002826D02000F5F708FA69
:10B0A000DFF8900B80ED000ADFF8580BD0F80805A8
:10B0B00002F00CF902000B00DFF87C1B05A801F080
:10B0C00039F905A800F0C6FF020092B205A92000D8
:10B0D000F5F719F9012084F8B40200F071BD00BF42
:10B0E000F01802089C270208012500F069BDDFF86E
:10B0F0004C1B2000F5F79EF9002802D10020002803
:10B1000033D02000F5F78EF901212000F5F749F939
:10B11000002802D10020002824D02000F5F7C8F92B
:10B12000DFF81C0B80ED000ADFF8D80AD0F8FC0429
:10B1300002F0CCF802000B00DFF8081B05A801F0B4
:10B14000F9F805A800F086FF020092B205A92000D8
:10B15000F5F7D9F8012084F8B40200F031BD00BF42
:10B16000F00F0208012500F02BBDDFF8DC1A2000EB
:10B17000F5F760F9002802D10020002833D0200024
:10B18000F5F750F901212000F5F70BF9002802D15D
:10B190000020002824D02000F5F78AF9DFF8AC0A57
:10B1A00080ED000ADFF85C0AD0F80C0502F08EF89A
:10B1B00002000B00DFF8981A05A801F0BBF805A8FB
:10B1C00000F048FF020092B205A92000F5F79BF8B5
:10B1D000012084F8B40200F0F3BC00BFB0270208DD
:10B1E000012500F0EDBCDFF86C1A2000F5F722F91C
:10B1F000002802D10020002835D02000F5F712F9F0
:10B2000001212000F5F7CDF8002802D10020002808
:10B2100026D02000F5F74CF9DFF83C0A80ED000A53
:10B22000DFF8E009D0F8000502F050F802000B004A
:10B23000DFF8281A05A801F07DF805A800F00AFF3C
:10B24000020092B205A92000F5F75DF8012084F80C
:10B25000B40200F0B5BC00BF0C100208542D020867
:10B26000012500F0ADBCDFF8F8192000F5F7E2F891
:10B27000002802D10020002835D02000F5F7D2F8B0
:10B2800001212000F5F78DF8002802D100200028C8
:10B2900026D02000F5F70CF9DFF8C80980ED000A88
:10B2A000DFF86009D0F8100502F010F802000B007A
:10B2B000DFF8B41905A801F03DF805A800F0CAFEB2
:10B2C000020092B205A92000F5F71DF8012084F8CC
:10B2D000B40200F075BC00BF08190208F81F02088C
:10B2E000012500F06DBCDFF8F01B2000F5F7A2F897
:10B2F000002802D10020002833D02000F5F792F872
:10B3000001212000F5F74DF8002802D10020002887
:10B3100024D02000F5F7CCF8DFF8C00B80ED000A50
:10B32000DFF8E008D0F8F00401F0D0FF02000B00D5
:10B33000DFF8AC1B05A800F0FDFF05A800F08AFEB1
:10B34000020092B205A92000F4F7DDFF012084F885
:10B35000B40200F035BC00BFB4090208012500F0BA
:10B360002FBCDFF8E01B2000F5F764F8002802D1BD
:10B370000020002831D02000F5F754F801212000EA
:10B38000F5F70FF8002802D10020002822D0200075
:10B39000F5F78EF8DFF86C0880ED070ADFF864082F
:10B3A000C06901F093FF02000B00DFF89C1B05A8A9
:10B3B00000F0C0FF05A800F04DFE020092B205A902
:10B3C0002000F4F7A0FF012084F8B40200F0F8BBDD
:10B3D000C4270208012500F0F3BBDFF8701B200032
:10B3E000F5F728F8002802D10020002832D02000EC
:10B3F000F5F718F801212000F4F7D3FF002802D157
:10B400000020002824D02000F5F752F8DFF8F407D8
:10B4100080ED080ADFF8EC07006A01F057FF020030
:10B420000B00DFF8301B05A800F084FF05A800F032
:10B4300011FE020092B205A92000F4F764FF01207A
:10B4400084F8B402BCE300BF28100208D827020821
:10B450000125B5E3DFF8001B2000F4F7EBFF00281F
:10B4600002D1002000282FD02000F4F7DBFF0121BB
:10B470002000F4F796FF002802D10020002821D0F8
:10B480002000F5F715F8DFF87C0780ED090ADFF8F2
:10B490007407406A01F01AFF02000B00DFF8C01ABF
:10B4A00005A800F047FF05A800F0D4FD020092B205
:10B4B00005A92000F4F727FF012084F8B4027FE3F8
:10B4C0004410020801257BE3DFF8981A2000F4F706
:10B4D000B1FF002802D1002000282FD02000F4F76F
:10B4E000A1FF01212000F4F75CFF002802D1002019
:10B4F000002821D02000F4F7DBFFDFF8080780EDFB
:10B500000A0ADFF80007806A01F0E0FE02000B0083
:10B51000DFF8541A05A800F00DFF05A800F09AFD09
:10B52000020092B205A92000F4F7EDFE012084F894
:10B53000B40245E3642D0208012541E3DFF82C1A2B
:10B540002000F4F777FF002802D10020002831D036
:10B550002000F4F767FF01212000F4F722FF002804
:10B5600002D10020002823D02000F4F7A1FFDFF84B
:10B57000940680ED0B0ADFF88C06C06A01F0A6FE87
:10B5800002000B00DFF8E81905A800F0D3FE05A8BB
:10B5900000F060FD020092B205A92000F4F7B3FEAE
:10B5A000012084F8B4020BE320190208EC270208FA
:10B5B000012505E3DFF8BC192000F4F73BFF002864
:10B5C00002D10020002831D02000F4F72BFF012108
:10B5D0002000F4F7E6FE002802D10020002823D046
:10B5E0002000F4F765FFDFF81C0680ED0C0ADFF899
:10B5F0001406006B01F06AFE02000B00DFF87819F8
:10B6000005A800F097FE05A800F024FD020092B204
:10B6100005A92000F4F777FE012084F8B402CFE2F8
:10B6200060100208742D02080125C9E2DFF84C19E8
:10B630002000F4F7FFFE002802D10020002833D0BC
:10B640002000F4F7EFFE01212000F4F7AAFE002805
:10B6500002D10020002825D02000F4F729FFDFF8D0
:10B66000A40580ED0D0AA248006806F0ADF8DFF8E9
:10B670009405406B01F02AFE02000B00DFF8001970
:10B6800005A800F057FE05A800F0E4FC020092B205
:10B6900005A92000F4F737FE012084F8B4028FE2F8
:10B6A0003819020801258BE2DFF8D8182000F4F7DA
:10B6B000C1FE002802D10020002833D02000F4F77A
:10B6C000B1FE01212000F4F76CFE002802D1002019
:10B6D000002825D02000F4F7EBFEDFF8280580EDE8
:10B6E0000E0A8348006806F06FF8DFF81805806BD3
:10B6F00001F0ECFD02000B00DFF88C1805A800F04B
:10B7000019FE05A800F0A6FC020092B205A92000CF
:10B71000F4F7F9FD012084F8B40251E20028020890
:10B7200001254DE2DFF864182000F4F783FE0028BD
:10B7300002D1002000282FD02000F4F773FE012151
:10B740002000F4F72EFE002802D10020002821D08E
:10B750002000F4F78AFE0700DFF8A804A0F8D074F0
:10B76000DFF8A004B0F8D024DFF8241805A800F012
:10B77000E1FD05A800F06EFC020092B205A92000D0
:10B78000F4F7C1FD012084F8B40219E27C1002082C
:10B79000842D0208012513E2DFF8F8172000F4F7E2
:10B7A00049FE002802D1002000282DD02000F4F707
:10B7B00039FE01212000F4F7F4FD002802D1002019
:10B7C00000281FD02000F4F750FE0700DFF83404F3
:10B7D000A0F8D274DFF82C04B0F8D224DFF8B81740
:10B7E00005A800F0A7FD05A800F034FC020092B205
:10B7F00005A92000F4F787FD012084F8B402DFE1F9
:10B80000501902080125DBE1DFF890172000F4F75A
:10B8100011FE002802D1002000282FD02000F4F7CC
:10B8200001FE01212000F4F7BCFD002802D1002018
:10B83000002821D02000F4F718FE0700DFF8C40329
:10B84000A0F8D474DFF8BC03B0F8D424DFF85017A4
:10B8500005A800F06FFD05A800F0FCFB020092B205
:10B8600005A92000F4F74FFD012084F8B402A7E1F8
:10B8700014150208740602080125A1E1DFF8241757
:10B880002000F4F7D7FD002802D10020002833D093
:10B890002000F4F7C7FD01212000F4F782FD002805
:10B8A00002D10020002825D02000F4F701FEDFF8A7
:10B8B000F80680ED000AD348D0F8180501F006FD1F
:10B8C00002000B00DFF8E41605A800F033FD05A820
:10B8D00000F0C0FB020092B205A92000F4F713FDAE
:10B8E000012084F8B4026BE114280208C81C00107F
:10B8F00050B40020012563E1DFF8B4162000F4F70E
:10B9000099FD002802D1002000282FD02000F4F754
:10B9100089FD01212000F4F744FD002802D1002018
:10B92000002821D02000F4F7A0FD0700B548A0F8BA
:10B930001475B448B0F81425DFF8781605A800F09F
:10B94000F9FC05A800F086FB020092B205A92000D0
:10B95000F4F7D9FC012084F8B40231E1C8120208DE
:10B9600028280208CC1C0010012529E1DFF8481620
:10B970002000F4F75FFD002802D1002000282DD020
:10B980002000F4F74FFD01212000F4F70AFD002804
:10B9900002D1002000281FD02000F4F766FD070028
:10B9A0009848A0F81C759748B0F81C25DFF80C16CD
:10B9B00005A800F0BFFC05A800F04CFB020092B205
:10B9C00005A92000F4F79FFC012084F8B402F7E0F9
:10B9D000E41202083C2802080125F1E0DFF8E01536
:10B9E0002000F4F727FD002802D1002000282FD0E6
:10B9F0002000F4F717FD01212000F4F7D2FC002805
:10BA000002D10020002821D02000F4F72EFD0700ED
:10BA10007C48A0F81E757B48B0F81E25DFF8A415F9
:10BA200005A800F087FC05A800F014FB020092B204
:10BA300005A92000F4F767FC012084F8B402BFE0F8
:10BA4000D01C0010681C0208301502080125B7E060
:10BA5000DFF874152000F4F7EDFC002802D1002077
:10BA600000282FD02000F4F7DDFC01212000F4F79E
:10BA700098FC002802D10020002821D02000F4F7F3
:10BA8000F4FC07005F48A0F820755E48B0F8202558
:10BA9000DFF8381505A800F04DFC05A800F0DAFA2B
:10BAA000020092B205A92000F4F72DFC012084F8D1
:10BAB000B40285E0D41C0010DC07020850280208FC
:10BAC00001257DE0DFF808152000F4F7B3FC00281D
:10BAD00002D10020002837D02000F4F7A3FC012178
:10BAE0002000F4F75EFC002802D10020002829D0B5
:10BAF0002000F4F7BAFC07004248A0F8227541483C
:10BB0000B0F82225DFF8CC1405A800F013FC05A836
:10BB100000F0A0FA020092B205A92000F4F7F3FBAE
:10BB2000012084F8B4024BE0E81C001060B400204F
:10BB30000013020864280208EC1C001068B40020FE
:10BB40001C13020801253BE0DFF88C142000F4F7F9
:10BB500071FC002802D1002000282ED02000F4F72C
:10BB600061FC2000F4F7FCFB002802D10020002833
:10BB700021D0B4F80601B4F8081111FA80F00021C0
:10BB80000155B4F806010219DFF8501405A800F0B9
:10BB9000D1FBB4F806010219DFF8441405A800F03F
:10BBA000C9FB05A9DFF83C04006807F0E8FA0120AA
:10BBB00084F8B40204E0012502E0012500E001253B
:10BBC000EDB2002D0DD0DFF8200400F043FA0200A2
:10BBD00092B2DFF814142000F4F795FB012084F8EA
:10BBE000B4020120F8F73ABF0020F8F737BF00BFD2
:10BBF00078280208F01C0010C81C02088C280208D3
:10BC0000FC1C001010180010381302081020020845
:10BC1000041D0010540C020828200208141D0010F6
:10BC2000B40C020840200208081D0010740C020821
:10BC300058200208181D0010D40C02084C150208E8
:10BC40000C1D0010940C0208681502081C1D001041
:10BC5000F40C020884150208101D001000080208E8
:10BC6000A0150208201D00102408020870B59AB023
:10BC700004000025B4F80401032802D000201AB003
:10BC800070BD032292A1B4F80201001900F014FA69
:10BC9000002840F01A8101212000F4F782FB0028DF
:10BCA00003D10020002800F0FE808AA12000F4F7D4
:10BCB000C1FB002802D1002000281BD000AA0DF1F2
:10BCC0000201CA48006803F0A2F8BDF80030BDF8D0
:10BCD0000220C74901A800F02DFB01A800F0BAF925
:10BCE000020092B201A92000F4F70DFB012084F8B4
:10BCF000B402D9E0BF492000F4F79CFB002803D12F
:10BD00000020002800F0CD802000F4F78BFB0121FB
:10BD10002000F4F746FB002803D10020002800F0A3
:10BD2000BE802000F4F7A1FB0600B34901A800F093
:10BD300001FB01A800F08EF9010001A800F040FA13
:10BD4000AE4901A800F0F6FA01A800F083F901005D
:10BD500001A800F035FAAA4901A800F0EBFA01A801
:10BD600000F078F9010001A800F02AFAA54901A81D
:10BD700000F0E0FA01A800F06DF9010001A800F060
:10BD80001FFAA14901A800F0D5FA01A800F062F954
:10BD9000010001A800F014FA9C4901A800F0CAFAB9
:10BDA00001A800F057F9010001A800F009FA98492C
:10BDB00001A800F0BFFA01A800F04CF9010001A8A9
:10BDC00000F0FEF9934901A800F0B4FA01A800F0D0
:10BDD00041F9010001A800F0F3F98F4901A800F032
:10BDE000A9FA01A800F036F9010001A800F0E8F96D
:10BDF0008A4901A800F09EFA01A800F02BF9010081
:10BE000001A800F0DDF9864901A800F093FA01A825
:10BE100000F020F9010001A800F0D2F9814901A841
:10BE200000F088FA01A800F015F9010001A800F05F
:10BE3000C7F97D4901A800F07DFA01A800F00AF9D0
:10BE4000010001A800F0BCF9784901A800F072FADD
:10BE500001A800F0FFF8010001A800F0B1F9744951
:10BE600001A800F067FA01A800F0F4F8010001A8A9
:10BE700000F0A6F936A101A800F05CFA01A800F0D4
:10BE8000E9F8010001A800F09BF9310089B2574898
:10BE9000006803F033F8012084F8B40204E00125BF
:10BEA00002E0012500E00125EDB2002D0BD04E4847
:10BEB00000F0D0F8020092B24B492000F4F723FAC8
:10BEC000012084F8B4020120D9E60020D7E6000062
:10BED0006C6F670064697200A0280208001D0010E2
:10BEE0005413020810B59AB00400B4F804010328F2
:10BEF00002D000201AB010BD032218A1B4F802012C
:10BF0000001900F0D9F8002819D14A4900A800F01A
:10BF100011FA00A800F09EF8020092B200A92000D9
:10BF2000F4F7F1F94448006807F0B4FE43480068AC
:10BF300005F066FE002084F8B4020120DAE7002054
:10BF4000D8E70000D4300208EC220208E0300208F2
:10BF50000D0A000000230208EC3002086466750038
:10BF600014230208F83002082823020804310208CA
:10BF70003C2302081031020850230208942D0208C5
:10BF800064230208A42D0208E01C0208B428020859
:10BF9000801C0208C8280208981C0208B42D020858
:10BFA000B01C0208BC150208281D0010B8070208C2
:10BFB000D8150208940B020870200208201202080B
:10BFC000DC280208001B020888200208B40B0208C3
:10BFD000A0200208D40B02088C3202081C3102088F
:10BFE000943202084CB40020D808020854B400204F
:10BFF000700402089C32020898040208C004020877
:10C00000A8FA010850FD0108F4020208BC00020869
:10C01000E8040208B820020828310208C42D0208EA
:10C02000D0200208F0280208042902081829020872
:10C030002C290208E4FA010870B4002074B400202E
:10C0400010B5040010000A000100200007F050FEA7
:10C05000200010BD00F10103810704D010F8011B7E
:10C0600089B18107FAD10268B2F10131914311F02F
:10C07000803F04BF50F8042FF6E710F8011B11B100
:10C0800010F8011BFBE7C01A704710B450F8041BEE
:10C0900081B102681218001D50F8043BDC0744BF50
:10C0A000A9F10104E31852F8044B43F8044B091FAB
:10C0B000F9D1EBE710BC70470300002013F0030F29
:10C0C00009D0521E22BF13F8010B11F801CBB0EBBF
:10C0D0000C00F3D07047121F22BF53F8040B51F825
:10C0E00004CB6045F7D0121D0AD200BA9CFA8CFC32
:10C0F000B0EB0C0038BF6FF0000088BF0120704724
:10C10000521E22BF13F8010B11F801CBB0EB0C004B
:10C11000F6D0521C08BF104670470A22002107F0D3
:10C12000AABE80B5002207F083FF41EC100B01BDD1
:10C130004FEAF17CBCF1E04C2CBFBCF5001F11E0D4
:10C140005FEA4C0C34BFBCF17F5F2EE05FEA9C0CD1
:10C150004FEA0C1C4FEA3C0CC10071F100414CEB62
:10C1600050707047C90241EA5051C00218BF41F0F7
:10C17000010141F000414FEA6C50C0F10900212853
:10C1800010D240EACC7CCCF1200C11FA0CF070F10A
:10C190000040CCF1200C21FA0CF00CF0004C40EBEC
:10C1A0000C0070474FEACC707047490011F5001F32
:10C1B00004D84FEACC10FF30C0057047C81770474D
:10C1C00038B50022002817D0002915D08A4239D26C
:10C1D000135C1E4C24681E4D6355521C1B4B1B6880
:10C1E0005B1C1A4C2360194B1B68B3F5006FEDD133
:10C1F000164B00241C60E9E713488079072809D111
:10C20000144807F079FF11490968114A10F07F00BE
:10C2100088540AE00C488079082806D10D4807F0B8
:10C220006BFF0A4909680A4A885408480068401C9C
:10C230000649086005480068B0F5006F02D1034860
:10C2400000210160002032BD3C00002084B40020A9
:10C2500050A50020004C00400B4909680B4A1268A9
:10C26000521A094B1B688B4206D3074B1B685B1A9B
:10C270005B008342F5D305E0034B1B68D3185B00DA
:10C280008342EED370470000240C00402C0C004089
:10C29000EFF31081016072B67047006880F3108878
:10C2A0007047002100220378002B01D100202FE0ED
:10C2B00000210278613A062A01D2017857390278C2
:10C2C000413A062A01D2017837390278303A0A2AEF
:10C2D00001D2017830394278002A02D10800C0B278
:10C2E00016E000224378613B062B01D24278573A90
:10C2F0004378413B062B01D24278373A4378303BB2
:10C300000A2B02D24078B0F1300252EA0110C0B2DA
:10C31000704750F8041B61B150F8042BD30744BF99
:10C32000A9F101039A18002342F8043B091FFAD12E
:10C33000EFE770470CB41CB5044604A801900A4608
:10C34000009401AB00A907487844183007F0D8FEE4
:10C35000009900220A7000285CBF0098001B16BCE0
:10C360005DF80CFBB70F0000002101810021017076
:10C37000002141700021817000214160DFF84414E8
:10C3800008607047704780B5DFF83C04006850F0E3
:10C390000800DFF834140860DFF83004A7210180BA
:10C3A000DFF82C04DFF82C140160DFF82C0400887F
:10C3B00050F08000DFF820140880DFF820040088A7
:10C3C00050F00100DFF814140880DFF814044FF671
:10C3D000FE710180DFF80C0401210180DFF8F80311
:10C3E000008850F00100DFF8F013088032208DF84B
:10C3F000000005208DF8010000208DF802000120CA
:10C400008DF8030000A808F0FCFC01BD0189491C5F
:10C410000181704738B5050000A8FFF739FFDFF844
:10C42000C80304682D8900A8FFF737FF4FF47A701E
:10C43000B4FBF0F04400DFF8980300684FF47A7121
:10C44000B0FBF1F040004543281932BDF8B50700B4
:10C450000C0000A8FFF71CFFDFF88C0305683E897D
:10C4600000A8FFF71AFF7868281ADFF88013B0FBDE
:10C47000F1F5F6B276004FF46160B5FBF0F03018DC
:10C4800020704FF46160B5FBF0F100FB11553C20CA
:10C49000B5FBF0F060703C20B5FBF0F100FB1155EE
:10C4A000A570F1BD80B5C848006850F08000C6494D
:10C4B0000860DFF83C0329210180DFF83803A02160
:10C4C0000160DFF83403008850F08000DFF82813A3
:10C4D0000880DFF82403008850F00400DFF8181308
:10C4E0000880DFF81403008850F00800C249088073
:10C4F0002C208DF8000001208DF8010000208DF81F
:10C50000020001208DF8030000A808F07AFC01BDAC
:10C510001CB50400B948006850F00200B749086033
:10C520000121042008F01DFD0121012008F019FD62
:10C5300003220821B24808F0D5FD4FF48070009026
:10C5400003208DF8050002208DF8040000208DF8EE
:10C55000060001208DF8070000A9A94808F066FD33
:10C5600003220621A64808F0BDFD402000900320CC
:10C570008DF8050002208DF8040000208DF80600DB
:10C5800001208DF8070000A99D4808F04FFD9D4847
:10C59000002101809C48808940009C4908609B489C
:10C5A0000068A1899A4A1268128802FB0100401EA5
:10C5B00098490860984800884FF6FE7108409649EF
:10C5C00008809648008850F40040944908809448B8
:10C5D000008850F07000924908809248008850F41A
:10C5E0008070904908809048008850F008008E497B
:10C5F00008808E48008850F001008C4908808C48E3
:10C600004FF6FE7101808B48008850F00100894987
:10C6100008808948008850F006008749088013BDCB
:10C62000794A9181784989894900784A1160774926
:10C6300009688089764A1268128802FB0010401E41
:10C640007449086070477C48008850F050007A496F
:10C6500008807047784800884FF68F710840764907
:10C66000088070471CB504000121022008F079FC05
:10C670000121012008F075FC0121042008F071FC63
:10C680005148006850F001004F49086001220F2115
:10C690006A4808F027FD4FF40040009003208DF811
:10C6A000050002208DF8040000208DF8060001200E
:10C6B0008DF8070000A9614808F0B8FC01220B21A1
:10C6C0005F4808F00FFD4FF40060009003208DF8E4
:10C6D000050002208DF8040000208DF806000120DE
:10C6E0008DF8070000A9564808F0A0FC608955495C
:10C6F0000880554801210160544800884FF6FE71BA
:10C700000840524908805248008850F001005049C2
:10C7100008805048008850F4C0404E4908804E4878
:10C72000008850F440504C4908804C480121016079
:10C730004B48008850F001004949088049484FF6AD
:10C74000FE7101804848008850F05000464908803A
:10C750004548008850F005004349088013BD1A4839
:10C76000006850F01000184908604048012101801D
:10C770003F4840F6412101603E48008850F080006B
:10C780003C4908803C48008850F001003A49088044
:10C790003A484FF6FE710180394800884FF68F7194
:10C7A0000840374908803648008850F02000344956
:10C7B000088070472F48008850F001002D490880FC
:10C7C0007047000080B4002040380240280C004030
:10C7D0002C0C004000A493D6000C0040140C004028
:10C7E000100C00400C0C0040240C004020A107005D
:10C7F000281C00402C1C0040001C00404438024013
:10C800000008024028040140101800103C040140B8
:10C810006CB400202C0401400C040140440401408D
:10C820001C040140200401400004014014040140A4
:10C8300010040140180401400804014000000240B7
:10C8400000040240280000402C0000400C00004082
:10C85000180000401C000040200000404000004044
:10C860001400004010000040080000402810004064
:10C870002C10004000100040141000401010004028
:10C880000410004040B24109DFF8042A012310F0EF
:10C890001F0013FA00F042F82100704740B241092E
:10C8A000DFF8F029012310F01F0013FA00F042F81E
:10C8B00021007047DFF8E0190860704710B50400E8
:10C8C000200000F039F8DFF8D009002101602000D5
:10C8D00010BD80B5DFF8C409006804F011F9DFF875
:10C8E000C009006804F048FBDFF8B409006804F0F0
:10C8F00029FBDFF8B009006808F04DFCDFF8A80953
:10C90000006808F0BCFD01BD10B500240021DFF86F
:10C910009009006804F04AFBDFF884090068407859
:10C92000002800D1A41C64B2002C03D064B2604281
:10C9300040B210BD0120FCE780B500F006F8DFF83A
:10C940005C09006804F0CDF901BD80B50820FFF74F
:10C9500099FF0820FFF7A2FF01BD80B5DFF83C0971
:10C960000068DFF848190968C161042008F018FE62
:10C9700001BD10B5DFF83819096800220A62C0B29B
:10C98000002810D0DFF81009006880210170DFF85E
:10C9900008090068B0F84400401CDFF8FC1809687A
:10C9A000A1F844008DE1DFF8F00800680078012864
:10C9B00032D1DFF8E8080068DFF8E0180968096993
:10C9C0008161DFF8D8080068DFF8D0180968C96904
:10C9D0000161DFF8C8080068DFF8D0180968416114
:10C9E000DFF8B8080068C068401CDFF8B0180968B4
:10C9F000C860DFF8B8080068DFF89C180968896823
:10CA0000401ADFF894180968C860DFF88C080068DD
:10CA1000DFF8981809688160DFF87C080068007802
:10CA2000022830D1DFF878080068DFF87418096848
:10CA300009694161DFF868080068DFF8641809686F
:10CA400089690161DFF858080068C068401CDFF898
:10CA500050180968C860DFF854080068DFF8381813
:10CA600009680969401ADFF8301809684861DFF879
:10CA700028080068DFF8341809680161DFF8200829
:10CA8000006804F018FDDFF8100800680078062838
:10CA900030D1DFF814080068DFF80C180968C9689D
:10CAA0000161DFF804080068DFF8FC1709684969CC
:10CAB000C160DFF8F40700688068401CDFF8E81701
:10CAC00009688860DFF8E007006808F0FFFCDFF81D
:10CAD000DC070068DFF8C0170968C96B401ADFF887
:10CAE000B81709680864DFF8B0070068DFF8BC17FA
:10CAF0000968C163DFF8A00700680078032812D135
:10CB0000DFF8A8070068DFF890170968096A401A7B
:10CB1000DFF8841709684862DFF87C070068DFF8EF
:10CB20008C1709680162DFF8700700680078042834
:10CB300030D1DFF86C070068DFF864170968496BCB
:10CB40008163DFF85C070068DFF854170968C96B78
:10CB50004163DFF84C070068006B401CDFF84017AA
:10CB600009680863DFF844070068DFF82C170968D4
:10CB70008969401ADFF820170968C861DFF81807CB
:10CB80000068DFF8281709688161DFF8140700687A
:10CB900004F092FCDFF8000700680078052840F0F8
:10CBA0008B80DFF80007006890F8E800012806D1C4
:10CBB000DFF8F0060068022180F8E8107CE0DFF87A
:10CBC000E406006890F8E800032819D1DFF8DC06D5
:10CBD0000068DFF8C4160968896A401ADFF8B816D9
:10CBE0000968C862DFF8B0060068DFF8C016096897
:10CBF0008162DFF8B0060068042180F8E8105BE08D
:10CC0000DFF8A006006890F8E800052806D1DFF8F4
:10CC100094060068062180F8E8104DE0DFF88406ED
:10CC2000006890F8E800072846D1DFF88006006821
:10CC3000DFF864160968096B401ADFF85C160968AA
:10CC40004863DFF854060068DFF86016096801637E
:10CC5000DFF858060468DFF84C06006808F04AFB65
:10CC6000DFF84006006808F077FBDFF84006006850
:10CC7000001BDFF8241609688863DFF828060068BF
:10CC8000002180F8E810DFF81C060068DFF81416B1
:10CC90000968896EC166DFF80C060068DFF80416C3
:10CCA0000968096F8166DFF8FC050068406E401C6A
:10CCB000DFF8F01509684866DFF8DC050068002138
:10CCC000017010BD80B50FE0DFF8E805008850F472
:10CCD0004070DFF8E0150880DFF8D4050068002117
:10CCE00001770020FFF745FEDFF8C4050068007FEC
:10CCF00000282ED0DFF8C005006806F0A0FFDFF89E
:10CD0000B805006806F08DFFDFF8A4050068007F15
:10CD10000028E9D0DFF89805006808F089FDDFF801
:10CD20007C05006803F017FFDFF87405006804F065
:10CD300013FADFF86C05006804F013FADFF86405F5
:10CD4000006808F03CFADFF86005006808F098FB1E
:10CD5000BAE7DFF86405006806F078FFDFF85805E9
:10CD6000006806F065FF01BD10B5040020780028BA
:10CD700008D0012822D0022821D0032820D08028E2
:10CD80001FD021E0200000F020F82078002802D1F8
:10CD9000200000F054F82078002802D1200000F094
:10CDA000C8F82078002802D1200000F048F9207847
:10CDB000002802D1200000F083F805E004E003E041
:10CDC00002E02000FFF77EFF10BD10B50400DFF881
:10CDD000CC04006803F0B2FFC0B2002802D10020EA
:10CDE000002829D0DFF8C8040068DFF8D0140162F9
:10CDF000DFF8B8040068606001202070DFF89C0450
:10CE0000006803F071FFDFF89404006840780028A0
:10CE100014D0DFF8880400684078012804D005D3D6
:10CE2000032803D001D301E000E0FFE700202070D9
:10CE30000120FFF79EFD01E00020207010BD10B51D
:10CE40000400DFF85C04006804F0A3FAC0B2002814
:10CE500002D10020002830D0DFF844040068DFF859
:10CE60004C1409688161DFF848040068DFF84C144D
:10CE70000162DFF838040068606002202070DFF88B
:10CE80002004006804F0C9FADFF814040068807810
:10CE9000002814D0DFF8080400688078012804D046
:10CEA00005D3032803D001D301E000E0FFE7002011
:10CEB00020700120FFF75DFD01E00020207010BD13
:10CEC00010B50400DFF8E4030068DFF8CC1309684C
:10CED000C96B401A4FF47A71B0FBF1F04000B0F525
:10CEE0007A7F23D9DFF8C0030068DFF8C013096830
:10CEF0004161DFF8BC030068DFF8C0130162DFF8AE
:10CF0000AC030068606006202070DFF89C030068B6
:10CF100008F0B7FADFF8900300684078002807D0DF
:10CF2000002020700120FFF724FD01E00020207088
:10CF300010BD10B50400DFF86803006804F05AFA69
:10CF40000DE0DFF87403006806F08EFEDFF8700372
:10CF5000FFF782F9DFF84803006804F04BFAC0B22B
:10CF6000FF28EED001063CD5C0B2FF2809D1DFF87A
:10CF70005003FFF771F9DFF84003006806F074FE14
:10CF8000F5E7DFF828030068216A401A41F2893189
:10CF9000884223D3C6480068DFF820130162C348E3
:10CFA0000068606003202070BD48006804F0F8F954
:10CFB000BB48006890F8250000283FD0B8480068BA
:10CFC00090F82500012802D0022801D000E0FFE7F8
:10CFD000002020700120FFF7CCFC2FE00020207003
:10CFE0002CE0C0B2012827D1AD480068AF490968DC
:10CFF000C163AF480068B1490162AC480068606035
:10D0000004202070A648006804F031FAA4480068A3
:10D0100090F82500002811D0A148006890F825005C
:10D02000012802D0022801D000E0FFE70020207094
:10D030000120FFF79EFC01E00020207010BD10B51C
:10D0400004009848006808F0C1F8C0B2002805D074
:10D050009448006890F8E800002801D1012000E021
:10D060000020C0B2002868D08E48006890F8E80020
:10D07000002833D18D480068216B401A41F2893174
:10D08000884228D38A4800688C4901628548006834
:10D09000012180F8E8108548006860600520207054
:10D0A0008048006808F098F87E48006890F83900D9
:10D0B000002800F0A8807B48006890F8390001281B
:10D0C00002D0022801D000E0FFE7002020700120FC
:10D0D000FFF74FFC97E00020207094E07148006853
:10D0E00090F8E800042840F08E8071480068734989
:10D0F00001626C480068052180F8E8106B48006800
:10D100006060052020706748006808F0ABF865484B
:10D11000006890F83900002875D06248006890F8DF
:10D120003900012802D0022801D000E0FFE70020EA
:10D1300020700120FFF71DFC65E05A48006890F858
:10D14000E800022827D15A4800685C490162554826
:10D150000068032180F8E8105448006860600520EA
:10D1600020705048006808F059F84E48006890F860
:10D170003900002847D04B48006890F83900012852
:10D1800002D0022801D000E0FFE70020207001203B
:10D19000FFF7EFFB37E04348006890F8E800062807
:10D1A0002CD140480068414909680167404800683F
:10D1B000424901623B480068072180F8E8103B487B
:10D1C00000686060052020703648006808F06CF840
:10D1D0003448006890F83900002814D031480068BD
:10D1E00090F83900012802D0022801D000E0FFE7C2
:10D1F000002020700120FFF7BCFB04E029480068F4
:10D20000002180F8E81010BD10B50400C9B2012952
:10D210001AD1DFF8B000006890ED380AB1EE400A8C
:10D22000DFF8A40080ED0D0ADFF89800006890EDAB
:10D23000390AB1EE400ADFF8900080ED0E0ADFF8FF
:10D240008400006804F0C0FADFF87C001249096825
:10D25000D1F8D410C163D4F8100100280ED094F88E
:10D26000180100280AD0DFF86000D4F8F4108166B5
:10D27000DFF85400D4F8F010C16607E0DFF848008A
:10D2800000218166DFF840000021C16610BD00006A
:10D2900080E100E080E200E05CB4002060B40020A7
:10D2A00068B4002040B4002064B40020240C004086
:10D2B00058B400200454004070B4002073C9000822
:10D2C000400D030050B40020101800105FF0FF0C58
:10D2D0001CEAD05114BF614506E0C110400721F09F
:10D2E000E04101F16051704779B900F0004100025E
:10D2F0000AD0B0FA80FC00FA0CF001F16051A1EB09
:10D300000C5101EBD0214005704741020CBF40F4A5
:10D31000E0016FF00001002070470268531C0360B9
:10D320001170704710B50400DFF804040460200099
:10D3300000F002F8200010BD10B50400002020709D
:10D3400000206070200000F01CF8200000F0C2F8FF
:10D3500010F0010084F82804200000F0E0F8C4F880
:10D360002C04002084F83004D4F82C04C0F30740C7
:10D37000262804D1102084F830040120207010BD2C
:10D38000704700B587B00121012007F0EAFD0121B7
:10D39000022007F0E6FD01214FF4804007F001FE76
:10D3A00001214FF4805007F0FCFD05220621E148E1
:10D3B00007F098FE4020009003208DF80500022021
:10D3C0008DF8040000208DF8060002208DF807007B
:10D3D00000A9D84807F02AFE05220721D54807F002
:10D3E00081FE8020009003208DF8050002208DF83A
:10D3F000040000208DF8060002208DF8070000A927
:10D40000CC4807F013FE05220321DFF8440E07F095
:10D4100069FE0820009003208DF8050002208DF899
:10D42000040000208DF8060002208DF8070000A9F6
:10D43000DFF81C0E07F0FAFD0420009003208DF8A1
:10D44000050001208DF8040000208DF80600022060
:10D450008DF8070000A9DFF8F80D07F0E7FDDFF809
:10D46000F40D042101800020ADF808004FF4827013
:10D47000ADF80A000020ADF80C000020ADF80E0059
:10D480000020ADF810004FF40070ADF8120000203D
:10D49000ADF814000020ADF816000720ADF8180014
:10D4A00002A9DFF8400E08F097FC07B000BDDFF8D6
:10D4B000380E00888007FAD5DFF8300EC9B2018037
:10D4C000DFF8240E0088C007FAD5DFF8200E0088A8
:10D4D000C0B2704710B50400DFF8140E04210180BB
:10D4E000DFF8000E008850F04000DFF8F81D0880DB
:10D4F000D7212000FFF7DBFFFF212000FFF7D7FF38
:10D50000DFF8501D04220A80DFF8D81D09884FF685
:10D51000BF721140DFF8CC2D1180C0B210BD38B5FC
:10D520000500DFF8CC0D04210180DFF8B80D00887C
:10D5300050F04000DFF8AC1D08809F212800FFF765
:10D54000B6FFFF212800FFF7B2FF04002402FF21ED
:10D550002800FFF7ACFF04432402FF212800FFF757
:10D56000A6FF04432402FF212800FFF7A0FF044385
:10D57000DFF8E00C04210180DFF8680D00884FF629
:10D58000BF710840DFF85C1D0880200032BD70B517
:10D5900004000E0015002078002853D02000FFF76B
:10D5A00099FF0006FAD500200028F7D1DFF8400DDA
:10D5B00004210180DFF82C0D008850F04000DFF8D6
:10D5C000241D0880D2212000FFF771FFB6B2B602F9
:10D5D000310CC9B22000FFF76AFF310AC9B220003E
:10D5E000FFF765FF3100C9B22000FFF760FFFF21A0
:10D5F0002000FFF75CFFFF212000FFF758FFFF210D
:10D600002000FFF754FFFF212000FFF750FF4FF4E9
:10D61000047605E0FF212000FFF749FF28706D1C0C
:10D620003000461E80B20028F4D1DFF8280C042117
:10D630000180DFF8B00C00884FF6BF710840DFF8BA
:10D64000A41C088070BDF8B504000D0016002078F9
:10D6500000286CD02000FFF73DFF0006FAD500201F
:10D660000028F7D1DFF8880C04210180DFF8740C62
:10D67000008850F04000DFF86C1C088084212000F6
:10D68000FFF715FF00212000FFF711FF0021200008
:10D69000FFF70DFF00212000FFF709FF4FF404778B
:10D6A00005E03000461C01782000FFF700FF38003D
:10D6B000471E80B20028F4D1DFF8980B04210180C6
:10D6C000DFF8200C00884FF6BF710840DFF8141C0B
:10D6D0000880DFF81C0C04210180DFF8080C0088AA
:10D6E00050F04000DFF8FC1B088083212000FFF78A
:10D6F000DEFEADB2AD02290CC9B22000FFF7D7FEA5
:10D70000290AC9B22000FFF7D2FE2900C9B22000C1
:10D71000FFF7CDFEDFF83C0B04210180DFF8C40BDE
:10D7200000884FF6BF710840DFF8B81B0880F1BDD4
:10D7300054B400200000024010B5040020780028F6
:10D7400001D1002015E001206070A21C0021200002
:10D75000FFF71DFFA01CC4F83404D4F8340400689B
:10D76000401CD4F834140860D4F834040068002154
:10D77000617010BD38B504002078002801D1002068
:10D7800032BD01206070A21C00212000FFF7FFFEC7
:10D79000A01CC4F83404D4F834040068401CD4F845
:10D7A00034140860D4F834040568D4F83404032130
:10D7B0004160D4F83404DFF83C1B89880181D4F837
:10D7C0003404DFF8301B09894181D4F83404DFF8D0
:10D7D000241B897A0173D4F83404DFF8181B898973
:10D7E000C181D4F83404DFF80C1B897B0174D4F8B0
:10D7F0003404DFF8001BC9694161D4F83404DFF850
:10D80000F41A096A8161D4F83404DFF8E81A496A25
:10D81000C161D4F83404DFF8DC1A896A0162D4F8F3
:10D820003404DFF8D01AC96A4162D4F83404DFF84E
:10D83000C41A096B8162D4F83404DFF8B81AC96BD2
:10D840008163D4F83404DFF8AC1AB1F84210818750
:10D85000D4F83404DFF89C1AB1F84410C187D4F826
:10D860003404DFF8901AB1F84610A0F84010D4F84C
:10D870003404DFF8801AB1F84810A0F84210D4F848
:10D880003404DFF8701AB1F84A10A0F84410D4F844
:10D890003404DFF8601AB1F84C10A0F84610D4F840
:10D8A0003404DFF8501AB1F84E10A0F84810D4F83C
:10D8B0003404DFF8401AB1F85010A0F84A10D4F838
:10D8C0003404DFF8301AB1F85210A0F84C10D4F834
:10D8D0003404DFF8201AB1F85410A0F84E10D4F830
:10D8E0003404DFF8101AB1F85610A0F85010D4F82C
:10D8F0003404DFF8001AB1F85810A0F85210D4F828
:10D900003404DFF8F019B1F85A10A0F85410D4F824
:10D910003404DFF8E019B1F85C10A0F85610D4F820
:10D920003404DFF8D019096E8165D4F83404DFF8C7
:10D93000C419496EC165D4F83404DFF8B819896E8A
:10D940000166D4F83404DFF8AC19C96E4166D4F826
:10D950003404DFF8A019096F8166D4F83404DFF8C5
:10D960009419D1F8C811C166D4F83404DFF88419C9
:10D97000496F0167D4F83404DFF87819896F41677B
:10D98000D4F83404DFF86C19C96F8167D4F8340413
:10D99000DFF86019D1F88010C167D4F83404DFF8DB
:10D9A0005419D1F88410C0F88010D4F83404DFF88A
:10D9B0004419D1F88810C0F88410D4F83404DFF882
:10D9C0003419D1F88C10C0F88810D4F83404DFF87A
:10D9D0002419D1F89010C0F88C10D4F83404DFF872
:10D9E0001419D1F89410C0F89010D4F83404DFF86A
:10D9F0000419D1F89810C0F89410D4F83404DFF862
:10DA0000F418D1F89C10C0F89810D4F83404DFF85A
:10DA1000E418D1F8A010C0F89C10D4F83404DFF852
:10DA2000D418D1F8A410C0F8A010D4F83404DFF84A
:10DA3000C418D1F8A810C0F8A410D4F83404DFF842
:10DA4000B418D1F8AC10C0F8A810D4F83404DFF83A
:10DA5000A418D1F8B010C0F8AC10D4F83404DFF832
:10DA60009418D1F8B410C0F8B010D4F83404DFF82A
:10DA70008418098A8185D4F83404DFF87818498A33
:10DA8000C185D4F83404DFF86C18898A0186D4F88B
:10DA90003404DFF86018C98A4186D4F83404DFF80A
:10DAA0005418098B8186D4F83404DFF84818498B60
:10DAB000C186D4F83404DFF83C18D1F8BC10C0F8A3
:10DAC000B810D4F83404DFF82C18D1F8B810C0F826
:10DAD000B410D4F83404DFF81C1891F8E01080F882
:10DAE000BC10D4F83404DFF80C18D1F8C010C0F81A
:10DAF0003811D4F83404DFF8FC17D1F8C410C0F89A
:10DB00003C11D4F83404DFF8EC17D1F8C810C0F891
:10DB10004011D4F83404DFF8DC17D1F8CC10C0F889
:10DB20004411D4F83404DFF8CC17D1F8D010C0F881
:10DB30004811D4F83404DFF8BC17D1F8D410C0F879
:10DB40004C11D4F83404DFF8AC17D1F8D810C0F871
:10DB50005011D4F83404DFF89C17D1F8DC10C0F869
:10DB60005411D4F83404DFF88C1791F8E11080F8E0
:10DB70005811D4F83404DFF87C17B1F8E210A0F89B
:10DB80005A11D4F83404DFF86C17B1F8E410A0F897
:10DB90005C11D4F83404DFF85C17D1F8E810C0F851
:10DBA0006011D4F83404DFF84C17D1F8EC10C0F849
:10DBB0006411D4F83404DFF83C17D1F8F010C0F841
:10DBC0006811D4F83404DFF82C17B1F8FA10A0F873
:10DBD0006C11D4F83404DFF81C17D1F8FC10C0F82D
:10DBE0007011D4F83404DFF80C17B1F80011A0F864
:10DBF0007411D4F83404DFF8FC16B1F80211A0F85F
:10DC00007611D4F83404DFF8EC16D1F80C11C0F812
:10DC100078117822DFF8E016D4F83404C03008F028
:10DC200007F9D4F83404DFF8CC1691F8881180F89D
:10DC30007C11D4F83404DFF8BC16D1F88C11C0F88C
:10DC40008011D4F83404DFF8AC16D1F89011C0F884
:10DC50008411D4F83404DFF89C16D1F89411C0F87C
:10DC60008811D4F83404DFF88C16D1F89811C0F874
:10DC70008C11D4F83404DFF87C16D1F89C11C0F86C
:10DC80009011D4F83404DFF86C16D1F8A011C0F864
:10DC90009411D4F83404DFF85C16D1F8A411C0F85C
:10DCA0009811D4F83404DFF84C16D1F8A811C0F854
:10DCB0009C11D4F83404DFF83C16D1F8AC11C0F84C
:10DCC000A011D4F83404DFF82C16D1F8B811C0F83C
:10DCD000A411D4F83404DFF81C1691F8891180F8E7
:10DCE000A811D4F83404DFF80C16B1F8C411A0F868
:10DCF000AA11D4F83404DFF8FC15D1F8CC11C0F81F
:10DD0000AC11D4F83404DFF8EC15D1F8D011C0F818
:10DD1000B011D4F83404DFF8DC15D1F8D411C0F810
:10DD2000B411D4F83404DFF8CC15D1F8D811C0F808
:10DD3000B811D4F83404DFF8BC15D1F8DC11C0F800
:10DD4000BC11D4F83404DFF8AC15D1F8E011C0F8F8
:10DD5000C011D4F83404DFF89C15D1F8E411C0F8F0
:10DD6000C411D4F83404DFF88C15D1F8B011C0F820
:10DD7000C811D4F83404DFF87C15D1F8B411C0F818
:10DD8000CC11D4F83404DFF86C15D1F8BC11C0F80C
:10DD9000D011D4F83404DFF85C15D1F8C011C0F804
:10DDA000D411D4F83404DFF84C15D1F8B814C0F805
:10DDB000D811D4F83404DFF83C15D1F8BC14C0F8FD
:10DDC000DC11D4F83404DFF82C15D1F8C014C0F8F5
:10DDD000E011D4F83404DFF81C15D1F8C414C0F8ED
:10DDE000E411D4F83404DFF80C1591F8C81480F865
:10DDF000E811D4F83404DFF8FC1491F8C91480F861
:10DE0000F011D4F83404DFF8EC1491F8CB1480F856
:10DE1000F111D4F83404DFF8DC1491F8CD1480F853
:10DE2000F211D4F83404DFF8D414C0F8EC11A21CB9
:10DE300000212000FFF707FC42F21070FEF70CFAF9
:10DE4000A21C02212000FFF7A2FBA01CC4F838048A
:10DE5000D4F83804DFF89C14D1F808140160D4F821
:10DE60003804DFF89014D1F80C144160D4F8380469
:10DE7000DFF88014D1F810148160D4F83804DFF88A
:10DE80007414D1F81414C160D4F83804DFF86414A1
:10DE9000D1F818140161D4F83804DFF85814D1F817
:10DEA0001C144161D4F83804DFF84814D1F8201468
:10DEB0008161D4F83804DFF83C14D1F82414C1612E
:10DEC000D4F83804DFF82C14D1F828140162D4F8FF
:10DED0003804DFF82014D1F82C144162D4F8380447
:10DEE000DFF81014D1F830148162D4F83804DFF868
:10DEF0000414D1F83414C162D4F83804DFF8F413F0
:10DF0000D1F838140163D4F83804DFF8E813D1F8F5
:10DF10003C144163D4F83804DFF8D813D1F8401426
:10DF20008163D4F83804DFF8CC13D1F84414C1630A
:10DF3000D4F83804DFF8BC13D1F848140164D4F8DD
:10DF40003804DFF8B013D1F84C144164D4F8380425
:10DF5000DFF8A013D1F850148164D4F83804DFF846
:10DF60009413D1F85414C164D4F83804DFF884133E
:10DF7000D1F858140165D4F83804DE49D1F85C149E
:10DF8000C0F8A410D4F83804DA49D1F86014416517
:10DF9000D4F83804D749D1F864148165D4F838042A
:10DFA000D449D1F86814C165D4F83804D149D1F8FE
:10DFB0006C140166D4F83804CE49D1F87014416667
:10DFC000D4F83804CB49D1F874148166D4F83804F5
:10DFD000C849D1F87814C166D4F83804C549D1F8D5
:10DFE0007C140167D4F83804C249D1F88014416721
:10DFF000D4F83804BF49D1F884148167D4F83804C0
:10E00000BC49D1F88814C167D4F83804B949D1F8AB
:10E010008C14C0F88010D4F83804B649D1F89014A4
:10E02000C0F88410D4F83804B249D1F89414C0F878
:10E030008810D4F83804AF49D1F89814C0F88C107F
:10E04000D4F83804AB49D1F89C14C0F89010D4F837
:10E050003804A849D1F8A014C0F89410D4F83804B2
:10E06000A449D1F8A414C0F89810D4F83804A149F0
:10E07000D1F8A814C0F89C10D4F838049D49D1F800
:10E08000AC14C0F8A010D4F838049A49D1F8B014F0
:10E09000C0F8F010D4F838049649B1F8CE14A0F8BE
:10E0A000A810D4F838049349B1F8D014A0F8AA10F5
:10E0B000D4F838048F49B1F8D214A0F8AC10D4F8D1
:10E0C00038048C49B1F8D414A0F8AE10D4F8380450
:10E0D0008849D1F8D814C0F8B010D4F8380485496C
:10E0E000D1F8DC14C0F8B410D4F838048149D1F860
:10E0F000E014C0F8B810D4F838047E49D1F8EC1414
:10E10000C0F8BC10D4F838047A49D1F8F414C0F837
:10E11000C810D4F838047749D1F8F814C0F8CC10F6
:10E12000D4F838047349D1F8FC14C0F8D010D4F8EE
:10E1300038047049D1F80015C0F8C010D4F838047C
:10E140006C49D1F80415C0F8F410D4F838046949C2
:10E15000D1F80815C0F8F810D4F838046549D1F89A
:10E160000C15C0F8FC10D4F838046249D1F8101529
:10E17000C0F80011D4F838045E49D1F8F014C0F8A2
:10E18000C410D4F838045B49B1F8B414A0F8D41022
:10E19000D4F838045749496BC0F8D810D4F838047B
:10E1A0005449896BC0F8DC10D4F838045149B1F8EF
:10E1B0001415A0F8E010D4F838044E49D1F8181519
:10E1C000C0F8E410D4F838044A49B1F81C15A0F896
:10E1D000E810D4F838044749B1F81E15A0F8EA1041
:10E1E000D4F838044349B1F82015A0F8EC10D4F85D
:10E1F00038044049B1F82215A0F8EE10D4F83804DC
:10E200003C49B1F80411A0F80411D4F83804394994
:10E21000B1F80611A0F80611D4F838043549B1F860
:10E220000811A0F80811D4F838043249B1F82415BF
:10E23000A0F80A11A21C02212000FFF704FA42F202
:10E240001070FEF709F8002060702800FFF798BAF8
:10E25000000402401804024010B504002078002891
:10E2600001D1002010BD01206070A21C01212000FE
:10E27000FFF78DF9A01CC4F83C04C022DFF8681B2E
:10E28000D4F83C0407F0D4FDC022DFF8601BD4F8BA
:10E290003C04C03007F0CCFDA21C01212000FFF798
:10E2A000D2F942F21070FDF7D7FFA21C0321200023
:10E2B000FFF76DF9A01CC4F84004A022DFF8301B62
:10E2C000D4F8400407F0B4FDA21C03212000FFF79E
:10E2D000BAF942F21070FDF7BFFF00206070012014
:10E2E000C0E7000000300140083001400C30014020
:10E2F0001A0402401018001020190010AA55AA553F
:10E3000010B50400A21C00212000FFF740F9A01C5A
:10E31000C4F834042078002802D1002000F062BD47
:10E32000D4F83404006810F1010F02D1002000F08D
:10E3300059BDD4F834044068032802D0002000F00E
:10E3400051BDD4F834040089DFF8A81A8880D4F8C5
:10E3500034044089DFF89C1A0881D4F83404007B27
:10E36000DFF8901A8872D4F83404C089DFF8841A70
:10E370008881D4F83404007CDFF8781A8873D4F8E4
:10E3800034044069DFF86C1AC861D4F83404806939
:10E39000DFF8601A0862D4F83404C069DFF8541A50
:10E3A0004862D4F83404006ADFF8481A8862D4F866
:10E3B0003404406ADFF83C1AC862D4F83404806A36
:10E3C000DFF8301A0863D4F83404806BDFF8241ABD
:10E3D000C863D4F83404808FDFF8181AA1F842001B
:10E3E000D4F83404C08FDFF80C1AA1F84400D4F834
:10E3F0003404B0F84000DFF8FC19A1F84600D4F866
:10E400003404B0F84200DFF8EC19A1F84800D4F861
:10E410003404B0F84400DFF8DC19A1F84A00D4F85D
:10E420003404B0F84600DFF8CC19A1F84C00D4F859
:10E430003404B0F84800DFF8BC19A1F84E00D4F855
:10E440003404B0F84A00DFF8AC19A1F85000D4F851
:10E450003404B0F84C00DFF89C19A1F85200D4F84D
:10E460003404B0F84E00DFF88C19A1F85400D4F849
:10E470003404B0F85000DFF87C19A1F85600D4F845
:10E480003404B0F85200DFF86C19A1F85800D4F841
:10E490003404B0F85400DFF85C19A1F85A00D4F83D
:10E4A0003404B0F85600DFF84C19A1F85C00D4F839
:10E4B0003404806DDFF83C190866D4F83404C06D6C
:10E4C000DFF830194866D4F83404006EDFF82419F8
:10E4D0008866D4F83404406EDFF81819C866D4F89A
:10E4E0003404806EDFF80C190867D4F83404C06E69
:10E4F000DFF80019C1F8C801D4F83404006FDFF860
:10E50000F4184867D4F83404406FDFF8E8188867D7
:10E51000D4F83404806FDFF8DC18C867D4F834040A
:10E52000C06FDFF8D018C1F88000D4F83404D0F8F8
:10E530008000DFF8C018C1F88400D4F83404D0F8A3
:10E540008400DFF8B018C1F88800D4F83404D0F89B
:10E550008800DFF8A018C1F88C00D4F83404D0F893
:10E560008C00DFF89018C1F89000D4F83404D0F88B
:10E570009000DFF88018C1F89400D4F83404D0F883
:10E580009400DFF87018C1F89800D4F83404D0F87B
:10E590009800DFF86018C1F89C00D4F83404D0F873
:10E5A0009C00DFF85018C1F8A000D4F83404D0F86B
:10E5B000A000DFF84018C1F8A400D4F83404D0F863
:10E5C000A400DFF83018C1F8A800D4F83404D0F85B
:10E5D000A800DFF82018C1F8AC00D4F83404D0F853
:10E5E000AC00DFF81018C1F8B000D4F83404D0F84B
:10E5F000B000DFF80018C1F8B400D4F83404808DFE
:10E60000DFF8F0170882D4F83404C08DDFF8E4177F
:10E610004882D4F83404008EDFF8D8178882D4F802
:10E620003404408EDFF8CC17C882D4F83404808ECE
:10E63000DFF8C0170883D4F83404C08EDFF8B417AD
:10E640004883D4F83404D0F8B800DFF8A817C1F82C
:10E65000BC00D4F83404D0F8B400DFF89817C1F83F
:10E66000B800D4F8340490F8BC00DFF8881781F8BB
:10E67000E000D4F83404D0F83801DFF87817C1F896
:10E68000C000D4F83404D0F83C01DFF86817C1F8B2
:10E69000C400D4F83404D0F84001DFF85817C1F8AA
:10E6A000C8007822D4F8340410F1C001DFF848071C
:10E6B00007F0BEFBD4F83404D0F84401DFF8341777
:10E6C000C1F8CC00D4F83404D0F84801DFF824179E
:10E6D000C1F8D000D4F83404D0F84C01DFF8141796
:10E6E000C1F8D400D4F83404D0F85001DFF804178E
:10E6F000C1F8D800D4F83404D0F85401DFF8F41687
:10E70000C1F8DC00D4F8340490F85801DFF8E416BE
:10E7100081F8E100D4F83404B0F85A01DFF8D416D7
:10E72000A1F8E200D4F83404B0F85C01DFF8C416B4
:10E73000A1F8E400D4F83404D0F86001DFF8B4168E
:10E74000C1F8E800D4F83404D0F86401DFF8A41666
:10E75000C1F8EC00D4F83404D0F86801DFF894165E
:10E76000C1F8F000D4F83404B0F86C01DFF8841676
:10E77000A1F8FA00D4F83404D0F87001DFF8741668
:10E78000C1F8FC00D4F83404B0F87401DFF8641662
:10E79000A1F80001D4F83404B0F87601DFF854167B
:10E7A000A1F80201D4F83404D0F87801DFF8441657
:10E7B000C1F80C01D4F8340490F87C01DFF8341669
:10E7C00081F88801D4F83404D0F88001DFF82416E9
:10E7D000C1F88C01D4F83404D0F88401DFF81416A1
:10E7E000C1F89001D4F83404D0F88801DFF8041699
:10E7F000C1F89401D4F83404D0F88C01DFF8F41592
:10E80000C1F89801D4F83404D0F89001DFF8E41589
:10E81000C1F89C01D4F83404D0F89401DFF8D41581
:10E82000C1F8A001D4F83404D0F89801DFF8C41579
:10E83000C1F8A401D4F83404D0F89C01DFF8B41571
:10E84000C1F8A801D4F83404D0F8A001DFF8A41569
:10E85000C1F8AC01D4F83404D0F8A401DFF8941561
:10E86000C1F8B801D4F8340490F8A801DFF8841591
:10E8700081F88901D4F83404B0F8AA01DFF87415DE
:10E88000A1F8C401D4F83404D0F8AC01DFF8641561
:10E89000C1F8CC01D4F83404D0F8B001DFF8541535
:10E8A000C1F8D001D4F83404D0F8B401DFF844152D
:10E8B000C1F8D401D4F83404D0F8B801DFF8341525
:10E8C000C1F8D801D4F83404D0F8BC01DFF824151D
:10E8D000C1F8DC01D4F83404D0F8C001DFF8141515
:10E8E000C1F8E001D4F83404D0F8C401DFF804150D
:10E8F000C1F8E401D4F83404D0F8C801DFF8F41406
:10E90000C1F8B001D4F83404D0F8CC01DFF8E41435
:10E91000C1F8B401D4F83404D0F8D001DFF8D4142D
:10E92000C1F8BC01D4F83404D0F8D401DFF8C41421
:10E93000C1F8C001D4F83404D0F8D801DFF8B41419
:10E94000C1F8B804D4F83404D0F8DC01DFF8A4141A
:10E95000C1F8BC04D4F83404D0F8E001DFF8941412
:10E96000C1F8C004D4F83404D0F8E401DFF884140A
:10E97000C1F8C404D4F8340490F8E801DFF8741442
:10E9800081F8C804D4F8340490F8F001DFF8641476
:10E9900081F8C904D4F8340490F8F101DFF8541474
:10E9A00081F8CB04D4F8340490F8F201DFF8441471
:10E9B00081F8CD04A21C02212000FEF7E8FDA01C76
:10E9C000C4F83804D4F838040068DFF82814C1F813
:10E9D0000804D4F838044068DFF81814C1F80C04AF
:10E9E000D4F838048068DFF80C14C1F81004D4F8A7
:10E9F0003804C068DFF8FC13C1F81404D4F83804F4
:10EA00000069DFF8F013C1F81804D4F8380440693D
:10EA1000DFF8E013C1F81C04D4F838048069DFF88B
:10EA2000D413C1F82004D4F83804C069DFF8C41343
:10EA3000C1F82404D4F83804006ADFF8B813C1F828
:10EA40002804D4F83804406ADFF8A813C1F82C046D
:10EA5000D4F83804806ADFF89C13C1F83004D4F885
:10EA60003804C06ADFF88C13C1F83404D4F83804D1
:10EA7000006BDFF88013C1F83804D4F83804406B19
:10EA8000DFF87013C1F83C04D4F83804806BD9491E
:10EA9000C1F84004D4F83804C06BD649C1F8440426
:10EAA000D4F83804006CD349C1F84804D4F83804C9
:10EAB000406CD049C1F84C04D4F83804806CCD497E
:10EAC000C1F85004D4F83804C06CCA49C1F85404E1
:10EAD000D4F83804006DC749C1F85804D4F8380494
:10EAE000D0F8A400C349C1F85C04D4F83804406DE0
:10EAF000C049C1F86004D4F83804806DBD49C1F83C
:10EB00006404D4F83804C06DBA49C1F86804D4F874
:10EB10003804006EB749C1F86C04D4F83804406E6C
:10EB2000B449C1F87004D4F83804806EB149C1F812
:10EB30007404D4F83804C06EAE49C1F87804D4F82F
:10EB40003804006FAB49C1F87C04D4F83804406F36
:10EB5000A849C1F88004D4F83804806FA549C1F8E9
:10EB60008404D4F83804C06FA249C1F88804D4F8EA
:10EB70003804D0F880009F49C1F88C04D4F83804D8
:10EB8000D0F884009B49C1F89004D4F83804D0F838
:10EB900088009849C1F89404D4F83804D0F88C005F
:10EBA0009449C1F89804D4F83804D0F890009149F9
:10EBB000C1F89C04D4F83804D0F894008D49C1F809
:10EBC000A004D4F83804D0F898008A49C1F8A40405
:10EBD000D4F83804D0F89C008649C1F8A804D4F8C9
:10EBE0003804D0F8A0008349C1F8AC04D4F8380444
:10EBF000D0F8F0007F49C1F8B004D4F83804B0F878
:10EC0000A8007C49A1F8CE04D4F83804B0F8AA00D2
:10EC10007849A1F8D004D4F83804B0F8AC007549AC
:10EC2000A1F8D204D4F83804B0F8AE007149A1F8C4
:10EC3000D404D4F83804D0F8B0006E49C1F8D80430
:10EC4000D4F83804D0F8B4006A49C1F8DC04D4F828
:10EC50003804D0F8B8006749C1F8E004D4F83804A3
:10EC6000D0F8BC006349C1F8EC04D4F83804D0F8FB
:10EC7000C8006049C1F8F404D4F83804D0F8CC00D6
:10EC80005C49C1F8F804D4F83804D0F8D0005949E8
:10EC9000C1F8FC04D4F83804D0F8C0005549C1F8D4
:10ECA0000005D4F83804D0F8F4005249C1F804053E
:10ECB000D4F83804D0F8F8004E49C1F80805D4F863
:10ECC0003804D0F8FC004B49C1F80C05D4F83804DE
:10ECD000D0F800014749C1F81005D4F83804D0F83D
:10ECE000C4004449C1F8F004D4F83804B0F8D400A2
:10ECF0004049A1F8B404D4F83804D0F8D8003D490C
:10ED00004863D4F83804D0F8DC003A498863D4F872
:10ED10003804B0F8E0003749A1F81405D4F83804F5
:10ED2000D0F8E4003349C1F81805D4F83804B0F835
:10ED3000E8003049A1F81C05D4F83804B0F8EA001E
:10ED40002C49A1F81E05D4F83804B0F8EC00294984
:10ED5000A1F82005D4F83804B0F8EE002549A1F850
:10ED60002205D4F83804B0F804012249A1F80401BE
:10ED7000D4F83804B0F806011E49A1F80601D4F809
:10ED80003804B0F808011B49A1F80801D4F8380488
:10ED9000B0F80A011749A1F82405A21C012120009E
:10EDA000FEF7F5FBA01CC4F83C04C022D4F83C14C8
:10EDB0000D4807F03DF8C022D4F83C0410F1C00122
:10EDC0000A4807F035F8A21C03212000FEF7DFFBFC
:10EDD000A01CC4F84004A022D4F84014044807F052
:10EDE00027F8012010BD0000F8190010B81A001013
:10EDF000781B00101018001020190010491C89B24F
:10EE0000B1F5805F00DB0521080080B270472DE975
:10EE1000F04104000D001600A71C002021780029F5
:10EE200001D1002034E04FF6FF70288000203080B0
:10EE30005FF005081BE0A21C414689B22000FEF7E6
:10EE4000A6FB388847F6AB0188420ED13879FF28F7
:10EE50000BD078882988884201D278882880308829
:10EE60007988884201D27888308018F101081FFA29
:10EE700088F8B8F5805FDEDB2888002806D1308866
:10EE80004FF6FF71884201D1002000E00120C0B29E
:10EE9000BDE8F0812DE9F84304000D000026A71C11
:10EEA0005FF0FF382078002801D1002023E05FF0D8
:10EEB000050919E0A21C494689B22000FEF767FB4C
:10EEC000388847F6AB0188420CD13879FF2809D041
:10EED0007888ADB2A84205D13869404502D24E4685
:10EEE000D7F8108019F101091FFA89F9B9F5805F87
:10EEF000E0DB300080B2BDE8F28300002DE9F04F86
:10EF0000A9B081468A4619F102040025514689B20A
:10EF10004846FFF7BFFF80461FFA88F8B8F1000F98
:10EF200002D129B0BDE8F08F464619F10202310046
:10EF300089B24846FEF72BFB208847F6AB01884292
:10EF400040F0F4832079FF2800F0F08360881FFAF6
:10EF50008AFA504540F0EA8300274AE1DFF8E817D3
:10EF600010A8FDF7E7F910A8FDF774F8010010A844
:10EF7000FDF726F9FFB2402000FB074090F84F0054
:10EF800010F07F0B1FFA8BFBBBF1000F04D1DFF8F1
:10EF9000BC1710A8FDF7CEF91FFA8BFBBBF1010FD0
:10EFA00004D1DFF8AC1710A8FDF7C4F91FFA8BFBEA
:10EFB000BBF1020F04D1DFF89C1710A8FDF7BAF9D6
:10EFC0001FFA8BFBBBF1030F04D1DFF88C1710A8DD
:10EFD000FDF7B0F91FFA8BFBBBF1040F04D1DFF88A
:10EFE0007C1710A8FDF7A6F91FFA8BFBBBF1060FE3
:10EFF00004D1DFF86C1710A8FDF79CF91FFA8BFB02
:10F00000BBF1050F04D1DFF85C1710A8FDF792F9EA
:10F0100010A8FDF71FF8010010A8FDF7D1F8FFB206
:10F02000402000FB0740B0F842B022208DF840009D
:10F030005F208DF841005F208DF842005F208DF841
:10F04000430022208DF844003B208DF8450000202D
:10F050008DF846005FEACB7002D557208DF843004B
:10F060005FEA8B7002D548208DF843005FEA4B5071
:10F0700002D545208DF841005FEA4B6002D5412062
:10F080008DF841005FEACB6002D54C208DF841003D
:10F090005FEA8B6002D552208DF841005FEA0B6079
:10F0A00002D553208DF841005FEA0B7002D54B204A
:10F0B0008DF841005FEA4B7002D543208DF8410086
:10F0C0005FEA0B5002D554208DF841005FEACB4037
:10F0D00002D54E208DF841005FEACB5002D5552075
:10F0E0008DF842005FEA8B5002D544208DF8420033
:10F0F00010A8FCF7AFFF010010A8FDF761F8FFB200
:10F10000402000FB0740428CDFF85C1610A8FDF79A
:10F1100011F910A8FCF79EFF010010A8FDF750F8A8
:10F12000FFB2402000FB0740B0F92620DFF8381678
:10F1300010A8FDF7FFF810A8FCF78CFF010010A83D
:10F14000FDF73EF8FFB2402000FB0740B0F9282051
:10F15000DFF8141610A8FDF7EDF810A8FCF77AFFF9
:10F16000010010A8FDF72CF8FFB2402000FB07407B
:10F17000828CDFF8F41510A8FDF7DCF810A8FCF776
:10F1800069FF010010A8FDF71BF8FFB2402000FB4B
:10F19000074090F92A20DFF8D01510A8FDF7CAF82B
:10F1A00010A8FCF757FF010010A8FDF709F8FFB2FF
:10F1B000402000FB074090F92B20DFF8AC1510A889
:10F1C000FDF7B8F810A8FCF745FF010010A8FCF700
:10F1D000F7FF73A110A8FDF7ADF810A8FCF73AFFF0
:10F1E000010010A8FCF7ECFF4FF47A70FDF734F83B
:10F1F0007F1CFFB2082F80F29982002D04D1FFB24C
:10F20000402000FB07400569FFB2402000FB07409B
:10F21000B0F9200000EE100AB8EEC00AF2EE040ABF
:10F2200080EE200A10EE100AFEF750F8CDE90E012C
:10F23000FFB2402000FB0740B0F91E0000EE100AAC
:10F24000B8EEC00AF2EE040A80EE200A10EE100AB0
:10F25000FEF73CF8CDE90C01FFB2402000FB07406F
:10F26000B0F91C0000EE100AB8EEC00AF2EE040A73
:10F2700080EE200A10EE100AFEF728F8CDE90A0108
:10F28000FFB2402000FB0740B0F91A0000EE100A60
:10F29000B8EEC00AF2EE040A80EE200A10EE100A60
:10F2A000FEF714F8CDE90801FFB2402000FB07404B
:10F2B000B0F9180000EE100AB8EEC00AF2EE040A27
:10F2C00080EE200A10EE100AFEF700F8CDE90601E4
:10F2D000FFB2402000FB0740B0F9160000EE100A14
:10F2E000B8EEC00AF2EE040A80EE200A10EE100A10
:10F2F000FDF7ECFFCDE90401FFB2402000FB074021
:10F30000B0F9140000EE100AB8EEC00AF2EE040ADA
:10F3100080EE200A10EE100AFDF7D8FFCDE90201B9
:10F32000FFB2402000FB07400069401B00EE100ABE
:10F33000B8EE400ADFED980A80EE200A10EE100ABF
:10F34000FDF7C4FFCDE90001B6B233006288DFF8F3
:10F350001C1410A8FCF7EEFF10A8FCF77BFE0100C0
:10F3600010A8FCF72DFFFFB2402000FB074090F8EB
:10F370004400FFB2402101FB074191F8451051EADA
:10F38000002B1FFA8BFB5FEA9B1B5FEA8B5009D5B2
:10F390005FEACB50C00D5FF0FF3110FB01F204E0DB
:10F3A0000D0A00005FEACB52D20D12B2DFF8B8139B
:10F3B00010A8FCF7BFFF10A8FCF74CFE010010A836
:10F3C000FCF7FEFEFFB2402000FB074090F845002E
:10F3D000FFB2402101FB074191F8461051EA002B92
:10F3E0001FFA8BFB5FEA1B1B5FEA8B5007D55FEAB6
:10F3F000CB50C00D5FF0FF3110FB01F202E05FEA7D
:10F40000CB52D20D12B2D84910A8FCF793FF10A826
:10F41000FCF720FE010010A8FCF7D2FEFFB240204E
:10F4200000FB074090F84600FFB2402101FB074176
:10F4300091F8471051EA002B1FFA8BFB5FEA9B0BF8
:10F440005FEA8B5007D55FEACB50C00D5FF0FF310C
:10F4500010FB01F202E05FEACB52D20D12B2C249B8
:10F4600010A8FCF767FF10A8FCF7F4FD010010A836
:10F47000FCF7A6FEFFB2402000FB074090F84700D3
:10F48000FFB2402101FB074191F8481051EA002BDF
:10F490005FEA8B52920D12B2B34910A8FCF74AFFF3
:10F4A00010A8FCF7D7FD010010A8FCF789FEFFB2F9
:10F4B000402000FB074090F84900FFB2402101FBCB
:10F4C000074191F84A1051EA002B1FFA8BFB5FEAC3
:10F4D0009B1B5FEA8B5007D55FEACB50C00D5FF0F6
:10F4E000FF3110FB01F202E05FEACB52D20D12B203
:10F4F0009D4910A8FCF71EFF10A8FCF7ABFD01000A
:10F5000010A8FCF75DFEFFB2402000FB074090F81A
:10F510004A00FFB2402101FB074191F84B1051EA2C
:10F52000002B1FFA8BFB5FEA1B1B5FEA8B5007D592
:10F530005FEACB50C00D5FF0FF3110FB01F202E03B
:10F540005FEACB52D20D12B2874910A8FCF7F2FE47
:10F5500010A8FCF77FFD010010A8FCF731FEFFB2F8
:10F56000402000FB074090F84B00FFB2402101FB18
:10F57000074191F84C1051EA002B1FFA8BFB5FEA10
:10F580009B0B5FEA8B5009D55FEACB50C00D5FF053
:10F59000FF3110FB01F204E000007A445FEACB5235
:10F5A000D20D12B2704910A8FCF7C4FE10A8FCF7E7
:10F5B00051FD010010A8FCF703FEFFB2402000FB44
:10F5C000074090F84C00FFB2402101FB074191F841
:10F5D0004D1051EA002B5FEA8B52920D12B2624934
:10F5E00010A8FCF7A7FE10A8FCF734FD010010A836
:10F5F000FCF7E6FDFFB2402000FB074090F84E000C
:10F60000C0B2C209D2B2584910A8FCF793FE10A8A4
:10F61000FCF720FD010010A8FCF7D2FDFFB240204E
:10F6200000FB074090F84E0010F07F024E4910A8F2
:10F63000FCF780FE10A8FCF70DFD010010A8FCF7F8
:10F64000BFFDFFB2402000FB0740806BFDF73EFE90
:10F65000CDE90001FFB2402000FB0740406BFDF701
:10F6600035FE02000B00424910A8FCF763FE10A80B
:10F67000FCF7F0FC010010A8FCF7A2FDFFB240204F
:10F6800000FB0740B0F9400000EE100AB8EEC00AD7
:10F69000F2EE040A80EE200A10EE100AFDF716FEC4
:10F6A000CDE90201FFB2402000FB0740B0F93E0067
:10F6B00000EE100AB8EEC00A10EE100AFDF706FEC2
:10F6C000CDE90001FFB2402000FB0740808F00EE33
:10F6D000100AB8EE400AF2EE040A80EE200A10EE9C
:10F6E000100AFDF7F3FD02000B00224910A8FCF7F9
:10F6F00021FE10A8FCF7AEFC010010A8FCF760FD8D
:10F70000FFB2402000FB074090F84F00C0B25FEA14
:10F71000D01B5FFA8BFB1FFA8BFBBBF1000F3FF492
:10F720001DAC154910A8FCF705FE1CE4761CB6B20A
:10F73000B6F5805F00DB0526B6B21FFA88F84645AD
:10F740007FF4F3ABFFF7EDBB743302088831020896
:10F7500094310208F42D0208042E0208142E020827
:10F76000A0310208AC31020864330208E4F9010850
:10F77000E42D0208002102086C3302082DE9F84349
:10F7800004002078002801D100205CE0002500263C
:10F7900000274FF6FF785FF0050908E01FFA89F9A6
:10F7A0001FFA88F8C14500D2C84619F101091FFAAD
:10F7B00089F9B9F5805F28DA14F50672494689B2ED
:10F7C0002000FDF7E4FEB4F8180247F6AB018842CA
:10F7D000E4D194F81C02FF28E0D0B4F81A02ADB2CC
:10F7E000854207D1D4F828028642DED2D4F82862B6
:10F7F0004F46DAE7B4F81A02ADB28542D5D2B4F872
:10F800001A52D4F828624F46CFE7BFB2002F09D171
:10F810001FFA88F84FF6FF70804501D0474607E091
:10F82000052705E0390089B22000FFF7E7FA070055
:10F83000ADB2002D01D1012500E06D1CA4F81452D9
:10F84000A4F812720120BDE8F28310B504004FF451
:10F850000472FF2114F50670FCF7F2FB47F6AB00CB
:10F86000A4F81802B4F81402A4F81A02FF2084F8CD
:10F870001C0210BD10B504002078002805D020001F
:10F88000FFF77CFF2000FFF7E0FF10BD10B5DFF8A9
:10F89000240B002101704FF4407005F0ADFADFF841
:10F8A000180B007800280DD1DFF8100B04F02CF9AC
:10F8B000DFF8502CDFF8081B06F0C1FADFF8F80A71
:10F8C00001210170DFF8400C006804F0AAF9DFF8AC
:10F8D000380C006804F0B3F9DFF8300CDFF8E41AF4
:10F8E0000160DFF8280C0068411EDFF8202C116051
:10F8F0000028F6D1DFF8D00A006810F00C000828C4
:10F9000030D0DFF8080CDFF8BC1A0160DFF8FC0B20
:10F910000068411EDFF8F42B11600028F6D1DFF8F3
:10F92000E80B006804F084F9DFF8DC0B006804F0F1
:10F930008DF9DFF8D80BDFF8D81B0160DFF8CC0BAE
:10F940000068411EDFF8C42B11600028F6D1DFF8F3
:10F95000B80B006804F065F9DFF8AC0B006804F040
:10F960006EF9CEE7DFF8640A0068C0F38050012822
:10F9700030D0DFF8980BDFF84C1A0160DFF88C0B01
:10F980000068411EDFF8842B11600028F6D1DFF8F3
:10F99000780B006804F04CF9DFF86C0B006804F099
:10F9A00055F9DFF8680BDFF8681B0160DFF85C0BC6
:10F9B0000068411EDFF8542B11600028F6D1DFF8F3
:10F9C000480B006804F02DF9DFF83C0B006804F0E8
:10F9D00036F9CEE7DFF83C0B007800280DD1DFF8D0
:10F9E000380BFDF79FFCDFF81C2BDFF8301B06F00F
:10F9F00026FADFF8200B01210170DFF8240B0068E4
:10FA0000FEF77EFCC0B2002802D00020002801D002
:10FA100000F00FFADFF8600D90F8E000002804D045
:10FA2000DFF8FC0A0068FFF725FFDFF8DC0A006852
:10FA300004F021F9C00702D40020002825D000F0EE
:10FA4000F8F917E0C00702D40020002818D0DFF82A
:10FA5000BC0ADFF8BC1A0160DFF8B00A0068411E7A
:10FA6000DFF8A82A11600028F6D1DFF89C0A0068A8
:10FA700004F0F3F8DFF8900A006804F0FCF8E1E71E
:10FA8000DFF8840A006804F0CCF8DFF8980A007800
:10FA900000280DD1DFF8900AFCF766FCDFF8642A35
:10FAA000DFF8881A06F0CBF9DFF8780A0121017037
:10FAB000DFF87C0A0068FCF766FCDFF8780A00785B
:10FAC00000280DD1DFF8700A02F004FADFF8342ABA
:10FAD000DFF8681A06F0B3F9DFF8580A012101705F
:10FAE000DFF85C0A007800280DD1DFF8580A05F02D
:10FAF0007DFDDFF8102ADFF8501A06F0A0F9DFF8D4
:10FB0000400A01210170DFF8440A007800280DD175
:10FB1000DFF83C0A00F0B8FFDFF8E829DFF8341A14
:10FB200006F08DF9DFF8240A01210170DFF8280AB8
:10FB3000007800280DD1DFF8240A01F0A7F9DFF8DA
:10FB4000C429DFF81C1A06F07AF9DFF80C0A012143
:10FB50000170DFF8100A007800280DD1DFF8080ADC
:10FB600005F0EAFADFF89C29DFF8001A06F067F9D9
:10FB7000DFF8F00901210170DFF8F40900780028AE
:10FB80000DD1DFF8F00905F067FCDFF87829DFF820
:10FB9000E81906F054F9DFF8D80901210170DFF8FF
:10FBA000DC09007800280DD1DFF8D409FCF782FECB
:10FBB000DFF85029DFF8CC1906F041F9DFF8BC096D
:10FBC00001210170DFF8C009007800280DD1DFF8AD
:10FBD000BC09F0F7D9FADFF82C29DFF8B41906F0E0
:10FBE0002EF9DFF8A40901210170DFF8A8090078D7
:10FBF00000280DD1DFF8A00901F0BAFDDFF80429D3
:10FC0000DFF8981906F01BF9DFF888090121017067
:10FC1000DFF88C09007800280DD1DFF8880902F0A0
:10FC20005DFADFF8E028DFF8801906F008F9DFF860
:10FC3000700901210170DFF8440B007800280DD114
:10FC4000DFF83C0B03F000F9DFF8B828DFF8341BCD
:10FC500006F0F5F8DFF8240B01210170DFF8280B1E
:10FC6000007800280DD1DFF8240B01F053FFDFF8F6
:10FC70009428DFF81C1B06F0E2F8DFF80C0B0121DA
:10FC80000170DFF8100B007800280DD1DFF8080BA9
:10FC900006F0DAF8DFF86C28DFF8001B06F0CFF882
:10FCA000DFF8F00A01210170DFF8F40A007800287B
:10FCB0000DD1DFF8F00A06F065F9DFF84828DFF823
:10FCC000E81A06F0BCF8DFF8D80A01210170DFF865
:10FCD000A80A0021A0F8F410DFF89C0A0021A0F87F
:10FCE000F610DFF8940A0021A0F8F810DFF8880A6F
:10FCF000002180F8CA14DFF8800A002180F8CC14B3
:10FD0000DFF8740A0121A0F8E414DFF86C0A00217E
:10FD1000A0F8E614DFF8600A0021A0F8E814DFF884
:10FD2000E807006803F0C9FFDFF84C0A90F8C9142F
:10FD3000DFF8780A006802F0F8F9DFF8700A006866
:10FD400002F01BFADFF8640A006802F07BFCDFF8BF
:10FD50005C0A006803F028F8DFF8540A0068FCF732
:10FD6000B8FDDFF84C0A0068FCF7CEFD40B2012870
:10FD700037DADFF83C0A0068FCF7A4FFDFF8300A46
:10FD80000068FCF7C1FD40B2012802DA40B200F081
:10FD900011FD062418E0DFF87407DFF8741701601E
:10FDA000DFF868070068411EDFF86027116000284F
:10FDB000F6D1DFF85407006803F04FFFDFF848077B
:10FDC000006803F051FF641E012CE4DADFF8380705
:10FDD000006803F02DFFDFF83007006803F036FFFE
:10FDE000FEE7062418E0DFF82407DFF82417016097
:10FDF000DFF818070068411EDFF81027116000289F
:10FE0000F6D1DFF80407006803F027FFDFF8F806F3
:10FE1000006803F029FF641E012CE4DADFF8E8062D
:10FE2000006803F005FFDFF8E006006803F00EFF4E
:10FE3000FEE780B5DFF8400900210182DFF83809CC
:10FE400000214182DFF8300900218182DFF8280992
:10FE50000021C182DFF8200900210183DFF81809A1
:10FE600000214183DFF8100900210160DFF8080953
:10FE700000218171DFF800090021C171DFF8F80865
:10FE800064218180DFF8F008002180F84010DFF85D
:10FE9000E8082821A0F84210DFF8DC085FF0FF3105
:10FEA000A0F84410DFF8D0080121A0F84610DFF8D0
:10FEB000C8085FF0FF31A0F84810DFF8BC085FF019
:10FEC000FF31A0F85010DFF8B0085FF0FF31A0F864
:10FED0005210DFF8A4085FF0FF31A0F85410DFF8EB
:10FEE00098080121A0F85610DFF88C080121A0F82D
:10FEF0004A10DFF884080121A0F84C10DFF87808D8
:10FF00000121A0F84E10DFF870080021A0F85A1067
:10FF1000DFF8640840F2FF31A0F85C10DFF8580801
:10FF20004FF4AF71A0F85810DFF84C08DFF8241A2E
:10FF30000166DFF84408DFF8201A4166DFF8380868
:10FF400000218166DFF830080021C166DFF828084B
:10FF5000DFF8081A0167DFF82008DFF8041AC0F894
:10FF6000C811DFF814080021C0F89C10DFF8080859
:10FF7000DFF8F0198167DFF800085FF07E51C0F804
:10FF80008810DFF8F407DFF8E019C0F88C10DFF80C
:10FF9000E807DFF8D819C0F8A010DFF8DC07DFF8B1
:10FFA000CC19C0F8A410DFF8D007DFF8C019C0F8EA
:10FFB000A810DFF8C407DFF8B819C0F8AC10DFF8F4
:10FFC000B807DFF8AC19C0F8B010DFF8AC07DFF8FD
:10FFD000A019C0F8B410DFF8A007DFF89819C0F82E
:10FFE000B810DFF89407DFF88C19C0F8BC10DFF800
:10FFF0008807DFF88419C0F8C010DFF87C07DFF845
:020000040801F1
:100000007819C0F8C410DFF87007DFF86C19C0F871
:10001000C810DFF86407DFF86419C0F8CC10DFF807
:100020005807DFF85C19C0F8D010DFF84C07DFF88C
:100030003819C0F8D410DFF84007DFF84019C0F8CD
:10004000D810DFF83407DFF83C19C0F8DC1078224C
:100050000021DFF83409FBF7F3FFDFF81C0700216C
:1000600080F8E010DFF81007002180F8E110DFF8D9
:1000700008072D21A0F8E210DFF8FC060021A0F807
:10008000E410DFF8F4060021C0F8E810DFF8E80615
:10009000DFF8F818C0F8EC10DFF8DC06DFF8F0182D
:1000A000C0F8F010DFF8D0060A21A0F8FA10DFF847
:1000B000C8065FF08041C0F8FC10DFF8BC065A218A
:1000C000A0F80011DFF8B0061E21A0F80211DFF839
:1000D000A8062821A0F80411DFF89C064B21A0F8FF
:1000E0000611DFF894060021A0F80811DFF8880651
:1000F0005FF08041C0F80C11DFF87C060021A0F809
:10010000C411DFF87406002180F88811DFF8680652
:10011000DFF88018C0F88C11DFF85C06DFF878187B
:10012000C0F89011DFF85006DFF83C18C0F89411C1
:10013000DFF844065FF07C51C0F89811DFF838060C
:10014000DFF85818C0F89C11DFF82C06DFF85018BB
:10015000C0F8A011DFF82006DFF84818C0F8A41195
:10016000DFF81406DFF83C18C0F8A811DFF808061D
:10017000DFF83418C0F8AC11DFF8FC05DFF82C18F4
:10018000C0F8B011DFF8F005DFF82418C0F8B4119A
:10019000DFF8E405DFF81C18C0F8B811DFF8D8055F
:1001A000DFF81418C0F8BC11DFF8CC050021C0F846
:1001B000C011DFF8C405022180F88911DFF8B80505
:1001C000DFF8F817C0F8CC11DFF8AC05DFF8F0174E
:1001D000C0F8D011DFF8A005DFF8E817C0F8D41197
:1001E000DFF894050021C0F8D811DFF88C05002154
:1001F000C0F8DC11DFF880050021C0F8E011DFF85D
:1002000078050021C0F8E411DFF86C05002180F8C2
:10021000C814DFF864050021A0F8CE14002056E0D1
:1002200080B2DFF8541511EBC001002281F8E821FB
:1002300080B2DFF8441511EBC001002281F8E921FA
:1002400080B2DFF8341511EBC0014FF47A72A1F8D7
:10025000EA2180B2DFF8201511EBC0014FF4FA62F9
:10026000A1F8EC2180B2DFF8101511EBC00140F2CB
:10027000DC52A1F8EE2180B2DFF8FC1411EBC001D2
:10028000002281F8A82280B2DFF8EC1411EBC00143
:10029000002281F8A92280B2DFF8DC1411EBC00142
:1002A0004FF47A72A1F8AA2280B2DFF8CC1411EBD5
:1002B000C0014FF4FA62A1F8AC2280B2DFF8B814A2
:1002C00011EBC00140F2DC52A1F8AE22401C80B21A
:1002D0001828A5DB00200FE089B280B20A22DFF8DF
:1002E000983402FB00328A18002382F86833491CD4
:1002F00089B20A29F0DB401C80B2102801DA002103
:10030000F6E7DFF87404642180F86813DFF8680406
:10031000642180F87313DFF86004642180F87E1391
:10032000DFF85404642180F88913DFF84C04642159
:1003300080F89413DFF84004642180F89F13DFF8FD
:100340003804642180F8AA13DFF82C04642180F8B3
:10035000B513DFF82404642180F8C013DFF8180413
:10036000642180F8CB13DFF810040021A0F81415E5
:10037000DFF80404DFF85016C0F81815DFF8F803AA
:100380001E21A0F81C15DFF8F0030021A0F81E15AF
:10039000DFF8E4031921A0F82015DFF8DC035A2167
:1003A000A0F82215DFF8D0030021A0F8241500F0F2
:1003B000FDF801BDF03300109FB40020EC330010B5
:1003C000213C010840420F00083802400438024036
:1003D000DFF8F805DFF8F815C0F8B814DFF8EC0519
:1003E000DFF8F015C0F8BC14DFF8E005DFF8E81519
:1003F000C0F8C014DFF8D405DFF8E015C0F8C41465
:10040000DFF8C8050121A0F8D014DFF8C0050121EC
:10041000A0F8D214DFF8B4050121A0F8D414DFF855
:10042000AC05DFF8B415C0F8D814DFF8A0055FF00C
:100430007E51C0F8DC14DFF89405DFF82815C0F809
:10044000E014DFF888055FF07C51C0F8EC14DFF8A9
:100450007C05DFF80015C0F8F414DFF87005DFF84C
:10046000F414C0F8F814DFF86405DFF8E814C0F8F5
:10047000FC14DFF85805DFF86815C0F80015DFF840
:100480004C05DFF86015C0F80415DFF84005DFF80B
:100490005415C0F80815DFF83405DFF84C15C0F81E
:1004A0000C15DFF82805DFF83815C0F81015DFF84F
:1004B0001C05DFF8B814C0F8F014DFF810050021AF
:1004C000C161DFF8080500210162DFF80005DFF8EF
:1004D0001C154162DFF8F40400218162DFF8EC04AE
:1004E000DFF87014C162DFF8E404DFF8041501637B
:1004F000DFF8D80400214163DFF8D00400218163D4
:100500007047000098B4002070B40020E833001059
:10051000404B4C00A0B40020381D001081D30008CF
:1005200054B40020A1B40020C833001085C30008D3
:1005300080B40020A2B40020D8330010F31E0108BC
:10054000A3B400208C33001029560108A4B4002065
:100550008C320010D70A0108A5B40020AC2D001081
:10056000030F0108A6B40020A0310010815101083A
:10057000A7B40020B033001077540108A8B40020BD
:10058000442F0010BDC80008A9B400207C21001031
:10059000B5020008AAB40020D02B0010A117010852
:1005A000ABB40020D426001029210108724828216C
:1005B00001817148282181726F4840F27121818147
:1005C0006D48782181736C485FF0FF31C0F880106E
:1005D0006948002180F8C9146748002180F8CB14CD
:1005E0006548002180F8CD1463480021C0F8081444
:1005F00061480A21C0F80C145F487021C0F810143B
:100600005D488221C0F814145B48DFF8E813C0F895
:10061000181459483C21C0F81C1457484621C0F80A
:1006200020145548DFF8D013C0F824145248DFF8DE
:10063000CC13C0F828145048DFF8C413C0F82C14A9
:100640004D48AA21C0F830144B48B521C0F83414E5
:1006500049481E21C0F838144748DFF8A813C0F8ED
:100660003C144548DFF8A013C0F840144248DFF8B6
:100670009C13C0F844144048DFF89413C0F84814A1
:100680003D48DFF89013C0F84C143B48DFF888135E
:10069000C0F850143848DFF88413C0F854143648B2
:1006A000DFF87C13C0F858143348DFF87813C0F82B
:1006B0005C1431485FF00111C0F860142E48DFF877
:1006C0006813C0F864142C48DFF86013C0F868148D
:1006D0002948DFF85C13C0F86C142748DFF854137E
:1006E000C0F870142448DFF85013C0F8741422487E
:1006F000DFF84813C0F878141F48DFF84413C0F837
:100700007C141D48DFF83C13C0F880141A48DFF849
:100710003813C0F884141848CC49C0F88814164817
:10072000CB49C0F88C141448CA49C0F89014124838
:10073000C949C0F894141048C849C0F898140E4824
:10074000C749C0F89C140C48C649C0F8A0140A4810
:10075000C549C0F8A4140848C449C0F8A8140648FC
:10076000C349C0F8AC1404480021A0F8B4140248EE
:10077000C049C0F8B014704710180010ACB4002085
:1007800064290010E12E0108ADB4002034240010CB
:100790001D1B0108AEB40020A8300010775F0108CF
:1007A000AFB40020000000103F6101086CB40020CD
:1007B0005CB4002038B540B24442AF48006803F052
:1007C00037FAAD48006803F041FAAC480100481E12
:1007D0000029FBD1AA480100481E0029FBD1E007EF
:1007E0002BD504251AE0A448006803F01AFAA248A1
:1007F000006803F02BFAA2480100481E0029FBD133
:100800009D48006803F014FA9B48006803F017FA4B
:100810009B480100481E0029FBD16D1E002DE2D12E
:100820009548006803F004FA9348006803F00EFA54
:1008300092480100481E0029FBD1A00727D58E4809
:10084000006803F003FA042512E08B48006803F007
:10085000E8F98B480100481E0029FBD18648006852
:1008600003F0E6F987480100481E0029FBD16D1E00
:10087000002DEAD18048006803F0DAF97E4800686C
:1008800003F0E4F97D480100481E0029FBD1600710
:1008900027D57948006803F0CBF9042512E07648A3
:1008A000006803F0CCF976480100481E0029FBD10E
:1008B0007148006803F0CAF972480100481E002917
:1008C000FBD16D1E002DEAD16B48006803F0B0F932
:1008D0006948006803F0BAF968480100481E002919
:1008E000FBD120077FF57BAF6348006803F0A0F9D8
:1008F0006148006803F0AAF904251AE05E48006820
:1009000003F09DF95C48006803F08BF95C48010036
:10091000481E0029FBD15848006803F097F9564853
:10092000006803F085F957480100481E0029FBD1F3
:100930006D1E002DE2D15048006803F079F94E4851
:10094000006803F083F94D480100481E0029FBD1DF
:1009500045E70000CDCC4C3E00004040000048423E
:10096000CDCC4C3F0000C8410000F041CDCCCC3D87
:100970009A99993F00005C420000344200002041F7
:100980000000A0410000A04020190010CD9B604253
:1009900030D02E4279E9063F000040C1F853A33E13
:1009A000BDC60E3E718F053EF0A7063F00007AC41B
:1009B00000401C455C8FC23E000020403333334171
:1009C000CDCC144100209945333323411018001039
:1009D0000AD7233C00803B450000C8429A99193E43
:1009E0003333B33E9A99193F9A99993E000080BFDC
:1009F0009A9919BF5D0039001A009B001E0046003D
:100A00001A0055005D00B4000A006E001E0040018F
:100A100032004600D200C0001800C0000100BA0039
:100A20000200C800010071000E0001001900010061
:100A30002F0001004600010030004B002100320071
:100A400019003200C8000100D200010002003C0081
:100A500028007800B400FA0001004001C400FA0048
:100A600001005E010A005E016E0022010100040126
:100A7000020064003200780070B4002080F0FA02B6
:100A8000404B4C008096980010B5040014F12400EF
:100A900005F064FB14F15C0005F060FB14F19400B8
:100AA00005F05CFB00202070002060700020E060FA
:100AB000002020610020E061002060610020A06132
:100AC000A020A070B020A070F020A070DFF89C03E0
:100AD0000460200010BD38B50400DFF89003002149
:100AE0000160250014F1940005F039FB14F15C005D
:100AF00005F035FB14F1240005F031FB280032BD70
:100B000000B585B00121082004F02BFA01214FF433
:100B1000804004F046FA00208DF80C0000208DF88B
:100B20000F000420029002A9D14804F07FFA0221AC
:100B3000032005F0ADFB0420009000208DF8040098
:100B400008208DF8050001208DF8060000A804F0AB
:100B5000E3FC05B000BD80B5012100F001F801BD46
:100B600030B587B004000D000020207000206070B8
:100B700041F288300090A07850F00F03DBB22022C1
:100B8000D021BC48006804F0CFFEC0B2002802D0DB
:100B90000020002803D00120607007B030BDB648A7
:100BA000206241F28830009021232322D021B148D5
:100BB000006804F0B9FEC0B2002802D0002000286E
:100BC00002D002206070E8E741F2883000900823EC
:100BD0002222D021A748006804F0A6FEC0B2002857
:100BE00002D00020002802D003206070D5E7EDB2CB
:100BF000002D02D001202070CFE742F2107001904A
:100C00000120009002AB0F22D0219A48006804F026
:100C1000DDFEC0B2002802D00020002802D004204F
:100C20006070BAE79DF80800D32802D005206070F4
:100C3000B3E7924800E0401E91490968490701D492
:100C40000028F8D1002802D106206070A5E742F202
:100C5000107001900820009002ABA622D021854898
:100C6000006804F0B3FEC0B2002802D000200028C3
:100C700002D00720607090E7002000E0401C80490F
:100C80000968490702D47D498842F7D3002802D178
:100C90000820607081E77A480068400702D4092084
:100CA00060707AE742F2107001900820009002AB69
:100CB000A622D0216F48006804F088FEC0B2002848
:100CC00002D00020002802D00A20607065E76D483D
:100CD000006802F0ADFF200000F036F8012020701F
:100CE0005BE70021017070471CB5040020780028E4
:100CF00002D10120607013BD200000F01FF8002811
:100D000002D00020002802D002206070F3E700200B
:100D1000019008200090231DA622D021554800688C
:100D200004F054FEC0B2002802D00020002802D0F7
:100D300003206070DFE700206070DCE75048006847
:100D4000C0F38000C0B2704710B504009FED450AA3
:100D500014F1240005F090FAB7EE000A14F1240013
:100D600005F08DFA9FED400A14F1240005F08DFA8C
:100D7000454890ED000AF7EE000AB4EE600AF1EE85
:100D800010FA06D5B7EE000A14F1240005F07AFA3D
:100D900006E03D4890ED000A14F1240005F072FAD7
:100DA00014F1240005F0DCF99FED2E0A14F15C002B
:100DB00005F062FAB7EE000A14F15C0005F05FFA84
:100DC0009FED290A14F15C0005F05FFA2E4890EDC2
:100DD000000AF7EE000AB4EE600AF1EE10FA06D54A
:100DE000B7EE000A14F15C0005F04CFA06E0264864
:100DF00090ED000A14F15C0005F044FA14F15C0077
:100E000005F0AEF99FED170A14F1940005F034FADD
:100E1000B7EE000A14F1940005F031FA9FED120AC2
:100E200014F1940005F031FA174890ED000AF7EE3E
:100E3000000AB4EE600AF1EE10FA06D5B7EE000A29
:100E400014F1940005F01EFA06E00F4890ED000A38
:100E500014F1940005F016FA14F1940005F080F9ED
:100E600010BD00008FC2353F0000484460B4002030
:100E7000000C024058B40020295C8F3D40420F0016
:100E8000100C024070B40020E81C001010B50400E3
:100E900014F1480005F062F914F1800005F05EF9E4
:100EA00014F1B80005F05AF914F1F00005F056F904
:100EB00014F5947005F052F914F5B07005F04EF980
:100EC00000206070002084F824000020A070002022
:100ED000E06000202061002060610020A06100200F
:100EE00084F8250000202063002060630020A063B8
:100EF0000020E06300202070DFF83C080460200040
:100F000010BD38B50400DFF830080021016025006D
:100F100014F5B07005F023F914F5947005F01FF97D
:100F200014F1F00005F01BF914F1B80005F017F901
:100F300014F1800005F013F914F1480005F00FF9E1
:100F4000280032BD00B583B00121042004F009F867
:100F500001214FF4804004F024F800208DF80400B3
:100F600000208DF807004FF48050009000A9DFF8B2
:100F7000CC0704F05BF807BD00B583B00121042065
:100F800003F0EFFF01214FF4804004F00AF8002045
:100F90008DF8040000208DF807004FF400600090E9
:100FA00000A9DFF8980704F041F807BD30B587B015
:100FB00004000D00002060700020A070DFF88007A2
:100FC00000903F2320223021DFF87807006804F0EA
:100FD000ABFCC0B2002802D00020002803D00120C2
:100FE000A07007B030BDDFF8580700901A23222206
:100FF0003021DFF85007006804F096FCC0B20028EA
:1010000002D00020002802D00220A070E9E75FF0A3
:101010006650E0615FF066502062DFF824070090C0
:10102000B02323223021DFF81C07006804F07CFC89
:10103000C0B2002802D00020002802D00220A070F8
:10104000CFE7EDB2002D02D001206070C9E742F277
:10105000107001900520009002ABA0223021DFF833
:10106000E406006804F0B2FCC0B2002802D0002000
:10107000002802D01E20A070B3E7DFF8CC5600E0B5
:101080006D1E200000F085F9002803D1002D01D04D
:10109000012000E00020C0B20028F1D1002D02D1D3
:1010A0000620A0709DE742F2107001900820009089
:1010B00002ABA6223021DFF88C06006804F086FC23
:1010C000C0B2002802D00020002802D00720A07063
:1010D00087E7002500E06D1C200000F05AF9002889
:1010E00005D1DFF86406854201D2012000E000202E
:1010F000C0B20028EFD1002D02D10820A07070E707
:10110000200000F046F9002802D00020002802D07C
:101110000920A07065E742F210700190082000904D
:1011200002ABA6223021DFF81C06006804F04EFC5A
:10113000C0B2002802D00020002802D00A20A070EF
:101140004FE7DFF80806006802F080FD200000F09D
:10115000D1F90120607044E780B50121FFF726FF37
:1011600001BD80B5012100F001F801BD30B587B0A7
:1011700004000D00002084F82400002084F82500DD
:1011800042F2107001900320009002AB0A223C2131
:10119000DFF8B005006804F019FCC0B2002802D0E6
:1011A0000020002804D0012084F8250007B030BDBD
:1011B0009DF80800482807D19DF80900342803D17C
:1011C0009DF80A00332803D0022084F82500EDE7BB
:1011D00042F2107001900120009002AB0F223C21DE
:1011E000DFF86005006804F0F1FBC0B2002802D00F
:1011F0000020002803D0012084F82500D6E79DF8C0
:1012000008003C2802D10220207001E0012020705B
:10121000DFF82C050090182300223C21DFF824057C
:10122000006804F081FBC0B2002802D00020002832
:1012300003D0032084F82500B8E72078022806D1DF
:10124000DFF80C052064DFF80C05606405E0DFF8CA
:1012500008052064DFF804056064DFF8E40400900A
:10126000212301223C21DFF8DC04006804F05CFB50
:10127000C0B2002802D00020002803D0042084F847
:10128000250093E7DFF8B8040090002302223C21F8
:10129000DFF8B004006804F047FBC0B2002802D0B9
:1012A0000020002803D0052084F825007EE7EDB259
:1012B000002D03D0012084F8240077E742F210705B
:1012C00001900620009002AB03223C21DFF8740459
:1012D000006804F07BFBC0B2002802D00020002888
:1012E00003D0032084F8250060E7002500208DF856
:1012F000080000E06D1C9DF80800C0071AD4DFF854
:101300004804854216D242F21070019001200090EC
:1013100002AB09223C21DFF82C04006804F056FBE4
:10132000C0B2002802D000200028E3D0062084F8B4
:1013300025003BE7002D03D1072084F8250035E781
:10134000DFF80404854203D1082084F825002DE746
:1013500042F2107001900620009002AB03223C2163
:10136000DFF8E003006804F031FBC0B2002802D0CF
:101370000020002803D0092084F8250016E78020EB
:1013800084F82600200000F043F9012084F82400AE
:101390000CE7DFF8CC030068C00A10F001007047CA
:1013A0001CB5040094F82400002803D1012084F81F
:1013B000250013BDFF2084F82600002001900120A5
:1013C000009014F1260309223C21DE48006804F055
:1013D000FDFAC0B2002802D00020002806D08020EC
:1013E00084F82600022084F82500E2E7002084F833
:1013F0002500DEE790F82610C9B2FF2905D090F845
:10140000262052F0800280F82620080602D5080027
:10141000C0B201E011F0010070471CB50400607813
:10142000002802D10120A07013BD2000FFF7B1FFFA
:10143000002802D00020002802D00220A070F3E78C
:101440000020019008200090231DA6223021BD48D5
:10145000006804F0BBFAC0B2002802D000200028C7
:1014600002D00320A070DFE70020A070DCE71CB5ED
:10147000040094F82400002803D1012084F82500FA
:1014800013BD002001900620009014F128030322D0
:101490003C21AC48006804F099FAC0B2002802D0A0
:1014A0000020002803D0012084F82500E8E7002070
:1014B00084F82500E4E7704710F128010A784B789A
:1014C00053EA022202858A78CB7853EA02224285C7
:1014D0000A79497951EA022181850178022907D1E7
:1014E000418DA04A1180818D41859E490988818561
:1014F0007047000010B504009FED8C0A14F14800FD
:1015000004F0BAFEB7EE000A14F1480004F0B7FE8A
:101510009FED870A14F1480004F0B7FE924890ED61
:10152000000AF7EE000AB4EE600AF1EE10FA06D5F2
:10153000B7EE000A14F1480004F0A4FE06E08A4861
:1015400090ED000A14F1480004F09CFE14F14800EC
:1015500004F006FE9FED750A14F1800004F08CFE85
:10156000B7EE000A14F1800004F089FE9FED700AC6
:1015700014F1800004F089FE7B4890ED000AF7EE3C
:10158000000AB4EE600AF1EE10FA06D5B7EE000AD2
:1015900014F1800004F076FE06E0734890ED000A36
:1015A00014F1800004F06EFE14F1800004F0D8FD08
:1015B0009FED5E0A14F1B80004F05EFEB7EE000A7B
:1015C00014F1B80004F05BFE9FED590A14F1B80065
:1015D00004F05BFE644890ED000AF7EE000AB4EEFA
:1015E000600AF1EE10FA06D5B7EE000A14F1B80061
:1015F00004F048FE06E05C4890ED000A14F1B800E3
:1016000004F040FE14F1B80004F0AAFD10BD000083
:1016100010B504009FED450A14F1F00004F02CFE13
:10162000B7EE000A14F1F00004F029FE9FED410A24
:1016300014F1F00004F029FE4C4890ED000AF7EE9A
:10164000000AB4EE600AF1EE10FA06D5B7EE000A11
:1016500014F1F00004F016FE06E0444890ED000A94
:1016600014F1F00004F00EFE14F1F00004F078FD27
:101670009FED2E0A14F5947004F0FEFDB7EE000AFB
:1016800014F5947004F0FBFD9FED2A0A14F5947094
:1016900004F0FBFD354890ED000AF7EE000AB4EEC9
:1016A000600AF1EE10FA06D5B7EE000A14F5947050
:1016B00004F0E8FD06E02D4890ED000A14F5947062
:1016C00004F0E0FD14F5947004F04AFD9FED170A54
:1016D00014F5B07004F0D0FDB7EE000A14F5B07048
:1016E00004F0CDFD9FED130A14F5B07004F0CDFDAC
:1016F0001E4890ED000AF7EE000AB4EE600AF1EE23
:1017000010FA06D5B7EE000A14F5B07004F0BAFD71
:1017100006E0164890ED000A14F5B07004F0B2FD32
:1017200014F5B07004F01CFD10BD00008FC2353FF1
:1017300000007A440000964268B40020000802408D
:10174000A086010058B4002040420F0070B4002071
:101750003DE79A3AFBDEAD3AB182A13A975CB33AE3
:10176000100802409CB40020EC1C0010F01C00107B
:1017700010B50400200004F0F1FC14F1380004F06E
:10178000EDFC14F1700004F0E9FC022084F8CC01B7
:10179000DFF860030460200000F016F8200010BDA0
:1017A00038B50400DFF84C0300210160250014F176
:1017B000700004F0D4FC14F1380004F0D0FC2000D8
:1017C00004F0CDFC280032BD10B504000020C4F8A0
:1017D000D4010020C4F8D8010020C4F8E0000020A3
:1017E000C4F8E4000020C4F8E8000020C4F8EC00CD
:1017F0000020C4F8F0000020C4F8F40094F8CC01F4
:1018000001283ED1DFF8F002D0F8B804C4F8F8009F
:10181000DFF8E402D0F8BC04C4F8FC00DFF8D8021A
:10182000D0F8C004C4F800010322032114F59E700F
:1018300004F058FD0322032114F5C27004F052FD98
:10184000D4F8F800C4F88C01D4F8F800C4F8A0016A
:10185000D4F8F800C4F8B401D4F8F800C4F8C8010A
:10186000D4F8F800C4F84401D4F8F800C4F85801DA
:10187000D4F8F800C4F86C01D4F8F800C4F880017A
:101880005BE0DFF87402D0F8B804FBF71FFDDFF867
:101890006C22DFF86C3204F03DFDFAF749FCC4F825
:1018A000F800DFF85402D0F8BC04FBF70FFDDFF8B6
:1018B0005422DFF8543204F02DFDFAF739FCC4F855
:1018C000FC00DFF83402D0F8C004FBF7FFFCDFF8BF
:1018D0003422DFF8343204F01DFDFAF729FCC4F895
:1018E00000010422042114F59E7004F0FBFC042284
:1018F000042114F5C27004F0F5FCD4F8F800C4F823
:101900008C01D4F8F800C4F8A001D4F8F800C4F8A9
:10191000B401D4F8F800C4F8C801D4F8F800C4F849
:101920004401D4F8F800C4F85801D4F8F800C4F819
:101930006C01D4F8F800C4F880015FF07E50C4F860
:1019400004010020C4F808010020C4F80C010020A4
:10195000C4F810019FED650A200004F08DFCB7EE7D
:10196000000A200004F08BFC9FED610A200004F0C7
:101970008CFCB2EE040A200004F084FC200004F089
:10198000EFFB9FED5A0A14F1380004F075FCB7EE36
:10199000000A14F1380004F072FC9FED550A14F1AE
:1019A000380004F072FCB2EE040A14F1380004F0BE
:1019B00069FC14F1380004F0D3FB9FED4C0A14F1DC
:1019C000700004F059FCB7EE000A14F1700004F046
:1019D00056FC9FED470A14F1700004F056FCB2EE7D
:1019E000040A14F1700004F04DFC14F1700004F0CE
:1019F000B7FBDFF80401406BFBF768FCDFF80C2154
:101A0000DFF80C3104F086FC00225FF0804304F024
:101A100053FD41EC100B04F072FE51EC100BFAF781
:101A200087FBC4F81C01DFF8D000406BFBF74EFCCD
:101A3000DFF8D820DFF8D83004F06CFC00225FF02B
:101A4000804304F039FD41EC100B04F061FE51ECD1
:101A5000100BFAF76DFBC4F820010020C4F8240134
:101A60000020C4F8280114F58E7004F05BFEDFF846
:101A70008800806BFBF72AFCDFF89020DFF89030BD
:101A800004F048FC00225FF0804304F015FD41ECB7
:101A9000100B04F034FE51EC100BFAF749FBC4F8BC
:101AA0002C010020C4F83001DFF84C00806BFBF7FC
:101AB0000DFCDFF85820DFF8583004F02BFC002232
:101AC0005FF0804304F0F8FC41EC100B04F020FEC2
:101AD00051EC100BFAF72CFBC4F834010020C4F8C9
:101AE000380114F5967004F01DFE10BD8FC2353F0D
:101AF0000000484450B4002010180010F168E3883A
:101B0000B5F8E43E2D431CEBE2361A3F4DC907778A
:101B100046DF913FDFF8301308607047DFF8281385
:101B200000220A60704730B585B004000D00DFF870
:101B3000580300884DF6FF710840DFF84C13088009
:101B40000095D2B2002A06D00020ADF80400002093
:101B5000ADF8080006E04FF48050ADF80400002016
:101B6000ADF808000020ADF806000020ADF80C002C
:101B70000C20ADF80A0000A9DFF8100302F05AFAB1
:101B8000DFF80403008850F02000DFF8FC12088022
:101B9000DFF8F402008850F40050DFF8EC120880FF
:101BA000E58005B030BD10B50400DFF8DC02008828
:101BB0004DF6FF710840DFF8D012088001215FF474
:101BC000002003F0FEF9002060700020A0700020CB
:101BD000E070002084F8900014F11000A06014F16F
:101BE0001000E0600020C4F894000020C4F89801C0
:101BF0000020C4F89C010F2020710120607110BDED
